:020000040800F2
:10800000D0C00020A1810008A981000879A900083A
:10801000AD810008AF810008B181000800000000B8
:10802000000000000000000000000000B381000814
:10803000B581000800000000B7810008B981000880
:10804000BB810008BB810008BB810008BB81000820
:10805000BB810008BB810008BB810008BB81000810
:10806000BB810008BB810008BB810008BB81000800
:10807000BB810008BB8100081F97000823970008F8
:10808000BB81000827970008BB810008BB8100085E
:10809000BB810008BB810008BB810008BB810008D0
:1080A000BB810008BB810008BB810008BB810008C0
:1080B0004D7E0108BB810008BB810008BB81000820
:1080C000BB810008BB810008BB810008BB810008A0
:1080D000BB810008198601081D8601082186010858
:1080E000DB9A0008BB810008BB810008BB81000847
:1080F000BB810008BB810008BB8100082B970008EA
:10810000BB810008BB810008BB810008BB8100085F
:108110001186010815860108BB810008BB81000893
:10812000BB810008BB810008BB810008BB8100083F
:10813000BB810008BB810008BB810008BB8100082F
:10814000BB810008BB810008BB810008BB8100081F
:10815000BB8100082F970008339700082586010887
:10816000BB810008BB810008BB810008BB810008FF
:10817000BB810008BB810008BB810008BB810008EF
:10818000BB810008BB810008DFF810D000F00CFCB8
:108190000048004741A30108AFF30080D0C0002091
:1081A0000648804706480047FEE7FEE7FEE7FEE791
:1081B000FEE7FEE7FEE7FEE7FEE7FEE7F17D0108EA
:1081C000898100082DE9F0410024061B254671F144
:1081D000000605DA01240027D0EB070067EB010158
:1081E000161E73F1000605DA0027D2EB07020125FF
:1081F00067EB030300F066FA86460E4617469C4678
:10820000AC4204D00025D0EB050E65EB010624B18D
:108210000020D2EB000760EB030C704631463A4673
:108220006346BDE8F081202A06DBCB17203A41FAED
:1082300002F043EAE07306E041FA02F3D040C2F1F3
:108240002002914008431946704740EA01039B070A
:1082500003D009E008C9121F08C0042AFAD203E0BB
:1082600011F8013B00F8013B521EF9D27047421E43
:1082700012F8013F002BFBD111F8013B02F8013B42
:10828000002BF9D17047421C10F8011B0029FBD1CB
:10829000801A704730B505460020034600E05B1C9D
:1082A000934205D2EC5CC85C201A01D1002CF6D1B7
:1082B00030BD2DE9FE4F804681EA0300C00F0C4619
:1082C000009021F0004123F00045B8EB0200A941E5
:1082D00005D24046214690461C460B46024623F0F6
:1082E0000040104347D0270DC7F30A00C3F30A51DB
:1082F0000290401A019040286BDAC3F3130040F457
:10830000801B0098924620B10023D2EB030A63EB56
:108310000B0B01985946C0F14002504600F003FA99
:1083200006460D4650465946019AFFF77CFF10EB72
:1083300008006141002487EA115284EAE7731A4376
:1083400040D0009A62B3019A012A4FEA075215DC25
:10835000001B61EB02014FF0004202EA0752CDE937
:108360000042001C41F5801132462B4600F08EFA87
:1083700003B0BDE8F08F40462146F9E7001B61EBF2
:108380000201001C41F5801300185B412018A2F582
:10839000001747EB030140EAD570B6196D4111E0B3
:1083A0006D084FEA360645EAC0754FEA0752001BD2
:1083B00061EB0201001C41F5801149084FEA3000D1
:1083C0000019514132462B4603B0BDE8F04F00F092
:1083D0004EBA0098012240000023D0EB020263EB6A
:1083E000E073009821464FEAE074B8EB000061EBBF
:1083F0000401E9E783F000435BE781F0004158E7BF
:108400002DE9FE4F81EA030404F0004421F000410D
:1084100000944FF0000B23F0004350EA01045ED0BB
:1084200052EA03045BD0C3F30A54C1F30A552C4447
:10843000A4F2F3340194A0FB0254C1F3130141F4FC
:108440008011C3F3130343F4801301FB024400FBC8
:10845000034E840A970A44EA815447EA8357A4FBEF
:10846000076802958D0A05FB07854FEA932C04FBEC
:108470000C542705029D4FEA065847EA1637B5EB1C
:1084800008056EEB070C870E920E47EA811742EA49
:108490008312A7FB0201B6EB0B0164EB00042B0D6A
:1084A00043EA0C335E1844EB1C50DA465146E7FBB6
:1084B0000201C5F313044FEA0B3343EA14534FEAA6
:1084C0000432019C43EA0603A4F10C040294009CCC
:1084D000CDE900B400F0DAF903B0BDE8F08F002078
:1084E0000146F9E72DE9F04D81EA030404F0004B61
:1084F00021F0004514464FF0000A23F0004150EAF5
:10850000050220D054EA01021DD0C5F30A570246E5
:10851000C5F31303C1F31300C1F30A5640F48015E9
:1085200043F48013A7EB0608101BD64608F2FD386B
:1085300073EB050002D308F1010801E092185B41DA
:10854000B8F1000F03DA00200146BDE8F08D0020ED
:108550004FF48011064684460EE0171B73EB0507A7
:1085600005D3121B63EB050306434CEA010C4908D3
:108570004FEA300092185B4150EA0107EDD152EA10
:10858000030012D082EA040083EA0501084305D003
:10859000101BAB4106D20122002306E000224FF05F
:1085A000004302E06FF0010253101AEB06004CEB9F
:1085B000085110EB0A0041EB0B01BDE8F04D00F053
:1085C00056B90EB540F2334102910021CDE90011B8
:1085D0000A460B4600F05AF903B000BD3EB5CA1773
:1085E000CB0F002450405140C0186141DA0740F2DF
:1085F00033430094CDE901232246234600F046F997
:1086000003B030BD70B5C1F30A5201F0004500243B
:10861000C1F3130140F2FF3341F480119A4201DAB1
:10862000002070BD40F233439A42A2F2334203DC91
:10863000524200F087F800E090402C43F1D04042D5
:1086400070BD70B5C1F30A5201F000450024C1F3BA
:10865000130140F2FF3341F480119A4202DA002004
:10866000014670BD40F233439A42A2F2334203DC2A
:10867000524200F067F801E000F055F82C43F0D0CA
:108680000023D0EB030063EB010170BD01F0004358
:1086900030B421F0004150EA010206D00A0DA2F5E3
:1086A0006072C1F31301002A02DC30BC0020704765
:1086B000440F44EAC104C100E01830BC00EBC250D2
:1086C00000F09EB82DE9F05F0546002092469B46DB
:1086D00088460646814640241BE0284641464746D8
:1086E000224600F02FF853465A46C01A914110D343
:1086F00011461846224600F016F82D1A67EB0108BD
:108700004F4622460120002100F00DF817EB00092A
:108710004E41201EA4F10104DFDC484631462A46C2
:108720004346BDE8F09F202A04DB203A00FA02F11C
:10873000002070479140C2F1200320FA03F319434F
:1087400090407047202A04DB203A21FA02F00021F1
:10875000704721FA02F3D040C2F120029140084351
:10876000194670470FB4002300B589B00CA90091D9
:108770000B996FF00042CB601E4B06931E4B079384
:108780000423CDE901321D4A089202466B460020BF
:1087900000F0B6F909B05DF814FB70B586B0064676
:1087A0004FF0FF300091CDE90101002015460C4645
:1087B00004903246694604A8FFF7D4FF02460498A5
:1087C000211825B108B1084600E020462860049829
:1087D00000280DD0002A02DD0098884208D0081B2E
:1087E0000094CDE901043246694604A8FFF7BAFFB8
:1087F00006B070BD398D0008578D0008CD8900087E
:108800000029A8BF7047401C490008BF20F00100A4
:10881000704710B4B0FA80FC00FA0CF050EA010482
:1088200004BF10BC704749B1CCF1200421FA04F414
:1088300011FA0CF118BF012121430843A3EB0C01ED
:10884000CB1D4FEA00614FEA102042BF002010BC50
:10885000704700EBC35010440029A4BF10BC704700
:10886000401C490008BF20F0010010BC704710B543
:10887000141E73F1000408DA401C41F10001921843
:108880005B411A4301D120F0010010BD2DE9F04DEC
:1088900092469B4611B1B1FA81F202E0B0FA80F241
:1088A00020329046FFF73FFF04460F4640EA0A0099
:1088B00041EA0B0153465A46084313D0114653EA86
:1088C000010019D0C8F140025046FFF73BFF0546B2
:1088D0000E46504659464246FFF725FF084305D04D
:1088E000012004E020463946BDE8F08D0020054314
:1088F00046EAE0762C4337430A986305E40AA0EB86
:1089000008000022FD0A44EA47540A3002D500203C
:108910000146E9E7010510196941DDE9084500193B
:108920006941BDE8F04DA2E770B521F00043034373
:108930000CD0C1F30A550024D5EB040564EB040305
:10894000D617AD1AB34102DB0020014670BD2018D6
:1089500041EB025170BD0EB5C10F80EAE0700844D2
:10896000CA07002140F233438DE80E000A460B4649
:10897000FFF78CFF03B000BD30B5041E71F1000499
:1089800004DB4FF00044404264EB0101141E73F11C
:10899000000405DB1C464FF00043524263EB040326
:1089A000994208BF904230BD064C074D06E0E06892
:1089B00040F0010394E8070098471034AC42F6D326
:1089C000FFF7E6FBE0CF010800D00108C0B24FF48A
:1089D000F05100F03BBA00002DE9FF4F087883B05A
:1089E0009946FF2805D0491C2D2804D000240020DA
:1089F00008E000200BE00124F9E700EB800003EB26
:108A00004000491C0B78FF2BF7D104B140420023F2
:108A10000293147819461D462D2C01D02B2C04D11D
:108A2000521C2D2C13D000240294AA461478FF2C3B
:108A30000FD00A25A3FB057801FB05814FF0000C40
:108A400003FB0C11521CE3194AEB0101EEE7012470
:108A5000EAE7814453EA010002D019F5C87F06DA3B
:108A600003980021C0E9001107B0BDE8F08F002590
:108A7000AE4E2F46DFF8B882184600F0FBF9CDE97C
:108A80000001B9F1000002DAC9F1000400E0044677
:108A90000023A74A1AEB030B42EB045A12E0E0074B
:108AA00007D02A46334638464146FFF7A9FC074619
:108AB00088462A46334610461946FFF7A1FC05466C
:108AC0000E466410002CEAD1DDE90001B9F1000F77
:108AD0005A46534606DAFFF705FD3A464346FFF786
:108AE00001FD05E0FFF78CFC3A464346FFF788FCA2
:108AF000029A0AB181F00041039AC2E90001B3E78A
:108B00002DE9FF4F1F468DB0D7E901464FF0FF38E2
:108B10002E2045464FF000090B90B9696D1C0E9848
:108B20008847396A824688470028F6D1BAF1FF3F64
:108B30000AD024F4D064002E11DDBAF12B0F08D036
:108B4000BAF12D0F0BD102E0404611B08DE744F48D
:108B50008064B9696D1C0E9888478246761E694606
:108B6000600501D52D2000E02B208DF8000001F1DB
:108B7000010B0DF1200809E0B9696D1C0E988847BA
:108B800082460F9844F40074761E0560002E02DDC4
:108B9000BAF1300FF0D00B998A453ED144F08004F1
:108BA00006E00F99681CA9F1010944F400740860FB
:108BB000B9696D1C761E0E98884782463028F0D021
:108BC0002BE00B998A4505D1200603D444F080049C
:108BD000761E18E0504611F00BF808B30DF11301A2
:108BE000761E44F400748B4508D2AAF130000BF8CD
:108BF000010B200607D5A9F1010003E0200602D4ED
:108C000009F101008146A00502D50F99681C086092
:108C1000B9696D1C0E9888478246002ED1DC53E05E
:108C2000002E51DDBAF1650F02D0BAF1450F4BD1DC
:108C3000A00549D5B9696D1C24F44074761E0E98C0
:108C400088478246002E0CDD2B2804D0BAF12D0F68
:108C500007D144F48074B9696D1C0E988847824628
:108C6000761EE00501D52D2100E02B2108F8011B1F
:108C7000CDF82C8021E00DF12901761E44F400741A
:108C800088450CD2AAF1300010F0FF0088F80000EF
:108C900002D10B99884509D908F1010806E0E005E1
:108CA00001D5244801E042F20F708146B9696D1C7C
:108CB0000E98884782460F980560002E04DD5046C6
:108CC00010F096FF0028D6D1F9690E988847FF204A
:108CD0008BF8000088F800000020069007904B46B3
:108CE0006A4608A906A8FFF777FEA00502D46FF030
:108CF00001002AE714F0240F0AD0E00714D1DDE9BF
:108D000006123868031D3B600068C0E900120BE0E2
:108D1000DDE90601FFF7BAFC0146E00704D1386837
:108D2000021D3A600068016028460EE7000014400A
:108D30000000F03FF1D8FFFF426842B1016811F82E
:108D4000013B23B1521EC0E90012184670470121B1
:108D5000C160881E704742685AB1C368016843B950
:108D600083688B4205D0491E521CC0E900120020C6
:108D700070474FF0FF3070472DE9F04D00231A4641
:108D80001B1A8A4103DB00200146BDE8F08DC1F3C8
:108D90000A52C1F3130141F480154FF0000BD107C3
:108DA00002D100186D41521E0027044640F2FF1107
:108DB000384601EB620A3E468046024600204FF4E8
:108DC0008011FFF7BFFCC2197141BB1846EB0100CF
:108DD000B4EB030C75EB000C04D3E41A65EB00054F
:108DE00017460E46241908F101006D4180463428CB
:108DF000E3DDF91946EB0600091BA84103D24FF049
:108E0000FF32134601E0002213461BEB070046EB3E
:108E10000A51BDE8F04DFFF72ABD000030B5041E31
:108E200071F1000404DB4FF00044404264EB0101A7
:108E3000141E73F1000405DB1C464FF00043524240
:108E400063EB04038B4208BF824230BD7F2801D907
:108E5000002208E0064A02EB5002C007127800D157
:108E6000120902F00F0201209040084070470000F4
:108E7000A0CF01080EB540F2334202920022CDE9A4
:108E800000221346FFF702FD03B000BD70B58C1839
:108E900010F8015B15F0070301D110F8013B2A110E
:108EA00006D110F8012B03E010F8016B01F8016BFB
:108EB0005B1EF9D12B0705D40023521E0DD401F8F7
:108EC000013BFAE710F8013BCB1A921C03E013F8C0
:108ED000015B01F8015B521EF9D5A142D8D30020F5
:108EE00070BD027803E010F8013B1A44D2B2491E6B
:108EF00089B2F8D21046704770B5ADF5287D0026CE
:108F00000D46ADF89462ADF8986200EB40012D4833
:108F100000EBC104608AA84251D9ADF898624AE0DA
:108F2000A089228A284481B2274800F0B1F8ADF820
:108F300094626A46208A0BE0BDF894326168C95C8D
:108F4000BDF89432D154BDF89412491CADF8941276
:108F5000BDF894128842EFD8401E81B21046FFF748
:108F6000C0FF1A498870228A0DF1FF31515C81429D
:108F700019D1ADF894620CE0BDF894126068BDF8A8
:108F80009422405CA1688854BDF89402401CADF85E
:108F90009402208ABDF89412401E8842ECDC012025
:108FA0000DF5287D70BD642011F05AF8BDF89802C7
:108FB000401CADF89802BDF898020628B0D30020F6
:108FC000EEE70000DCAD01083C7A00202212002010
:108FD000F0B50D46064600EB46011C48002200EBAA
:108FE000C104ADF5257D608AA8422BD9694606E00B
:108FF000A0686368805C98548854521C92B2208A9E
:10900000401E9042F4DC208A401E81B26846FFF781
:1090100068FF228A0DF1FF3100275054A089228A6F
:10902000284481B2684600F02FF929463046FFF700
:1090300063FF012807D0642011F012F87F1CBFB233
:10904000062FEBD300200DF5257DF0BDDCAD01082A
:1090500038B50025ADF800500DF08EF90A4C20709F
:1090600000F088F821780948242907D0272908D05A
:10907000282902D1022180F8A51138BD80F8A55118
:1090800038BD0121F7E7000022120020D422002081
:109090002DE9F041064615460C46012080F3108864
:1090A000254F0020B8800DF047F9000609D40120B3
:1090B00010F0D6FFB888401C80B2B880C828F2D320
:1090C00035E0B888C82832D21C4F1021384601F04C
:1090D000A6F90821384601F0A4F9E82000F030F89C
:1090E000C4F3871000F02CF8A006000E00F028F85A
:1090F000002000F025F80024002000F021F8641C76
:10910000A4B2042CF8D3002405E0FF2000F018F8E6
:109110003055641CA4B2AC42F7D31021384601F09C
:1091200080F9002080F310880120BDE8F081002044
:1091300080F31088F9E700002212002000000240AE
:1091400070B50B4C0546022120460DF00FFA0028A1
:10915000F9D0294620460DF012FA012120460DF0E3
:1091600005FA0028F9D020460DF007FAC0B270BD0C
:109170000030014010B5012080F310881A4C002007
:10918000A0800DF0D9F8000609D4012010F068FF86
:10919000A088401C80B2A080C828F2D320E0A0881C
:1091A000C8281DD2114C1021204601F038F90821A1
:1091B000204601F036F93D20FFF7C2FF2A20FFF7D5
:1091C000BFFF8020FFF7BCFFA720FFF7B9FF1021EA
:1091D000204601F026F9002080F31088012010BD00
:1091E000002080F3108810BD2212002000000240F1
:1091F0002DE9F04106460D46012080F31088204CF1
:109200000020A0800DF098F8000609D4012010F08D
:1092100027FFA088401C82B2A280C82AF2D32AE08D
:10922000A088C82827D2174F1021384601F0F7F838
:109230000821384601F0F5F88420FFF781FF00206F
:10924000FFF77EFF0020FFF77BFF0020FFF778FF8E
:10925000002404E0305DFFF773FF641CA4B2AC424D
:10926000F8D31021384601F0DCF8002080F3108894
:109270000120BDE8F081002080F31088F9E70000AC
:10928000221200200000024070B50D46012181F33A
:1092900010881146FFF7ACFF002832D01B4C00208D
:1092A000A0800DF049F8000609D4012010F0D8FE86
:1092B000A088401C80B2A080C828F2D322E0A088F9
:1092C000C8281FD2124C1021204601F0A8F808210E
:1092D000204601F0A6F88320FFF732FFC5F3871080
:1092E000FFF72EFFA806000EFFF72AFF0020FFF76A
:1092F00027FF1021204601F094F8002080F3108809
:10930000012070BD002080F3108870BD2212002063
:109310000000024010B500231A4604E010F8014B8B
:109320006340521CD2B28A42F8D3184610BD0000E6
:1093300010B50446392011F093F8E0B211F0B0F8FE
:10934000C4F3072011F0ACF8C4F3074011F0A8F8FB
:10935000200E11F0A5F84FF48051034801F061F898
:10936000BDE810400FF050BA000402402DE9F04172
:10937000054614460E463A2011F072F8F0B211F08C
:109380008FF8300A11F08CF8104F4FF480563146A8
:10939000384601F046F8B0463E460FF035FA1D2833
:1093A00011D1284600F0A4F807463B2011F058F8E8
:1093B0004146304601F035F83D44002CEDD0208880
:1093C00038442080E9E7BDE8F08100000004024055
:1093D0002DE9F041054614460E463C2011F040F8B8
:1093E000F0B211F05DF8300A11F05AF8114F4FF455
:1093F00080563146384601F014F80CB10020208028
:10940000B0463E460FF000FA1E2811D1284600F063
:1094100017F907463D2011F023F84146304601F088
:1094200000F83D44002CEDD0208838442080E9E746
:10943000BDE8F0810004024010B50CF0C5FE08B193
:1094400000F028F8BDE81040302000F09FB8014639
:10945000362000F089B810B508B100F0A5F8BDE8D5
:109460001040342000F092B810B5044600F09CF88B
:1094700020785C2801D02F2803D10021642000F03F
:10948000FBF8BDE81040322000F080B8682000F002
:109490004BB8000010B5222010F0E2FF10F0D6FF0C
:1094A00004464FF48051024800F0BBFF204610BD37
:1094B000000402402DE9F04110F0C8FF064610F00C
:1094C000C5FF054610F0C2FF044610F0BFFF074677
:1094D0004FF48051054800F0A4FF46EA052040EA19
:1094E000044040EA0760BDE8F0810000000402404B
:1094F00070B50546272010F0B3FF10F0A7FF044613
:10950000260007D010F0A2FF641E05F8010B14F02E
:10951000FF04F7D14FF48051024800F082FF30463B
:1095200070BD00000004024010B504460C2010F08D
:1095300097FF204610F0B4FFBDE81040FFF7BABF18
:1095400010B504460A2010F08BFF204610F0A8FF4B
:1095500010F07CFF04464FF48051024800F061FF98
:10956000204610BD0004024010B50C4610F078FFF4
:10957000204610F095FF4FF48051034800F051FF52
:10958000BDE810400FF040B90004024010B510F0E3
:1095900067FF4FF48051034800F043FFBDE81040DF
:1095A0000FF032B90004024070B50546012010F0FA
:1095B00057FF10F04BFF432828D22B20FFF7C0FFA6
:1095C000102823D22F2010F04BFF002010F068FF4E
:1095D0003220FFF7DBFF142818D1CF20FFF7B0FFB0
:1095E000040013D04C20FFF79FFF00EB04214C2018
:1095F00000F042F85020FFF797FF00EB04215020C5
:1096000000F03AF80021702000F036F82F2010F01A
:1096100027FF2C7806E015F8014F5C2C01D02F2C89
:1096200000D10024204610F03BFF002CF3D1BDE810
:1096300070404FF48051014800F0F3BE0004024036
:1096400070B505462D2010F00BFF10F0FFFE04460C
:10965000260007D0287810F023FF641E6D1C14F03C
:10966000FF04F7D14FF48051024800F0DAFE304693
:1096700070BD00000004024070B505460C460D2088
:1096800010F0EEFE284610F00BFFE0B210F008FFDD
:10969000C4F3072010F004FFC4F3074010F000FFEC
:1096A000200E10F0FDFEBDE870404FF480510148DF
:1096B00000F0B7BE0004024070B5094DFF2213460A
:1096C00005F5807605E010F8014B54402A5D5A40BC
:1096D000335D491E89B2F6D242EA032070BD000014
:1096E0006CAB010870B500221346154605E010F872
:1096F000014BA2186B41491E89B20029F7D1100C09
:1097000040EA034092B2801845EB13414FEA014210
:1097100042EA104108186FEA000080B270BD08F0FC
:109720009DBA08F03BBA08F009BA08F067BA00F031
:10973000BBBF0BF09DBC0000074A904201D2074816
:1097400001E005481038064A8B0001EA020101D504
:10975000C160704781607047106402400060024041
:109760007D0F7D0F0029016802D041F0010101E069
:1097700021F00101016070472DE9F043016821F0FB
:10978000010101600021016041608160C1600161EF
:10979000212141613C493C4A3D251039904202D18A
:1097A0008D60BDE8F083384A4FF4746618329042F9
:1097B00001D18E60F5E7344A4FF47417303290428D
:1097C00001D18F60EDE7304A4FF0746C483290421F
:1097D00002D1C1F808C0E4E72B4B2C4A6033984211
:1097E00001D1CA60DDE7284C294B7834A04201D171
:1097F000CB60D6E7DFF89080264C08F19008404512
:1098000001D1CC60CDE7DFF880804FF03D5908F101
:10981000A808404502D1C1F80C90C2E71E49DFF804
:1098200078800839404501D10D60BAE71A4D1835E6
:10983000A84201D10E60B4E7174D3035A84201D1DE
:109840000F60AEE7144D4835A84202D1C1F800C000
:10985000A7E7114D10496035091FA84201D10A60E0
:109860009FE70D4A7832904201D10B6099E70A4A8E
:109870009032904201D10C6093E7074AA83290429F
:109880008FD1C1F800908CE7106002403D000020AD
:10989000400F002000003D20106402400B0607D559
:1098A000436912B143F0800301E023F08003436178
:1098B000802908D0002A026801F01E0101D00A4365
:1098C00000E08A430260704730B50368124ACC68F2
:1098D00013400A682243D1E905452C432243CC6951
:1098E00022430C6A22434C6A22438C6A22434C6B0B
:1098F00022438C6B22431A430260426922F0070321
:10990000D1E90B2422431A4342610A6942604A6842
:1099100082608968C16030BD3F801CF02DE9FC4148
:10992000012120200CF058FC01268DF80460002550
:109930008DF8065003208DF805001B4C302700974A
:109940008DF807506946204600F016FD302120466C
:1099500000F067FD154C84F8305684F8325684F8D0
:10996000316684F833664FF4FA70C4F8380600F0B4
:109970001FF894F8A803802814D1A4F580504565F9
:10998000232084F8AD03052084F8AC0384F8AB737E
:10999000142084F8AA03202084F8A90384F8A8538B
:1099A00000F042F8BDE8FC8100140240D4220020FF
:1099B0007CB510F029FCD02010F0F6FB10F058FC1C
:1099C000002010F0F1FB10F053FC10F01DFCD12032
:1099D00010F0EAFB10F04CFC00246D4601E0062C70
:1099E00001D2012000E0002010F0AEFB2855641CDD
:1099F000E4B2072CF3D310F021FC0A489DF80610BE
:109A000041719DF8051001719DF80410C1709DF819
:109A1000021081709DF8011041709DF800100170D6
:109A20007CBD00007C2600207CB51848002401780D
:109A30008DF8001041788DF8011081788DF80210B2
:109A400001218DF80310C1788DF8041001798DF88B
:109A5000051040798DF8060010F0D6FBD02010F0EC
:109A6000A3FB10F005FC002010F09EFB10F000FCA2
:109A70006D46285D10F098FB10F0FAFB641CE4B210
:109A8000072CF6D310F0DAFB7CBD00007C2600200A
:109A900070B5094D0022134605F5807605E010F8F3
:109AA000014B54402A5D5A40335D491E89B2F6D2BB
:109AB00042EA032070BD00006CAB0108072A00D900
:109AC000072240EA002021B1012901D1D040C0B2D3
:109AD00070479040C0F3072070477047072A00D9AD
:109AE000072240EA002029B1012902D19040C0F3A9
:109AF00007207047D040C0B27047000070B5ADF588
:109B0000327D00260D46ADF8BC62ADF8C06200EBB8
:109B10004001324800EBC104608AA8425CD9ADF82C
:109B2000C06255E0012264212D4800F0A9F92C48BB
:109B300000788DF80000382842D1228AE06802FBC4
:109B40000501274800F09CF9ADF8BC626A46208AFE
:109B50000BE0BDF8BC326168C95CBDF8BC32D154C1
:109B6000BDF8BC12491CADF8BC12BDF8BC1288424D
:109B7000EFD8401E81B2104600F044FA228A0DF15F
:109B8000FF31515C81421BD1ADF8BC620EE0BDF8E3
:109B9000BC226168895CA26800FB0520BDF8BC227C
:109BA0001154BDF8BC02401CADF8BC02208ABDF8BF
:109BB000BC12401E8842EADC01200DF5327D70BDEA
:109BC000642010F04DFABDF8C002401CADF8C00290
:109BD000BDF8C0020628A5D30020EEE760A9010861
:109BE00060550020F0B50E46074600EB47012648B9
:109BF000ADF5317D002500EBC1048DF8BC52608AC3
:109C0000B0423DD900210846FFF778FF012837D13F
:109C1000694609E0A268401E00FB06206268285CD5
:109C2000505548556D1CADB2208AA842F2D8002587
:109C3000208AE16800FB0611401E82B2134800F042
:109C40009DF9208A401E81B2684600F0DBF98DF84C
:109C5000BC02208AE168012201447043401E014495
:109C6000AFA800F08BF931463846FFF747FF0128CF
:109C700007D0642010F0F4F96D1CADB2062DD7D3D7
:109C800000200DF5317DF0BD60A901086055002070
:109C9000F0B5ADF5317D2C4D00208DF8BC022B4E7A
:109CA000288000243FE000206F4607E056F832206D
:109CB0004968125C0A543A54401C80B2298801EB6E
:109CC000410206EBC2010B8A5B1E8342EEDC288850
:109CD00000EB400006EBC000008A401E81B238460F
:109CE00000F090F98DF8BC02288800EB400006EBEC
:109CF000C000C168008A00FB0411401E82B21448F3
:109D000000F03CF92888012200EB400006EBC0007F
:109D1000C168008A01446043401E0144AFA800F0BE
:109D20002DF9641CA4B2288800EB400006EBC000AB
:109D3000408AA042B7D82888401C80B228800A28D0
:109D4000AFD30DF5317DF0BD1000002060A90108F2
:109D5000605500207CB5012108460CF03DFA012039
:109D60008DF8040002258DF8055000248DF806407A
:109D70008DF807001820154E00906946304600F017
:109D8000FBFA05221146304600F032FB052206217F
:109D9000304600F02DFB05220721304600F028FB5D
:109DA000A02000908DF8045003208DF805008DF858
:109DB00006408DF807406946304600F0DDFA402045
:109DC00000906946304600F0D7FA7CBD00000240A2
:109DD000F8B5002634460096FFF7BCFF00F0A0F867
:109DE0002248641C8442FCD3214C0821204600F008
:109DF00016FB1021204600F014FB062000F076F838
:109E00000821204600F00DFB0821204600F007FB4A
:109E10001021204600F005FB012000F067F800202B
:109E200000F064F80821204600F0FBFA1148D0F851
:109E30001C0208B9FFF72CFF0F4D2E800F4E002497
:109E400005E0C0B22146FFF759FE641CA4B2288881
:109E500000EB400106EBC101498AA142F1D880B272
:109E6000401C80B228800A28E9D3F8BDFFFF0F000C
:109E700000000240000043421000002060A90108D9
:109E80002DE9F0410546002416460F46012080F3D7
:109E90001088DFF854800821404600F0C0FA1021F5
:109EA000404600F0BEFA032000F020F8C7F3074058
:109EB00000F01CF8C7F3072000F018F8F8B200F023
:109EC00015F806E0002000F011F8641C05F8010BFD
:109ED000A4B2B442F6D30821404600F0A2FA002012
:109EE00080F31088BDE8F0810000024070B50B4C93
:109EF0000546022120460CF039FB0028F9D02946FE
:109F000020460CF03CFB012120460CF02FFB0028E2
:109F1000F9D020460CF031FBC0B270BD00300140DA
:109F200010B5012186B008030CF092F9124C2046BE
:109F30000CF0F2FA0021ADF808106015ADF80A0037
:109F40003820ADF80C000720ADF80010ADF8100077
:109F5000ADF804104FF48270ADF80610ADF80E1095
:109F6000ADF80200694620460CF00BFB01212046AB
:109F70000CF0C8FA06B010BD003001402DE9F041E8
:109F80000546002416460F46012080F31088DFF8AE
:109F900070800821404600F042FA1021404600F04F
:109FA00040FA0620FFF7A2FF0821404600F039FAE8
:109FB0000821404600F033FA1021404600F031FA03
:109FC0000220FFF793FFC7F30740FFF78FFFC7F3A8
:109FD0000720FFF78BFFF8B2FFF788FF05E028782E
:109FE000FFF784FF641CA4B26D1CB442F7D30821B0
:109FF000404600F016FA002080F31088BDE8F0819A
:10A0000000000240027803E010F8013B1A44D2B28B
:10A01000491E89B2F8D210467047000070B51E4A3A
:10A02000907A012825D1002595721C491C480F24DF
:10A030004E780123F6B14D70D0F82852D0F8346232
:10A0400045EAC605D0F83062D0F82C02B60046EAE0
:10A0500040000543AC43CC708878CC78A04208D14E
:10A0600008710C78A04204D0D0710870002800D08C
:10A07000937170BD4B70D0F82852D0F8346245EA25
:10A08000C605D0F83062D0F82C02B60046EA40008F
:10A090000543AC438C70DFE7D4120020C9120020C6
:10A0A000000042422DE9F041ADF57C7D00273D46A0
:10A0B000ADF8E873FFF7C0F9142808D0664880F8B7
:10A0C000A75310F009F90DF57C7DBDE8F0816348D8
:10A0D000FFF7CAF9614C103C1428207006D04228C2
:10A0E00079D00120FFF7B3F92570ECE7FFF7CEF93F
:10A0F000C4E90205A046BDF8E803FFF719F9FAAA7A
:10A100004FF4FA716846FFF731F955A1684610F02F
:10A1100047F9A080544C6E46F0B1E11901F5805129
:10A1200081F8FD567F1CBFB2282FF6D34746304436
:10A130004EA110F035F978800021001F0AE0BA889E
:10A140000A443244D378621802F5805282F8FD3610
:10A15000491C89B28142F2DB45A1684610F020F922
:10A160004746A8F80400F0B10021621802F58052B9
:10A1700082F82557491C89B22829F6D330443BA1DF
:10A1800010F00EF97880002109380AE0BA880A44F4
:10A190003244137A621802F5805282F82537491C3E
:10A1A00089B28142F2DB35A1684610F0F9F8B88037
:10A1B000F8B10021621802F5805282F84D57491C0F
:10A1C00089B21429F6D3304428A110F0E9F8788038
:10A1D00000210D380BE03AE0BA880A443244137B80
:10A1E000621802F5805282F84D37491C89B28142CB
:10A1F000F2DB26A1684610F0D3F8B880F0B1002158
:10A20000621802F5805282F8B756491C89B2322989
:10A21000F6D3304415A110F0C3F878800021C01F98
:10A220000AE0BA880A4432449379621802F58052EF
:10A2300082F8B736491C89B28142F2DB0021032043
:10A24000FFF7D0FC0120FFF702F901203BE70348AC
:10A25000FFF701F937E70000D42200203812002070
:10A2600041504E3D00000000D41200203B00000091
:10A27000574946494E414D453D0000005749464922
:10A2800050415353574F52443D00000053455256DE
:10A2900045523D002F4910B5884206D1012108469C
:10A2A0000BF0A6FF002101204FE02B49884206D188
:10A2B000012102200BF09CFF0021022045E02749EC
:10A2C000884206D1012104200BF092FF00210420D6
:10A2D0003BE02349884206D1012108200BF088FF8A
:10A2E0000021082031E01F49884206D101211020B9
:10A2F0000BF07EFF0021102027E01B49884206D189
:10A30000012120200BF074FF002120201DE01749BF
:10A31000884206D1012140200BF06AFF0021402035
:10A3200013E01349884206D1012180200BF060FF21
:10A330000021802009E00F4988420AD184150121BB
:10A3400020460BF055FF00212046BDE810400BF0E1
:10A350004FBF10BD00000240000402400008024050
:10A36000000C02400010024000140240001802409D
:10A37000001C024000200240F0B5002201274FF0EF
:10A38000030C0B6807FA02F52B40AB422CD1066890
:10A3900053000CFA03F4A64306600E79D0F800E0EF
:10A3A0009E4046EA0E0606600E79012E01D0022E6E
:10A3B00012D18668A64386604E79D0F808E09E40A8
:10A3C00046EA0E0686604668AE43466045688E796A
:10A3D0009640B6B235434560C568A543C560CC79A3
:10A3E0009C40C3681C43C460521C102AC9D3F0BDF2
:10A3F0004B07DB0E9A40C90810B500EB8100016ADB
:10A400000F249C40A1430162016A1143016210BD07
:10A410000246002012690A4200D0012070474183A1
:10A4200070470183704700002DE9F04F7C4E0025F6
:10A430002DED028B85B030782C46012852D14FF09B
:10A44000000986F8009006F1020898F80000DFF88D
:10A45000D4A14FF0010BF52804D098F819004F282B
:10A460007DD080E098F8021098F8010041EA0024BD
:10A470006B482146801CFFF71FF908EB040149785F
:10A4800018F8042041EA022181422BD198F80310E8
:10A49000654FF1292BD06548F22953D0F32921D1FA
:10A4A0004C4680F8889280F87CB2F520387087F8A6
:10A4B00001900520B870F320F870592038710521FB
:10A4C0005948FFF7F9F8010A7971B87158480760DF
:10A4D0005749072008390860554801210C38FFF713
:10A4E00041F9747005B0BDEC028BBDE8F08F5246A7
:10A4F000511901F5805181F8FD966D1CADB2282DE2
:10A50000F6D30020241F09E008EB00010B79111895
:10A5100001F5805181F8FD36401C80B2A042F3DB8A
:10A5200000210320FFF75EFB0028DBD00AF000FFCC
:10A53000F52038704C4687F801900520B870F1205E
:10A54000BAE70CE080F888B280F87DB2F520387068
:10A550004C4687F801900520B870F220ACE798F8D7
:10A560001A004B281CD02E4832A1801C0FF018FF77
:10A57000060002D002218AF8021008EB0607B87B19
:10A580002D4D41280FD0B87B5628ABD14846C5F891
:10A59000799785F87D97C5F8799785F87D07A1E7C4
:10A5A0008AF802B09EE76946C146321902EB0900FB
:10A5B000027C0A55641C8846A4B24046092CF4D398
:10A5C0000EF062F951EC100BFEF760F800EE100A85
:10A5D0009FED1A8A1A484A46C0EE080AC0EDDD0A05
:10A5E000B87E85F8780700204146331813441B7F56
:10A5F0000B54401C80B20928F7D368460EF044F98A
:10A6000051EC100BFEF742F800EE100AC0EE080AFB
:10A6100010EE900AC5F8790797F82700BDE700000B
:10A6200012000020D4120020FC030020D45200208D
:10A63000AC640240524D4300D42200200000C842C6
:10A64000D426002070B5144C40F2244631462046F2
:10A650000EF04DF800281ED0314620460DF0E4FFE4
:10A660000E4D00212846FFF77DF8314620460DF0BB
:10A67000DBFF0B492846FFF75FF82088201D008884
:10A68000291D4FF47A70086001212846FFF76AF807
:10A6900004490120087070BD001401402864024084
:10A6A000008800101200002010B5104C0E49204602
:10A6B000FFF742F800212046FFF754F80C4C4021E8
:10A6C00020460EF00DF80028F9D0084C0949783CD6
:10A6D0002046FFF731F801212046FFF743F80649ED
:10A6E0000120487010BD000000802020A0640240BE
:10A6F0000014014000880010120000202DE9F043F2
:10A7000001218FB088050BF067FDDFF88C9048467B
:10A71000FFF732F84020050103900024CDE90545FC
:10A72000C60207940894CDE909461C4F0B944FF0DC
:10A730002068CDE900870C940D94694648460E9434
:10A74000FFF7C2F8012210214846FFF7A7F8DFF80B
:10A750004890A9F178094846FFF70EF84FF47A704F
:10A76000CDE90340CDE9054507940894CDE90946B4
:10A770000B480B940C940D94CDF800800E94CDE909
:10A78000017069464846FFF79FF801214846FEF7E9
:10A79000E9FF0FB0BDE8F083A0640240041401405B
:10A7A000140000207CB5012104200BF015FD164E8D
:10A7B000082206213046FFF71BFE082207213046FB
:10A7C000FFF716FE02218DF8051000258DF80650C2
:10A7D0000124C0208DF8074000908DF804106946D0
:10A7E0003046FFF7C9FD600200908DF804408DF8F7
:10A7F000065003208DF805008DF807406946304665
:10A80000FFF7BAFD7CBD0000000802402DE9F041D1
:10A81000FFF7C8FF4FF4E13000F078F8FFF76EFF64
:10A8200000F056F82448002505708570012141701C
:10A83000C17042F210718160214E20483060204F7B
:10A840000E20083F3860A7F1040801214046FEF7BA
:10A8500089FF1C4C657060780028FCD04FF4FA70BA
:10A860000FF0FEFB4FF4165000F050F81349002093
:10A87000154A103101EB000C135C401CC0B28CF87F
:10A8800008300A28F6D3114A0020131803F5805324
:10A8900093F8F93601EB000C401CC0B28CF8133071
:10A8A0000428F2D331601920386001214046FEF7B8
:10A8B00059FF6570BDE8F0813C2A0020E4070020C4
:10A8C000AC64024012000020B0A40108D4120020A1
:10A8D00038B545208DF8000002208DF801000124D4
:10A8E0008DF802408DF80340684607F003FF4720CB
:10A8F0008DF800008DF8014000208DF802008DF8E1
:10A900000340684607F0F6FE38BD00001FB5044658
:10A91000012120200BF09CFC0020ADF804000094E5
:10A92000ADF80600ADF80800ADF80C000C200D4C99
:10A93000ADF80A00694620460DF010FF01212046BF
:10A940000DF075FE012240F2244120460DF0EEFE8E
:10A95000102120460DF068FE0122C02120460DF096
:10A9600070FE1FBD001401400249C8790022CA715F
:10A9700070470000D412002002480068C00700D0D1
:10A9800000BEFEE7F0ED00E002494AF6AA200860AA
:10A99000704700000030004010B50FF09DFCBDE88E
:10A9A000104064200FF05CBB2DE9F04F83466AA095
:10A9B000ADF57D7D002500689A460F46A946FB90BF
:10A9C000ADF8E853042A25D8644C94F8AC03302140
:10A9D00001EB101302EBC20000EB021260481618E4
:10A9E000337194F8AC0300F00F003030707194F8BC
:10A9F000AB0301EB1010B07194F8AB0300F00F0043
:10AA00003030F071FEF718FD142807D084F8A793B2
:10AA10000FF062FC0DF57D7DBDE8F08FDFF8408121
:10AA2000A8F1240898F8000014280ED03046FEF74C
:10AA30001BFD88F80000142807D042287ED0012092
:10AA4000FEF705FD88F80090E4E74FF47A7087423E
:10AA500000D90746FEF71AFDC8E902094E46FEF77F
:10AA600067FC94F8AB13302000EB11118DF8001047
:10AA700094F8AB1301F00F0130318DF8011094F808
:10AA8000AA1300EB11118DF8021094F8AA1301F02B
:10AA90000F0130318DF8031094F8A91300EB111158
:10AAA0008DF8041094F8A91301F00F0130318DF8DE
:10AAB000051094F8A81300EB11108DF8060094F817
:10AAC000A80300F00F0030308DF80700BAF1000F36
:10AAD00003D0BAF1010F02D004E0542000E052206C
:10AAE0008DF808003A208DF809000A236C4617E01B
:10AAF0000BEB550108780009B0FBF3F2C2EBC20280
:10AB00001044621930309072087800F00F00B0FBEA
:10AB1000F3F1C1EBC10108443030AD1CD072ADB2CD
:10AB2000B5EB470FE4D303EB470081B2FAAA204606
:10AB3000FEF74EFCFAAA0221FBA800E007E0FEF7B0
:10AB400047FC0120FEF783FC88F8006062E730468E
:10AB5000FEF781FC5EE700000D0A0000D422002011
:10AB60004C1200202DE9F04F00272DED028BA1B0F3
:10AB70008DF828708DF800708DF82070CDE912776F
:10AB8000CDE900778DF808708DF80C708DF8107095
:10AB90008DF81470ADF818709FEDFE0A0797DFF876
:10ABA000F8938DED070AFD4C41F6823504F125003E
:10ABB0000C9004F59C5004F5804A01264FF0D50B0B
:10ABC000DFF8DC8304F580540B90A0E094F8B20A1F
:10ABD00028B384F8B27ABAF83812D9F88C204846EB
:10ABE000C2F57A7291421AD1D0F88C00C0F57A7011
:10ABF000AAF83002E84800218830FEF7B3FDE648A5
:10AC0000E8498830FEF798FD88F800604FF47A70C4
:10AC1000C9F88C00E04801218830FEF7A3FD94F8C4
:10AC2000BE0A20B384F8BE7ABAF83A12D9F84420A2
:10AC30004846C2F57A72914219D1406CC0F57A70DB
:10AC4000AAF83202D44800214030FEF78BFDD248EA
:10AC5000D5494030FEF770FD88F801604FF47A70F6
:10AC6000C9F84400CC4801214030FEF77BFD94F840
:10AC7000CA0A20B384F8CA7ABAF83C12D9F8142068
:10AC80004846C2F57A72914219D14069C0F57A708E
:10AC9000AAF83402C04800211030FEF763FDBE4818
:10ACA000C2491030FEF748FD88F802604FF47A710F
:10ACB000C9F81410B84801211030FEF753FD94F87C
:10ACC000D60A20B384F8D67ABAF83E12D9F82C20E6
:10ACD0004846C2F57A72914219D1C06AC0F57A70BD
:10ACE000AAF83602AC4800212830FEF73BFDAA48FE
:10ACF000AF492830FEF720FD88F803604FF47A70E2
:10AD0000C9F82C00A44801212830FEF72BFD94F847
:10AD1000B20A94F8BE1A084494F8CA1A94F8D62ACB
:10AD20001144C8427FF452AF05F0E7BC017819B175
:10AD300007708DF8087010E0417819B147708DF8F0
:10AD400008600AE0817811B18770022003E0C178C1
:10AD500019B1C77003208DF808009DF8080000EBBA
:10AD6000400101EB00118D4800EB011000F580500F
:10AD700090F8561B9DF8080000EB4002C2EBC01291
:10AD80008C4810F83200C1280BD19DF8080000EB68
:10AD90004002C2EBC012874800EBC200807808284E
:10ADA0000CD0082985F07484DFE811F0201F2700FB
:10ADB0005D098512211AC51B4C1F3A238AF8886247
:10ADC0009DF8080030B1012807D002280FD00328D1
:10ADD00008D10FE04FF4804101E04FF40051764874
:10ADE000FFF71DFB7548C0F8887205F051BC4FF4A1
:10ADF0008051F4E74FF40061F1E79DF80800DFF8B7
:10AE0000B48100EB4001C1EBC01108EBC1004078F8
:10AE1000002106F0C5FD8DF810008DF82070DFF8D8
:10AE20007C911BE09DF808009DF8201000EB40028B
:10AE300002EB001009EB001000EB011000F5805050
:10AE400090F8810B9DF8101088429DF8200002D1E7
:10AE50008DF8100012E0401C8DF820009DF80800CD
:10AE600000EB400101EB001009EB001000F58050F1
:10AE700090F8570B9DF820209042D3D89DF80800F9
:10AE800000EB4001C1EBC01008EBC00080780A2243
:10AE9000B2EB101F9DF8080000EB4002C2EBC0109F
:10AEA00008EBC000807801D100F00F008DF80C0095
:10AEB0009DF80C0010B910208DF80C009DF80800CA
:10AEC0009DF80C1000EB4002C2EBC01208EBC20070
:10AED00008444078ADF818009DF8080000EB4001E8
:10AEE000C1EBC01108EBC1009DF80C10491C07F024
:10AEF0003CF98DF800009DF8080000EB4001C1EB23
:10AF0000C01108EBC1009DF80C10084480789DF832
:10AF10000010884245F0BC839DF80800424600EBD3
:10AF20004001C1EBC01008EBC0004078002805F0DC
:10AF3000AF839DF8080000EB4001C1EBC0109DF805
:10AF40000C1002EBC0000844C1789DF8080000EB2B
:10AF5000001303EB002309EBC30C9DF810304846A7
:10AF600003EB03130CEBC30303F5005383F85410F6
:10AF70009DF808109DF8103009EB0111194401F5F6
:10AF8000805181F8107BBDF81810CE2929D029DC1A
:10AF9000B92915E00000000000600240D412002032
:10AFA0001008002000880020008020102080001061
:10AFB00000880010AC6200200018024000004242ED
:10AFC0007ED008DC5A29B2D0B2297AD0B529F7D080
:10AFD000B6299FD1FEE3C32974D0C52973D0CA29ED
:10AFE00098D1F8E3E129FCD006DCD52909D0D7298E
:10AFF0009DD0D9298ED17CE2E52965D0E72989D178
:10B00000EAE39DF8081001EB4103C3EBC11108EB23
:10B01000C101C97884F8A2119DF80810C84601EB57
:10B02000410202EB0112014600EB02109DF81020D4
:10B0300000EB021094F8A2212844A6EBD213027868
:10B0400063F3000202709DF8080000EB400202EB7F
:10B0500000109DF8102001EB001000EB021094F896
:10B06000A22128445309027863F3410202709DF83B
:10B07000080000EB400202EB001001EB00129DF80B
:10B08000100002EB001000F5805090F8820BC0F326
:10B0900040029DF8080000EB001303EB002008EBD2
:10B0A000C0019DF8100000EB001001EBC00000F59E
:10B0B000005090F83000C0F34000824255D004E0C8
:10B0C000E8E3F4E3AFE3F3E3F3E39DF8080000EB18
:10B0D000001101EB002008EBC0029DF81000414672
:10B0E00000EB001002EBC00042F2300210449DF869
:10B0F000082002EB420303EB02129DF8103008EB2C
:10B10000021202EB031202F5805292F8822B5308CE
:10B11000027863F3410202709DF8080000EB4002E0
:10B1200002EB00109DF8102001EB001000EB021064
:10B1300000F5805090F8820B800717D59DF8080025
:10B14000D92200EB001303EB002008EBC0019DF8AF
:10B15000100000EB001001EBC00000F5005042773A
:10B160009DF808100220FEF73DFD46E09DF808001E
:10B1700000EB001202EB002001EBC0029DF8100072
:10B1800000EB001002EBC00000F5005080F82560D5
:10B190009DF80800D92200EB001303EB002001EB1F
:10B1A000C0039DF8100000EB001003EBC00000F599
:10B1B000005042779DF8080000EB400202EB0010BF
:10B1C00001EB00129DF8100002EB001042191078FC
:10B1D00020F0200313709DF8080000EB001202EB32
:10B1E000002008EBC0019DF8100000EB001001EBFF
:10B1F000C00000F5005080F856609DF808004346F6
:10B2000000EB400101EB001008EB00119DF810006D
:10B2100001EB001000F5805090F8820B00F0010166
:10B220009DF8080000EB001202EB002008EBC002C2
:10B230009DF8100000EB001002EBC00000F500507C
:10B2400090F8300000F00100814204F04E849DF837
:10B2500008009DF8102000EB001101EB00201946BA
:10B2600003EBC00002EB021200EBC20042F230021C
:10B2700010449DF8082002EB420303EB02129DF8F4
:10B28000103001EB021202EB031202F5805292F829
:10B29000822B037862F3000303709DF8080000EB33
:10B2A000400202EB00109DF8102001EB001000EBB3
:10B2B000021000F5805090F8820BC0079DF808003E
:10B2C00039D000EB001202EB002001EBC0029DF828
:10B2D000100000EB001002EBC00000F5005090F8E9
:10B2E000560000289DF8080000EB001202EB002039
:10B2F00001EBC0029DF8100000EB001002EBC00053
:10B3000000F5005028D080F855709DF8080000EB3B
:10B31000400202EB001001EB00129DF8100002EB5E
:10B3200000104219107820F00103137094F862079E
:10B33000A8B104F0DABB00EB400202EB00109DF86C
:10B34000102001EB001000EB02102844027822F0DC
:10B350002003037004F0FEBA80F85560E6E7087D2C
:10B360000128E6D1486DCA8A9042E2D29DF80800D1
:10B3700000EB001202EB002001EBC0029DF8100070
:10B3800000EB001002EBC00000F5005090F85500F3
:10B390000128CED19DF8080000EB001202EB00203E
:10B3A00001EBC0029DF8100000EB001002EBC000A2
:10B3B00000F5005090F88F000028BAD19DF80800E1
:10B3C00000EB400202EB001001EB00129DF81000B0
:10B3D00002EB001000F5805090F8802B9DF80800DB
:10B3E00000EB001303EB002001EBC00000F5005060
:10B3F00042749DF80800C32200EB001303EB002009
:10B4000001EBC0039DF8100000EB001003EBC0003F
:10B4100000F5005042779DF8080000EB400202EB77
:10B42000001008EB00119DF8100001EB001000F572
:10B430008050C0F8847B9DF808100220FEF7D2FBF4
:10B440008DF82870414619E09DF8080000EB0012C5
:10B4500002EB002001EBC0029DF8100000EB001091
:10B4600002EBC0029DF82800104400F5005080F85F
:10B4700057709DF82820521C8DF828209DF8280030
:10B480001428E1D38DF8287019E09DF8080000EB2E
:10B49000001202EB002001EBC0029DF8100000EB4F
:10B4A000001002EBC0009DF82820104400F5005069
:10B4B00080F873709DF82800401C8DF828009DF8D6
:10B4C00028000A28E1D334E79DF8080000EB0012B9
:10B4D00002EB002001EBC0029DF8100000EB001011
:10B4E00002EBC00000F50050007E012804F0258327
:10B4F0007BE49DF80810C84601EB410303EB011102
:10B5000009EB011000F5805090F85C0B00289DF8C5
:10B510000C0002D00A28EBD195E00828E8D18DF87C
:10B52000287024E09DF8080000EB4001C1EBC0103A
:10B530009DF8281002EBC0000844C07800F00F000E
:10B54000092818D89DF8080000EB4001C1EBC01095
:10B550009DF8281002EBC0000844C07800F0F0000D
:10B56000902808D89DF82800401C8DF828009DF8E8
:10B5700028000628D6D39DF828000628B8D39DF8C1
:10B58000080000EB4001C1EBC01002EBC000C07826
:10B5900001049DF8080000EB4003C3EBC01002EB70
:10B5A000C000007941EA00239DF8080000EB40014B
:10B5B000C1EBC01002EBC000407903439DF80800C6
:10B5C00000EB001101EB002008EBC00C9DF810000F
:10B5D000414600EB00100CEBC00000F50050C0F835
:10B5E00031309DF8080000EB4003C3EBC01002EBC4
:10B5F000C000807903049DF8080000EB400CCCEB00
:10B60000C01002EBC000C07943EA00239DF8080097
:10B6100000EB400CCCEBC01002EBC000007A0343FF
:10B620009DF8080000EB001202EB002001EBC001C6
:10B630009DF8100000EB001001EBC00000F5005079
:10B64000C0F83530A8E08DF8287024E09DF8080097
:10B6500000EB4001C1EBC01002EBC0019DF82800D7
:10B660000844C07800F00F00092818D89DF8080099
:10B6700000EB4001C1EBC0109DF8281002EBC000A8
:10B680000844C07800F0F000902808D89DF8280001
:10B69000401C8DF828009DF828000828D6D39DF876
:10B6A00028000828C4F0F4879DF8080000EB40014A
:10B6B000C1EBC01002EBC00081799DF8080000EBDF
:10B6C0004003C3EBC01002EBC000C07841EA006148
:10B6D0009DF8080000EB4003C3EBC01002EBC00074
:10B6E000007903049DF8080000EB400CCCEBC0107F
:10B6F00002EBC000407943EA002001439DF80800B6
:10B7000000EB001303EB002008EBC0039DF81000D2
:10B7100000EB001003EBC00000F50050C0F8311042
:10B720009DF8080000EB4001C1EBC01002EBC00027
:10B73000817A9DF8080000EB4003C3EBC01002EBD8
:10B74000C000C07941EA00619DF8080000EB4003A9
:10B75000C3EBC01002EBC000007A03049DF80800A0
:10B7600000EB400CCCEBC01002EBC000407A43EA87
:10B77000002001439DF8080000EB001202EB0020BE
:10B7800008EBC0029DF8100000EB001002EBC000B7
:10B7900000F50050C0F835109DF8080000EB0011CE
:10B7A00001EB002008EBC0029DF81000414600EBC1
:10B7B000001002EBC00000F50050007E032804F0EA
:10B7C00065839DF8080000EB400202EB001001EBDE
:10B7D000001202E06EE0CAE3F4E39DF8100002EB11
:10B7E000001004F046BB9DF8080000EB001303EBCB
:10B7F000002008EBC00104F0DDBB9DF8080000EB61
:10B80000001202EB002001EBC0029DF8100000EBDB
:10B81000001002EBC00000F5005090F8260001284F
:10B8200004F0538364E69DF8081001EB011303EB69
:10B83000012100EBC1039DF8101001EB011103EB96
:10B84000C10101F5005181F81DB09DF8081001EB10
:10B85000011202EB012100EBC10101F50051CE7490
:10B860009DF8081001EB410202EB011109EB0110F8
:10B870009DF8101000EB01102844017841F02001E0
:10B88000F0E39DF8081001EB011303EB012109EB34
:10B89000C101B0E79DF8081001EB011202EB012194
:10B8A00000EBC10101F50051CF74C322E9E7ADE01F
:10B8B000D3E05EE39DF8081001EB410303EB0111B7
:10B8C00000EB011101F5805191F85C1B00299DF8F6
:10B8D000081001EB4103C3EBC11102EBC10158D0C9
:10B8E000C9780B049DF8081001EB410CCCEBC11199
:10B8F00002EBC101097943EA01239DF8081001EB2D
:10B90000410CCCEBC11108EBC10149790B439DF807
:10B91000081001EB011202EB012100EBC1029DF8BE
:10B92000101001EB011102EBC10101F50051CB64D4
:10B930009DF8081001EB011202EB012100EBC1029E
:10B940009DF8101001EB011102EBC10101F500514E
:10B95000097E02293BD09DF80810C52201EB011396
:10B9600003EB012100EBC1039DF8101001EB011165
:10B9700003EBC10101F500514A779DF8081001EB76
:10B98000011202EB012109EBC10000F50050C77460
:10B99000AEE50B799DF8081001EB410CCCEBC11121
:10B9A00008EBC101C97843EA01229DF8081001EBB8
:10B9B000011303EB012100EBC1039DF8101001EB13
:10B9C000011103EBC10101F50051CA64B0E79DF814
:10B9D000081001EB011202EB012100EBC10101F59E
:10B9E0000051CF749DF80810032201EB011303EB03
:10B9F000012100EBC1039DF8101001EB011103EBD5
:10BA0000C10101F500510A76D922F3E29DF8081030
:10BA100001EB011202EB012100EBC10101F5005124
:10BA2000CE749DF8081001EB011303EB012100EB2C
:10BA3000C1039DF8101001EB011103EBC10101F5E9
:10BA4000005181F81DB09DF8081001EB410202EB96
:10BA5000011109EB011004F083BB9DF80810CE46DC
:10BA600001EB410303EB011109EB011000F58050DC
:10BA700090F85C0B00289DF80C0002D00E2887D1AE
:10BA8000A0E00C2884D18DF8287024E09DF80810DF
:10BA900001EB4100C0EBC1109DF8281002EBC00083
:10BAA0000844C07800F00F00092818D89DF8081045
:10BAB00001EB4100C0EBC11002EBC0019DF8280072
:10BAC0000844C07800F0F000902808D89DF82800BD
:10BAD000401C8DF828009DF828000A28D6D39DF830
:10BAE00028000A28C4F0D4850020CDE9000038469B
:10BAF0008DF828701FE0DDE900131B0243EA116393
:10BB00000902CDE900139DF8081001EB4103C3EBD6
:10BB1000C1119DF8283002EBC1011944C978DDE953
:10BB2000003C194340EA0C03CDE900139DF82810AE
:10BB3000491C8DF828109DF828100529DBD3DDE974
:10BB4000003C9DF8081001EB011808EB01210EEBF9
:10BB5000C1099DF81010F04601EB011109EBC1017C
:10BB600001F50059C9F839304946C1F83DC00023F4
:10BB7000CDE900338DF828001FE0DDE900131B023A
:10BB800043EA11630902CDE900139DF8081001EBA7
:10BB90004103C3EBC1119DF8283002EBC1011944E8
:10BBA000097ADDE9003C194340EA0C03CDE90013B2
:10BBB0009DF82810491C8DF828109DF8281005299B
:10BBC000DBD39DE08DF8287024E09DF8081001EB90
:10BBD0004100C0EBC1109DF8281002EBC0000844E2
:10BBE000C07800F00F00092818D89DF8081001EB64
:10BBF0004100C0EBC1109DF8281002EBC0000844C2
:10BC0000C07800F0F000902808D89DF82800401C6B
:10BC10008DF828009DF828000C28D6D39DF8280020
:10BC20000C28C4F035850020CDE9000038468DF899
:10BC300028701FE0DDE900131B0243EA11630902CB
:10BC4000CDE900139DF8081001EB4103C3EBC111CE
:10BC50009DF8283002EBC1011944C978DDE9003CA8
:10BC6000194340EA0C03CDE900139DF82810491C44
:10BC70008DF828109DF828100629DBD3DDE9003C5B
:10BC80009DF8081001EB011808EB01210EEBC1092A
:10BC90009DF81010F04601EB011109EBC10101F50F
:10BCA0000059C9F839304946C1F83DC00023CDE9F3
:10BCB00000338DF828001FE0DDE900131B0243EA82
:10BCC00011630902CDE900139DF8081001EB41034F
:10BCD000C3EBC1119DF8283002EBC1011944497A28
:10BCE000DDE9003C194340EA0C03CDE900139DF85F
:10BCF0002810491C8DF828109DF828100629DBD340
:10BD0000DDE900129DF8080000EB001303EB0020B2
:10BD100008EBC0039DF8100000EB001003EBC0001F
:10BD200000F50053C3F841101846C0F845209DF8AF
:10BD30000800F04600EB001101EB00200EEBC00202
:10BD40009DF8100000EB001002EBC00000F5005061
:10BD5000027E9DF8080000EB001303EB00200EEBC1
:10BD6000C00000F50050007D824244F0018494F848
:10BD70006207E0BBC8F835709DF8080000EB0011C1
:10BD800001EB00219DF8100008EBC10100EB001051
:10BD900001EBC00042F23901014410220C98FCF77B
:10BDA00054FA9DF8080000EB001101EB00219DF80A
:10BDB000100008EBC10100EB001001EBC0003130B6
:10BDC00000F500504146026841F8192F406848606C
:10BDD0009DF8080000EB400101EB001108EB011099
:10BDE0009DF8101000EB011000F5805000E040E0DD
:10BDF00090F8801B88F818100B998A6AC8F83920C7
:10BE0000898DA8F83D109DF8080000EB001101EBAA
:10BE100000219DF8100008EBC10100EB001001EBC0
:10BE2000C00000F50050C16CC8F821109DF8080052
:10BE300000EB400101EB001108EB01109DF8101020
:10BE400000EB011000F58050D0F8841BC8F83F10BB
:10BE5000D8F8540081B20220FDF7BAF8002106207C
:10BE6000FDF7C0FED8F85410491CC8F8541004F06F
:10BE700078BB9DF8080000EB400101EB001108EBD6
:10BE800001109DF8101000EB01102844017841F0DA
:10BE9000080101709DF80810022004F064BB9DF8B1
:10BEA000080000EB001101EB002008EBC0029DF838
:10BEB0001000414600EB001002EBC00000F50050FE
:10BEC00080F856709DF8080000EB001303EB00208B
:10BED00008EBC0039DF8100000EB001003EBC0005E
:10BEE00000F5005080F81DB09DF8080000EB00122E
:10BEF00002EB002001EBC0029DF8100000EB0010E7
:10BF000002EBC00000F50050007E042844F0C0831E
:10BF10009DF8080000EB400202EB00109DF8102095
:10BF200001EB001000EB02102844027842F080027E
:10BF300002709DF8080000EB001202EB002001EBFC
:10BF4000C00000F50050C6749DF80800052200EB03
:10BF5000001303EB002008EBC0019DF8100000EB7C
:10BF6000001001EBC00000F5005002765AE45A467A
:10BF700087E484F8A0669DF8081001EB011202EB3B
:10BF8000012100EBC1029DF8101001EB011102EB41
:10BF9000C10101F50051097E00299DF8081001EB4F
:10BFA000011202EB01210ED000EBC1029DF810102E
:10BFB00001EB011102EBC10101F50051897EB229AB
:10BFC00026D02FE44BE000EBC10101F50051CF7406
:10BFD0009DF8081001EB011202EB012100EBC102F8
:10BFE0009DF8101001EB011102EBC10101F50051A8
:10BFF0000E765A469DF8081001EB011303EB012160
:10C0000009EBC10304F00FBB00F50050427709E4CF
:10C010009DF8081001EB011202EB012100EBC101B8
:10C0200001F50051CF749DF80810B22201EB011305
:10C0300003EB012100EBC1039DF8101001EB01118E
:10C0400003EBC10101F500514A779DF8081001EB9F
:10C05000011202EB012109EBC10204F010BB84F8CC
:10C06000A07684E7C0E39DF8080000EB4001C1EB37
:10C07000C010FE4911F83000042809D09DF80800CE
:10C0800000EB4002C2EBC01011F83000152801D1BE
:10C09000ADF818009DF80800F44900EB4002C2EB2F
:10C0A000C01001EBC00042789DF8080000EB40038F
:10C0B000C3EBC01011F8300042EA0020A0F5805117
:10C0C000303922D09DF8080000EB4001C1EBC010D0
:10C0D000E64901EBC00042789DF8080000EB400300
:10C0E000C3EBC01011F8300042EA0020A0F58052E6
:10C0F000313A0CD09DF8080000EB4002C2EBC010B2
:10C1000011F83000022804D019E0A62015E0A7207D
:10C1100013E09DF8080000EB4002C2EBC01001EBF9
:10C12000C00002799DF8080000EB4003C3EBC0108B
:10C1300001EBC000C07842EA0020ADF818009DF87D
:10C140000800DFF82C9300EB001101EB002109EB54
:10C15000C10101F500518A7C8DF810209DF808106E
:10C1600009EB01109DF81010084400F5805080F88C
:10C17000107BBDF8180043F23002811A90427DD046
:10C1800009DC04287BD015287AD0A6280DD0A72852
:10C1900044F07E82FBE0B1F5C06F72D0A1F5C061C2
:10C1A00001396FD00429F3D1FEE39DF8080000EBBC
:10C1B000001101EB002009EBC00000F500504946DA
:10C1C000C7749DF8080000EB001202EB002009EB99
:10C1D000C0029DF8100000EB001002EBC00000F55B
:10C1E0000050007E032839D09DF8080000EB0012B3
:10C1F00002EB002001EBC0029DF8100000EB0010E4
:10C2000002EBC00000F50050007E082840D09DF8E9
:10C21000080000EB001202EB002001EBC0029DF8C9
:10C22000100000EB001002EBC00000F50050007E93
:10C230000D2841D09DF8080000EB001202EB002011
:10C2400001EBC0029DF8100000EB001002EBC000F3
:10C2500000F50050407FA52842D052E09DF808002C
:10C26000042200EB001303EB002001EBC0039DF858
:10C27000100000EB001003EBC00004E011E16DE1E1
:10C2800015E338E374E300F500500276A82265E375
:10C290009DF80800092200EB001303EB002001EBDE
:10C2A000C0039DF8100000EB001003EBC00000F588
:10C2B00000500276A92251E39DF808000E2200EBFF
:10C2C000001303EB002001EBC0039DF8100000EB0E
:10C2D000001003EBC00000F500500276A2223DE3FF
:10C2E0009DF8080000EB400202EB00109DF81020C2
:10C2F00001EB001000EB02102844027842F0040227
:10C3000002709DF8080000EB001202EB002001EB28
:10C31000C0029DF8100000EB001002EBC00000F519
:10C320000050807EA12804F0B3819DF8080000EB46
:10C33000001202EB002001EBC0029DF8100000EBA0
:10C34000001002EBC00000F50050827E9DF808004E
:10C3500000EB001303EB002001EBC0039DF810007D
:10C3600000EB001003EBC00000F5005042779DF891
:10C370000800A12200EB001303EB002009EBC00131
:10C380009DF8100000EB001001EBC000FDE39DF8EC
:10C39000080000EB001101EB002009EBC00000F5E4
:10C3A00000504946C7749DF8080000EB001202EBEC
:10C3B000002009EBC0029DF8100000EB001002EB1A
:10C3C000C00000F50050007E05289DF8080000EB35
:10C3D000001202EB00200DD001EBC0029DF810000E
:10C3E00000EB001002EBC00000F50050007E0928B1
:10C3F00007D018E001EBC00000F50050C77406221A
:10C4000000E00A229DF8080000EB001303EB002077
:10C4100001EBC0039DF8100000EB001003EBC0001F
:10C4200000F5005002769DF8080000EB001202EBC8
:10C43000002001EBC0029DF8100000EB001002EBA1
:10C44000C00000F50050407FA42828D19DF80800C6
:10C4500000EB400202EB00109DF8102001EB0010F1
:10C4600000EB02102844027804E00000AC620020D7
:10C47000D412002042F0200202709DF8080000EB68
:10C48000001202EB002001EBC0029DF8100000EB4F
:10C49000001002EBC00000F5005080F85570A1229A
:10C4A0005CE28DF8287014A9FE4A13E09DF808009C
:10C4B00000EB4003C3EBC0109DF8283002EBC00036
:10C4C0001844C0789DF82830C8549DF82800401CB6
:10C4D0008DF828009DF828000628E7D3062114A827
:10C4E0000DF0D4FDCDE91207129A000A8018B84663
:10C4F00047EB08014FF480720023FBF763FE9DF8C1
:10C50000080000EB001101EB002009EBC0039DF8CF
:10C51000100000EB001003EBC00000F500500277A4
:10C520009DF8080000EB001202EB002009EBC000B0
:10C5300000F5005080F813809DF8080000EB001211
:10C5400002EB002009EBC0029DF8100000EB001088
:10C5500002EBC00000F500500676FEE19DF80800F1
:10C5600000EB001101EB002009EBC0029DF8100068
:10C57000494600EB001002EBC00000F50050007EC1
:10C5800006282ED19DF8080000EB001202EB0020D7
:10C5900001EBC00000F50050C7749DF808000722A9
:10C5A00000EB001303EB002001EBC0039DF810002B
:10C5B00000EB001003EBC00000F5005002769DF880
:10C5C0000800A72200EB001303EB002001EBC003DF
:10C5D0009DF8100000EB001003EBC00000F50050C8
:10C5E00042779DF8080000EB001202EB002001EBFF
:10C5F000C0029DF8100000EB001002EBC00000F537
:10C600000050007E01289DF8080000EB001202EBAC
:10C61000002059D001EBC0029DF8100000EB001083
:10C6200002EBC00000F50050007E07289DF80800CE
:10C6300000EB001202EB00204DD001EBC0029DF890
:10C64000100000EB001002EBC00000F50050007E6F
:10C650000B289DF8080000EB001202EB002053D0DD
:10C6600001EBC0029DF8100000EB001002EBC000CF
:10C6700000F50050007E0C289DF8080000EB001229
:10C6800002EB002058D001EBC0029DF8100000EB37
:10C69000001002EBC00000F50050007E0E2852D0C2
:10C6A0009DF8080000EB001202EB002001EBC00235
:10C6B0009DF8100000EB001002EBC00000F50050E8
:10C6C000007E0F287DD051E401EBC00000F5005042
:10C6D000C774022205E001EBC00000F50050C774EA
:10C6E00008229DF8080000EB001303EB002001EB8B
:10C6F000C0039DF8100000EB001003EBC00000F534
:10C7000000500276A32229E101EBC00000F50050A1
:10C71000C7749DF808000C2200EB001303EB002007
:10C7200001EBC0039DF8100000EB001003EBC0000C
:10C7300000F500500276B2E601EBC00000F50050B3
:10C74000C7740D22CDE79DF808000F2200EB0013FF
:10C7500003EB002001EBC00C9DF8100000EB001073
:10C760000CEBC00000F5005002769DF80800A122F5
:10C7700000EB001303EB002001EBC00C9DF8100050
:10C7800000EB00100CEBC00000F5005042779DF864
:10C79000080000EB001303EB002001EBC00C9DF838
:10C7A000100000EB00100CEBC00000F5005082768A
:10C7B0009DF8080000EB400202EB001001EB0010B6
:10C7C00000E013E09DF8102000EB021028440278EE
:10C7D00042F0800202709DF8080000EB400202EB7C
:10C7E000001009EB0010FDE3017010E49DF8080053
:10C7F00000EB001202EB002001EBC0029DF81000DC
:10C8000000EB001002EBC00000F50050807EA12874
:10C810002ED09DF80800A32200EB001303EB0020AC
:10C820009DF8103001EBC00003EB031300EBC300D5
:10C8300000F5005042779DF8080000EB001202EB73
:10C84000002001EBC0029DF8100000EB001002EB8D
:10C85000C00000F50050807EA228C6D09DF80800D8
:10C8600000EB001202EB002009EBC000FFF78DB8CF
:10C870009DF80800A12200EB001303EB002001EB60
:10C88000C0039DF8100000EB001003EBC00000F5A2
:10C89000005042779DF8080000EB001202EB0020E8
:10C8A00002E00000AC62002009EBC000FDE39DF84F
:10C8B0000800A12200EB001101EB002009EBC003EE
:10C8C0009DF8100000EB001003EBC00000F50050D5
:10C8D00082769DF8080000EB001303EB002009EBC3
:10C8E000C0039DF8100000EB001003EBC00000F542
:10C8F00000504277B2E79DF8080000EB001101EB11
:10C90000002009EBC0029DF81000494600EB001022
:10C9100002EBC00000F50050007E062843F0B88608
:10C920009DF8080000EB001202EB002001EBC000B4
:10C9300000F50050C7749DF80800072200EB0013B3
:10C9400003EB002001EBC0039DF8100000EB00108A
:10C9500003EBC00000F500500276A7229DF8080006
:10C9600000EB001303EB002009EBC00103F022BB36
:10C970009DF8080000EB001101EB002109EBC1015B
:10C9800001F500514846CF749DF80810A72201EB2D
:10C99000011303EB012109EBC1039DF8101001EB1A
:10C9A000011103EBC10100E0FDE201F500514A77FE
:10C9B0009DF80810DFF804CD01EB4102C2EBC11174
:10C9C0000CEBC101497930299DF8081001EB4102B7
:10C9D00044D0C2EBC1110CEBC101497931299DF85A
:10C9E00008107DD001EB4102C2EBC1110CEBC1017B
:10C9F000497933299DF8081001EB410271D0C2EB4F
:10CA0000C1110CEBC101497934299DF8081001EBE3
:10CA1000410202EB01119DF8102000EB011101EB26
:10CA2000021129440A7871D022F001020A709DF89F
:10CA3000081001EB410202EB011100EB01129DF81D
:10CA4000101002EB01114A19117821F00203137042
:10CA50000021CDE900118DF82870D3E102EB01111E
:10CA60009DF8102000EB011101EB021129440A7816
:10CA700022F001020A709DF8081001EB410202EB5E
:10CA800001119DF8102000EB011101EB0211294466
:10CA90000A7822F002020A709DF8081001EB0112D8
:10CAA00002EB012100EBC1029DF8101001EB011116
:10CAB00002EBC10101F50051C97E3129C8D19DF8B1
:10CAC000081001EB410202EB011100EB01129DF88D
:10CAD000101002EB01114A19117821F0200301E036
:10CAE00015E026E113709DF8081001EB011202EB2E
:10CAF000012100EBC1029DF8101001EB011102EBC6
:10CB0000C10101F5005181F85570A1E731E101EB58
:10CB1000011202EB012100EBC1029DF8101001EBA4
:10CB2000011102EBC10101F5005191F856100029E5
:10CB30009DF8081001EB011202EB012100EBC1028C
:10CB40009DF8101001EB011102EBC10101F500513C
:10CB50007ED081F855709DF8081001EB410202EB80
:10CB6000011100EB01129DF8101002EB01114A199E
:10CB7000117821F0010313709DF8081001EB4102B8
:10CB800002EB011100EB011100E0FDE39DF8102024
:10CB900001EB021129440A7822F002020A7094F88B
:10CBA00062170029B1D1017D0129AED1416DC28A40
:10CBB0009142AAD29DF8081001EB011202EB01216B
:10CBC00000EBC1029DF8101001EB011102EBC10155
:10CBD00001F5005191F85510012996D19DF80810E2
:10CBE00001EB011202EB012100EBC1029DF81010D4
:10CBF00001EB011102EBC10101F5005191F88F1019
:10CC00000029CFD19DF808104FF0104201EB01131D
:10CC100003EB012100EBC1039DF8101001EB0111A2
:10CC200003EBC10101F500510A629DF8081001EB08
:10CC3000410202EB011100EB01129DF8101002EB12
:10CC4000011101F5805191F8802B9DF8081000E04A
:10CC50005CE001EB011303EB012100EBC10101F5E5
:10CC600000514A749DF8081001EB011202EB0121FA
:10CC700000EBC1029DF8101001EB011102EBC101A4
:10CC800001F500510A7E9DF8081001EB011303EB3A
:10CC9000012100EBC10101F50051097D8A4284D1D7
:10CCA0009DF8081001EB011202EB012100EBC1021B
:10CCB0009DF8101001EB011102EBC10101F50051CB
:10CCC0008F779DF80810A42201EB011303EB0121DB
:10CCD00000EBC1039DF8101001EB011103EBC10142
:10CCE00001F500518A769DF80810A32201EB01138B
:10CCF00003EB012100EBC1039DF8101001EB0111C2
:10CD000003EBC10101F500514A77A1E681F85560B6
:10CD10009DF8081001EB410202EB011100EB01123A
:10CD20009DF8101002EB01114A19117841F001032E
:10CD300021E702EB01119DF8102000EB011101EB3E
:10CD4000021129440A7842F001020A709DF8081085
:10CD500001EB410202EB011100EB01129DF81010F2
:10CD600002EB01114A19117841F002031370A2225B
:10CD700014E022F020020A709DF8081001EB410235
:10CD800002EB011100EB01129DF8101002EB0111F2
:10CD90004A19117821F002031370A9229DF8081096
:10CDA00001EB011303EB012100EBC1039DF810100F
:10CDB00001EB011103EBC10101F500518A7647E651
:10CDC000DDE90012120142EA11720901CDE90012F7
:10CDD0009DF8081001EB4102C2EBC1119DF828201B
:10CDE0000CEBC10111448979DDE900383039CA17EB
:10CDF000194342EA0802CDE900129DF82810491CA7
:10CE00008DF828109DF828100629D9D39DF8081010
:10CE1000009A01EB011303EB012100EBC1039DF824
:10CE2000101001EB011103EBC10101F50051C1F834
:10CE300031200022CDE900228DF8287021E0DDE9C3
:10CE40000012120142EA11720901CDE900129DF8A7
:10CE5000081001EB4102C2EBC1119DF828200CEB38
:10CE6000C1011144497BDDE900383039CA17194343
:10CE700042EA0802CDE900129DF82810491C8DF8FD
:10CE800028109DF828100429D9D39DF80810009A7D
:10CE900001EB011303EB012100EBC1039DF810101E
:10CEA00001EB011103EBC10101F50051CA6400223D
:10CEB000CDE900228DF8287021E0DDE90012120191
:10CEC00042EA11720901CDE900129DF8081001EB48
:10CED0004102C2EBC1119DF828200CEBC1011144A5
:10CEE000497CDDE900383039CA17194342EA0802A3
:10CEF000CDE900129DF82810491C8DF828109DF8E6
:10CF000028100629D9D39DF80810009A01EB0113C7
:10CF100003EB012100EBC1039DF8101001EB01119F
:10CF200003EBC10101F50051C1F835209DF808104F
:10CF300001EB4102C2EBC1110CEBC1014A799DF832
:10CF4000081001EB011303EB012100EBC1039DF875
:10CF5000101001EB011103EBC10101F50051CA767C
:10CF60009DF8081001EB410202EB011100EB0112E8
:10CF70009DF8101002EB011101F5805191F8822B00
:10CF80009DF8081001EB011303EB012100EBC10335
:10CF90009DF8100000EB001003EBC00000F50050FE
:10CFA00080F8302021E49DF8080000EB001101EB2F
:10CFB000002009EBC00000F50050C7749DF8080080
:10CFC00000EB001202EB002009EBC0019DF81000FD
:10CFD00000EB001001EBC00000F50050007E0A28B5
:10CFE00077D000E0FDE39DF8080000EB001101EBB5
:10CFF000002009EBC0029DF81000494600EB00102C
:10D0000002EBC00000F50050027E9DF8080000EB26
:10D01000001303EB002009EBC00000F50050007D79
:10D02000824213D194F86207F0B39DF808009DF88E
:10D03000101000EB400202EB001009EB001000EBB7
:10D0400001102844017841F0080101709DF80800A2
:10D05000A72100EB001202EB002009EBC0029DF8B3
:10D060001000CC4600EB001002EBC00000F50050B1
:10D0700041779DF80800A22100EB001202EB00208E
:10D0800009EBC0029DF8100000EB001002EBC0009D
:10D0900000F5005081769DF8080000EB001101EBCF
:10D0A00000200CEBC00101E026E0F8E39DF8100041
:10D0B00000EB001001EBC00000F5005080F8567046
:10D0C0000021CDE900118DF82870DFF8F085A1E08E
:10D0D000FFE79DF808000B2100EB001202EB002295
:10D0E0009DF8100009EBC20200EB001002EBC0003B
:10D0F00000F500500176A9E7C846C1F835709DF8E3
:10D10000080000EB001101EB00219DF8100009EB75
:10D11000C10100EB001001EBC00042F239010144F3
:10D1200010220C98FBF791F89DF8080000EB001115
:10D1300001EB00219DF8100008EBC10100EB00108D
:10D1400001EBC000313000F500504146026841F863
:10D15000192F406848609DF8080000EB400101EB82
:10D16000001108EB01109DF8101000EB011000F504
:10D17000805090F8801B88F818109DF8080000EB8C
:10D18000001101EB00219DF8100008EBC10100EB3C
:10D19000001001EBC00000F50050C16CC8F8211070
:10D1A0000B9940468A6A40F8392F898D8180D8F8DA
:10D1B000540081B20220FBF70BFF00210620FCF790
:10D1C00011FDD8F85400401CC8F854000021052077
:10D1D000FCF708FD3AE7090141EA10710001CDE9C9
:10D1E00000019DF8080000EB4001C1EBC0109DF864
:10D1F000281008EBC0000844C07ADDE9002330386D
:10D20000C11710431943CDE900019DF82800401CC7
:10D210008DF828009DF828000A28DDE90001DAD3FE
:10D220009DF8082002EB021303EB02220CEBC20371
:10D230009DF8102002EB021203EBC20202F500532C
:10D24000C3F839001A46C2F83D100020CDE90000AD
:10D250008DF8287020E0DDE90001090141EA107134
:10D260000001CDE900019DF8080000EB4001C1EB91
:10D27000C0109DF8281008EBC0000844407DDDE98F
:10D2800000233038C11710431943CDE900019DF840
:10D290002800401C8DF828009DF828000A28DAD3C1
:10D2A000DDE900129DF8080000EB001303EB0020FD
:10D2B0000CEBC003EBE39DF8080000EB4001C1EB71
:10D2C000C010FE4911F83000042809D09DF808006C
:10D2D00000EB4002C2EBC01011F83000152801D15C
:10D2E000ADF818009DF80800894600EB4002C2EB3B
:10D2F000C01001EBC00042789DF8080000EB40032D
:10D30000C3EBC01011F8300042EA0020A0F58051B4
:10D31000303922D09DF8080000EB4001C1EBC0106D
:10D3200009EBC000494642789DF8080000EB400335
:10D33000C3EBC01019F8300042EA0020A0F580527B
:10D34000313A0CD09DF8080000EB4002C2EBC0104F
:10D3500011F83000022804D01BE0A62017E0A72017
:10D3600015E09DF8080000EB4002C2EBC01001EB95
:10D37000C00002799DF8080000EB4003C3EBC01029
:10D3800009EBC000C07800E02CE142EA0020ADF8D3
:10D3900018009DF8080000EB001101EB0021C848BF
:10D3A00000EBC10101F500518A7C8DF810209DF839
:10D3B000081000EB01129DF81010114401F5805186
:10D3C00081F8107BBDF81810A7297DD007DC04294F
:10D3D0007BD015297AD0A62943F05A813AE001F58D
:10D3E0001D61B1F5804104D0112970D01229F3D10B
:10D3F000FEE39DF8081001EB011202EB012100EBA6
:10D40000C1029DF8101001EB011102EBC10101F501
:10D410000051097E0029DFD19DF8081001EB0112AF
:10D4200002EB012100EBC10101F50051CF749DF821
:10D43000081001EB011202EB012100EBC1029DF883
:10D44000101001EB011102EBC10101F500510E7644
:10D45000A72288E19DF8081001EB011202EB0121DF
:10D4600000EBC10101F50051CF749DF8081001EBEC
:10D47000011202EB012100EBC1029DF8101001EB3B
:10D48000011102EBC10101F50051097E02292BD0E7
:10D490009DF8081001EB011202EB012100EBC10223
:10D4A0009DF8101001EB011102EBC10101F50051D3
:10D4B000097E05292CD09DF8081001EB011202EB22
:10D4C000012100EBC10203E090E0DBE006E229E28B
:10D4D0009DF8101001EB011102EBC10101F50051A3
:10D4E000497FA52928D038E09DF80810032201EBD8
:10D4F000011303EB012100EBC1039DF8101001EBB8
:10D50000011103EBC10101F500510A76A9222AE1BC
:10D510009DF80810062201EB011303EB012100EB3B
:10D52000C1039DF8101001EB011103EBC10101F5DE
:10D5300000510A76A22216E19DF8081001EB410283
:10D5400002EB01119DF8102000EB011101EB02111B
:10D5500029440A7842F004020A709DF8081001EB91
:10D56000011202EB012100EBC1029DF8101001EB4A
:10D57000011102EBC10101F50051897EA12903F0DF
:10D5800087809DF8081001EB011202EB012100EBEE
:10D59000C1029DF8101001EB011102EBC10101F570
:10D5A00000518A7E9DF8081001EB011303EB012165
:10D5B00000EBC1039DF8101001EB011103EBC10159
:10D5C00001F500514A779DF80810A12201EB0113E3
:10D5D00003EB012100EBC1039DF8100000EB0010EC
:10D5E00003EBC00000F500508276DBE49DF80810E4
:10D5F00001EB011202EB012100EBC1029DF81010BA
:10D6000001EB011102EBC10101F50051497FA42991
:10D6100022D19DF8081001EB410202EB01119DF8A7
:10D62000102000EB011101EB021129440A7842F0AD
:10D6300020020A709DF8081001EB011202EB012193
:10D6400000EBC1029DF8101001EB011102EBC101CA
:10D6500001F5005181F855709DF8081001EB011299
:10D6600002EB012100EBC10101F50051CF749DF8DF
:10D670000810A12201EB011303EB012100EBC10112
:10D6800002F098BC9DF8081001EB011202EB012199
:10D6900000EBC1029DF8101001EB011102EBC1017A
:10D6A00001F50051097E01299DF8081001EB0112D6
:10D6B00002EB012138D000EBC10203E0AC62002094
:10D6C000D41200209DF8101001EB011102EBC101F2
:10D6D00001F50051097E04299DF8081001EB0112A3
:10D6E00002EB012127D000EBC1029DF8101001EBE5
:10D6F000011102EBC10101F50051097E06299DF8D7
:10D70000081001EB011202EB012136D000EBC1023F
:10D710009DF8101001EB011102EBC10101F5005160
:10D72000097E072978D03DE400EBC10101F50051E5
:10D73000CF74022205E000EBC10101F50051CF7466
:10D7400005229DF8081001EB011303EB012100EB0A
:10D75000C1039DF8101001EB011103EBC10101F5AC
:10D7600000510A76A3229DF8081001EB011303EB88
:10D77000012100EBC10302F056BF00EBC10101F52E
:10D780000051CF749DF80810072301EB011202EB42
:10D79000012100EBC10C9DF8101001EB01110CEB05
:10D7A000C10101F500510B769DF80810A12301EB92
:10D7B000011202EB012100EBC10C9DF8101001EBEE
:10D7C00001110CEBC10101F500514B779DF80810D8
:10D7D00001EB410202EB011100EB01119DF8102059
:10D7E00000E00EE001EB021129440A7842F08003C8
:10D7F0000B709DF8081001EB410202EB011100EBE8
:10D8000001109DF8101000EB01102844017841F040
:10D810000401FEF7E9BFFFE79DF8081001EB0112D4
:10D8200002EB012100EBC1029DF8101001EB011188
:10D8300002EBC10101F50051897EA12930D09DF88C
:10D840000810A32201EB011303EB01219DF8103016
:10D8500000EBC10103EB031301EBC30101F5005120
:10D860004A779DF8081001EB011202EB012100EB51
:10D87000C1029DF8101001EB011102EBC10101F58D
:10D880000051897EA22902F003879DF8081001EB60
:10D89000011202EB012100EBC100FEF776B819E09E
:10D8A0009DF80810A12201EB011303EB012100EB0D
:10D8B000C1039DF8101001EB011103EBC10101F54B
:10D8C00000514A779DF8081001EB011202EB01218B
:10D8D00000EBC10000F50050C67486E69DF8081004
:10D8E000A12201EB011303EB012100EBC1039DF821
:10D8F000101001EB011103EBC10101F500514A7752
:10D900009DF8081001EB011303EB012100EBC103AB
:10D910009DF8101001EB011103EBC10101F500515D
:10D920008A76B2E79DF8081001EB011202EB0121A3
:10D9300000EBC10101F50051CF749DF80810A7223A
:10D9400001EB011303EB012100EBC1039DF8101063
:10D9500001EB011103EBC10101F500514A779DF87C
:10D960000810CC4601EB4102C2EBC11109EBC10129
:10D97000497930299DF8081001EB41024FD0C2EBE4
:10D98000C1110CEBC101497931299DF808107CD0F7
:10D9900001EB4102C2EBC1110CEBC1014979332902
:10D9A0009DF8081001EB410270D0C2EBC1110CEBE5
:10D9B000C101497934299DF8081001EB410267D073
:10D9C000C2EBC1110CEBC101497935297DD09DF81D
:10D9D000081001EB410202EB01119DF8102000EB51
:10D9E000011101EB021129440A7822F001020A70A8
:10D9F0009DF8081001EB410202EB011100EB01124E
:10DA00009DF8101002EB01114A19117821F0020360
:10DA100013700021CDE900118DF82870CFE102EBE1
:10DA200001119DF8102000EB011101EB02112944B6
:10DA30000A7822F001020A709DF8081001EB4102F9
:10DA400002EB01119DF8102000EB011101EB021116
:10DA500029440A7822F002030B709DF8081001EBAC
:10DA6000011202EB012100EBC1039DF8101001EB44
:10DA7000011103EBC10101F50051C97E3129C8D163
:10DA80009DF8081001EB410203E00FE022E19FE363
:10DA900040E102EB011100EB01129DF8101002EBC6
:10DAA00001114A19117821F02003B1E701EB0112AD
:10DAB00002EB012100EBC1029DF8101001EB0111F6
:10DAC00002EBC10101F5005100E043E191F856106D
:10DAD00000299DF8081001EB011202EB012100EB77
:10DAE000C1029DF8101001EB011102EBC10101F51B
:10DAF00000517ED081F855709DF8081001EB41026D
:10DB000002EB011100EB01129DF8101002EB011164
:10DB10004A19117821F0010313709DF8081001EBE8
:10DB2000410202EB01119DF8102000EB011101EB05
:10DB3000021129440A7822F002020A7094F862174E
:10DB400000299CD1017D012999D1416DC28A914260
:10DB5000BFF45FAF9DF8081001EB011202EB012149
:10DB600000EBC1029DF8101001EB011102EBC101A5
:10DB700001F5005191F855100129E2D19DF80810E6
:10DB800001EB011202EB012100EBC1029DF8101024
:10DB900001EB011102EBC10101F5005191F88F1069
:10DBA0000029CED19DF808104FF0104201EB01136F
:10DBB00003EB012100EBC1039DF8101001EB0111F3
:10DBC00003EBC10101F500510A629DF8081001EB59
:10DBD000410202EB011100EB01129DF8101002EB63
:10DBE000011101F5805191F8802B9DF8081001E09A
:10DBF00068E15CE001EB011303EB012100EBC101E3
:10DC000001F500514A749DF8081001EB011202EB76
:10DC1000012100EBC1029DF8101001EB011102EB94
:10DC2000C10101F500510A7E9DF8081001EB0113B6
:10DC300003EB012100EBC10101F50051097D8A428E
:10DC40009BD19DF8081001EB011202EB012100EBC2
:10DC5000C1029DF8101001EB011102EBC10101F5A9
:10DC600000518F779DF80810A42201EB011303EBFC
:10DC7000012100EBC1039DF8101001EB011103EB32
:10DC8000C10101F500518A769DF80810A32201EB2D
:10DC9000011303EB012100EBC1039DF8101001EB10
:10DCA000011103EBC10101F500514A77B1E681F89A
:10DCB00055609DF8081001EB410202EB011100EBE9
:10DCC00001129DF8101002EB01114A19117841F070
:10DCD000010321E702EB01119DF8102000EB011177
:10DCE00001EB021129440A7842F001020A709DF802
:10DCF000081001EB410202EB011100EB01129DF84B
:10DD0000101002EB01114A19117841F0020313704F
:10DD1000A22220E002EB01119DF8102000EB01117E
:10DD200001EB021129440A7822F020020A709DF8C2
:10DD3000081001EB410202EB011100EB01129DF80A
:10DD4000101002EB01114A19117821F0020313702F
:10DD5000A92200E0A1229DF8081001EB011303EBBA
:10DD6000012100EBC1039DF8101001EB011103EB41
:10DD7000C10101F500518A764BE6DDE9001212017E
:10DD800042EA11720901CDE900129DF8081001EB79
:10DD90004102C2EBC1119DF828200CEBC1011144D6
:10DDA0008979DDE900383039CA17194342EA080297
:10DDB000CDE900129DF82810491C8DF828109DF817
:10DDC00028100829D9D39DF80810009A01EB0113F7
:10DDD00003EB012100EBC1039DF8101001EB0111D1
:10DDE00003EBC10101F50051C1F831200022CDE95A
:10DDF00000228DF8287021E0DDE90012120142EACC
:10DE000011720901CDE900129DF8081001EB4102E1
:10DE1000C2EBC1119DF828200CEBC1011144C97B54
:10DE2000DDE900383039CA17194342EA0802CDE962
:10DE300000129DF82810491C8DF828109DF8281014
:10DE40000629D9D39DF80810009A01EB011303EBC2
:10DE5000012100EBC1039DF8101001EB011103EB50
:10DE6000C10101F50051CA640022CDE900228DF8FC
:10DE7000287021E0DDE90012120142EA1172090165
:10DE8000CDE900129DF8081001EB4102C2EBC1116F
:10DE90009DF828200CEBC1011144497DDDE90038D3
:10DEA0003039CA17194342EA0802CDE900129DF839
:10DEB0002810491C8DF828109DF828100829D9D35E
:10DEC000FFF721B89DF80810804601EB011202EB24
:10DED000012200EBC20000F50050C7749DF8080055
:10DEE00000EB001202EB002008EBC0019DF81000CF
:10DEF00000EB001001EBC00000F50050007E03288D
:10DF000073D09DF8080000EB001101EB002008EB36
:10DF1000C0029DF81000414600EB001002EBC0006B
:10DF200000F50050027E9DF8080000EB001303EBA3
:10DF3000002008EBC00000F50050007D824213D1A4
:10DF400094F86207F0B39DF808009DF8101000EBFC
:10DF5000400202EB001008EB001000EB0110284417
:10DF6000017841F0080101709DF8080000EB0011F4
:10DF700001EB002008EBC0019DF8100000EB001041
:10DF800001EBC00000F5005080F856709DF80800C5
:10DF9000A72100EB001202EB002008EBC0029DF865
:10DFA000100000EB001002EBC00000F500504177BC
:10DFB0009DF80800A22100EB001202EB002008EB04
:10DFC000C00200E024E09DF8100000EB001002EB1E
:10DFD000C00000F5005081760021CDE900110A460D
:10DFE0008DF828704946A2E0FFE79DF8080004215B
:10DFF00000EB001202EB00229DF8100008EBC202B9
:10E0000000EB001002EBC00000F500500176ABE71A
:10E01000C1F835709DF8080000EB001101EB0021FC
:10E020009DF8100008EBC10100EB001001EBC000EF
:10E0300042F23901014410220C98FAF706F99DF8D2
:10E04000080000EB001101EB00219DF8100008EB27
:10E05000C10100EB001001EBC000313000F50050B1
:10E060004146026841F8192F406848609DF8080051
:10E0700000EB400101EB001108EB01109DF81010BE
:10E0800000EB011000F5805090F8801B88F8181004
:10E090009DF8080000EB001101EB00219DF8100035
:10E0A00008EBC10100EB001001EBC00000F50050CF
:10E0B000C16CC8F821100B9940468A6A40F8392F84
:10E0C000898D8180D8F8540081B20220FAF780FF50
:10E0D00000210620FBF786FDD8F85400401CC8F844
:10E0E000540000210520FBF77DFD3DE7009812015B
:10E0F00042EA10720001CDE900029DF8080000EB31
:10E100004002C2EBC0109DF8282001EBC000104473
:10E11000C07ADDE9003C3038C217184342EA0C02ED
:10E12000CDE900029DF82800401C8DF828009DF8DC
:10E1300028000C28DAD3DDE900239DF8080000EB65
:10E14000001C0CEB002008EBC00C9DF8100000EB4D
:10E1500000100CEBC00000F5005CCCF839206046E4
:10E16000C0F83D300022CDE900228DF8287021E072
:10E17000DDE90002120142EA10720001CDE900025D
:10E180009DF8080000EB4002C2EBC0109DF828206B
:10E1900001EBC0001044C07DDDE9003C3038C217FF
:10E1A000184342EA0C02CDE900029DF82800401C09
:10E1B0008DF828009DF828000C28D9D3DDE900123D
:10E1C0009DF8080000EB001303EB002008EBC003F0
:10E1D0009DF8100000EB001003EBC00000F50053A9
:10E1E000C3F841101846C0F8452002F051BAFE4B62
:10E1F0009DF808009DF8101003EB0010084400F58E
:10E20000805080F8107B9DF80800DFF8E08300EB79
:10E210004001C1EBC01008EBC000407870280AD163
:10E220009DF8080000EB4001C1EBC01008EBC000F6
:10E230008078FA2833D09DF8080000EB4001C1EB4C
:10E24000C01008EBC00040789DF8080000EB4001CA
:10E25000C1EBC01018F830009DF8080000EB001169
:10E2600001EB002003EBC00000F50050817C8DF82D
:10E2700010109DF8080003EB00119DF810000844F1
:10E2800000F5805080F8107BBDF8180001284CD0B4
:10E2900065287CD0B128A8D0B628A6D103E0B1204B
:10E2A000ADF81800D8E79DF8080000EB001101EB6D
:10E2B000002003EBC0019DF8100000EB001001EB03
:10E2C000C00000F50050007E01288ED19DF80800A6
:10E2D00000EB001101EB002003EBC00000F5005043
:10E2E000C7749DF8080000EB001101EB002003EB60
:10E2F000C0019DF8100000EB001001EBC00000F51C
:10E30000005006769DF80800B12100EB001202EBE8
:10E31000002003EBC0029DF8100000EB001002EBA0
:10E32000C00000F5005041775FE79DF8080000EB62
:10E330004001C1EBC01008EBC00000790128F3D008
:10E340000228F1D00328EFD00528EDD19DF8080070
:10E3500000EB001101EB002003EBC0019DF8100061
:10E3600000EB001001EBC00000F50050007E00281B
:10E37000DAD19DF8080000EB001101EB002003EB5F
:10E38000C00000F50050C7749DF8080000E033E0BD
:10E3900000EB001101EB002003EBC0019DF8100021
:10E3A00000EB001001EBC00000F5005006769DF870
:10E3B0000800B62100EB001202EB002003EBC002C4
:10E3C0009DF8100000EB001002EBC00000F50050BB
:10E3D00041779DF80800B22100EB001202EB00200B
:10E3E00003EBC0029DF8100000EB001002EBC00030
:10E3F00000F500508176F8E69DF8080000EB40013A
:10E40000C1EBC01008EBC0000079B922ADF81820AC
:10E410009DF8080000EB4001C1EBC01008EBC00004
:10E42000007900F00F018DF814108DF828701FE0AE
:10E430009DF8080000EB400101EB001003EB001118
:10E440009DF8280001EB001000F5805090F8811B2A
:10E450009DF8080000EB400CCCEBC01018F8300021
:10E460005038814214D09DF82800401C8DF82800B7
:10E470009DF8080000EB400101EB001003EB0010D9
:10E4800000F5805090F8570B9DF828108842CFD89F
:10E490009DF828009DF8141008448DF810009DF890
:10E4A000080000EB001101EB002003EBC00C9DF80D
:10E4B000100000EB00100CEBC00000F50050007ED7
:10E4C000012812D09DF8080000EB001101EB00209C
:10E4D00003EBC0019DF8100000EB001001EBC00041
:10E4E00000F50050007E012885D19DF8080000EB62
:10E4F000001101EB002003EBC00000F50050C774D1
:10E500009DF80800022100EB001C0CEB002003EB3F
:10E51000C00C9DF8100000EB00100CEBC00000F5E3
:10E52000005001769DF8080000EB001101EB00207F
:10E5300003EBC001F8E39DF8080000EB400101EB9C
:10E540000011294800EB011000F5805090F85C0B99
:10E5500020B101286FD00228C6D19BE2DFF8889055
:10E560009DF8081009EB410000F58040B0F830023A
:10E57000801F81B29DF80800DFF8708000EB400238
:10E58000C2EBC01208EBC200401CFBF7ABF8CDE9B0
:10E5900012079DF8081009EB410000F58040B0F823
:10E5A00030129DF80800414400EB4002C2EBC0105D
:10E5B0006FF0040202EBC0000844042108F0F0F8F8
:10E5C000DDE91223C117CDE900015040594008434D
:10E5D0008AD19DF8080009EB001000F5805080F802
:10E5E000107B9DF8080003E0D4120020AC620020EC
:10E5F00000EB4002C2EBC012404600EBC2000079C3
:10E60000ADF81800BDF818003128A5D19DF8081004
:10E6100009EB410000F58040B0F830024121183884
:10E6200090FBF1F0C217CDE9000284F844058DF8A3
:10E630002870B846CCE0D5E09DF8080000EB40011A
:10E64000C1EBC011FE4800EBC1019DF8280000EBB2
:10E6500080100844017D9DF8282009EB020000F598
:10E66000805080F845159DF8080000EB4001C1EB93
:10E67000C011F34800EBC1019DF8280000EB8010A9
:10E68000084408211A3008F057F88DED070A10EEFB
:10E69000100A9DF8282009EB021101F58051C1F8FC
:10E6A00055059DF8080000EB4001C1EBC011E4489E
:10E6B00000EBC1019DF8280000EB80100844082100
:10E6C000323008F039F88DED070A10EE100A9DF887
:10E6D000282009EB021101F58051C1F851059DF880
:10E6E000080000EB4001C1EBC011D54800EBC101AF
:10E6F0009DF8280000EB8010084408213A3008F00B
:10E700001BF88DED070A10EE100A9DF8282009EB82
:10E71000021101F58051C1F859059DF8080000EB80
:10E720004001C1EBC011C64800EBC1019DF82800B3
:10E7300000EB801008440821423007F0FDFF8DED0A
:10E74000070A10EE100A9DF8282009EB021101F5C6
:10E750008051C1F85D059DF8080000EB400101EB18
:10E76000001109EB01109DF8281000EB011028445E
:10E77000017841F0800101709DF8081009EB41001B
:10E7800000F58040B0F83012AD4801449DF8080013
:10E7900000EB4002C2EBC0124FF0FF3000EBC200B2
:10E7A000095C9DF8080000EB001202EB00229DF8C6
:10E7B000100009EBC20300EB001003EBC00000F5F2
:10E7C000005080F854109DF82800401C8DF8280057
:10E7D0009DF82800DDE90012401A78EB0200FFF6F0
:10E7E0002BAF02E59DF80800DFF8548200EB4001F2
:10E7F000C1EBC01008EBC000437D9DF8080000EBA2
:10E800004002C2EBC01008EBC000807D43EA00204C
:10E81000C317CDE900039DF80800152100EB400265
:10E82000C2EBC01008EBC000FAF746FFCDE91207B3
:10E83000DDE90010129B784059400143D1D19DF889
:10E84000080000EB4001C1EBC011404618F8311040
:10E85000491E8DF81010DFF8EC919DF808104A461B
:10E860009DF8103009EB0111194401F5805181F830
:10E87000107B9DF81010494401F5805181F84575D1
:10E880009DF8101009EB011101F58051C1F8557583
:10E890009DF8081001EB4103C3EBC11100EBC1016E
:10E8A00091F806C09DF8081001EB4103C3EBC111BC
:10E8B00000EBC10149794CEA012100EE101AF8EE93
:10E8C000400A9FED610A9DF8081080EE801A01EB66
:10E8D0004103C3EBC11100EBC10191F804C09DF8E5
:10E8E000081001EB4103C3EBC11100EBC101C97872
:10E8F0004CEA012100EE901A9DF81010F8EE600A23
:10E9000071EE200A10EE90CA02EB011101F5805160
:10E91000C1F851C59DF8081001EB4103C3EBC111CB
:10E9200000EBC10191F80AC09DF8081001EB41030A
:10E93000C3EBC11100EBC101497A4CEA012100EEA1
:10E94000901A9DF80810B8EE601AC1EE000A01EBAB
:10E950004103C3EBC11100EBC10191F808C09DF860
:10E96000081001EB4103C3EBC11100EBC101C979F0
:10E970009DF810304CEA012100EE101AB8EE400A62
:10E9800030EE800A10EE101A02EB031202F58052EC
:10E99000C2F859159DF8081001EB4102C2EBC111F4
:10E9A00000EBC100C07A00069DF8080000EB4001B2
:10E9B000C1EBC01008EBC000027B9DF8080000EB23
:10E9C0004003C3EBC01008EBC000C07A42EA00204D
:10E9D0000AD400EE100ADFED1D0AB8EE400A20EE60
:10E9E000200A10EE100A0BE0404280B2F9F7E9FD70
:10E9F0009FED171B53EC112BF9F702FDF9F746FEBB
:10EA00009DF8102009EB021101F58051C1F85D0558
:10EA10009DF808009DF8102000EB400101EB00106C
:10EA200009EB001000EB02102844027842F080024B
:10EA300002709DF8080000EB4002C2EBC0120BE030
:10EA4000AC620020D412002000FF7F470000803D10
:10EA5000000000000000B0BF08EBC200C27D9DF8BE
:10EA6000080000EB001303EB002009EBC0039DF846
:10EA7000100000EB001003EBC00000F5005080F820
:10EA800054209DF8080000EB400202EB001009EB57
:10EA90000010D0E09DF80800DFF8989400EB4001EA
:10EAA000C1EBC01009EBC000C3799DF8080000EB72
:10EAB0004002C2EBC01009EBC000007A43EA00201C
:10EAC000C317CDE900039DF80800072100EB4002C1
:10EAD000C2EBC01009EBC000FAF7EEFDCDE912075A
:10EAE000DDE90010129B7840594001437ED19DF82A
:10EAF000080000EB4001C1EBC01119F83100401EC5
:10EB00008DF81000DFF830849DF8081008EB011034
:10EB100000F5805080F8107B9DF8101008EB010084
:10EB200000F5805080F845759DF8080000EB400125
:10EB3000C1EBC01109EBC1008079F9F742FD41EC4E
:10EB4000110B9FEDFE0B0AF037F99DF80800B0EEAF
:10EB5000408AF0EE608A00EB4001C1EBC01109EB86
:10EB6000C10002799DF8080000EB4001C1EBC01123
:10EB700009EBC100C07842EA0020F9F722FD53EC0E
:10EB8000182BF9F7AFFCF9F781FD9DF8101008EB91
:10EB9000011101F58051C1F855059DF8101008EBE1
:10EBA000011000F58050C0F851759DF8101008EB69
:10EBB000011000F58050C0F859759DF8101008EB51
:10EBC000011000F58050C0F85D759DF8080000EB5D
:10EBD000400101EB001108EB01109DF8101000EB53
:10EBE00001102844017841F0800200E08EE20270BA
:10EBF0009DF8080000EB4001C1EBC01109EBC1001A
:10EC0000427A9DF8080000EB001101EB00219DF80D
:10EC1000100008EBC10300EB001003EBC00000F58F
:10EC2000005080F854209DF8080000EB400101EBF3
:10EC3000001108EB011000F5805090F8570B84F894
:10EC40004405CEE59DF80800DFF8E88200EB4001BE
:10EC5000C1EBC01008EBC0004146C3789DF8080026
:10EC600000EB4002C2EBC01008EBC000807843EA22
:10EC700000208DF80C009DF8080000EB4002C2EB6C
:10EC8000C0109DF80C2008EBC000104443789DF89C
:10EC9000080000EB4002C2EBC0109DF80C2001EB15
:10ECA000C000805C43EA0020C317CDE900039DF853
:10ECB00008009DF80C1000EB4002C2EBC01008EBFE
:10ECC000C000FAF7F9FCCDE91207DDE90001129B5B
:10ECD000794058400843B4D19DF8080000EB40014A
:10ECE000C1EBC01008EBC00040788DF810008DF823
:10ECF000287091491CE09DF8080000EB400202EBEF
:10ED000000109DF8282001EB001000EB021000F528
:10ED1000805090F8810B9DF8102090429DF82800BB
:10ED200003D18DF8100013E0FDE3401C8DF828009E
:10ED30009DF8080000EB400202EB001001EB001010
:10ED400000F5805090F8570B9DF828209042D2D8BB
:10ED50009DF8080000EB400202EB001001EB0012EE
:10ED60009DF8100002EB00102844027842F0800267
:10ED700002709DF8080000EB4002C2EBC01008EBE7
:10ED8000C0000079ADF818009DF808009DF810202B
:10ED900001EB0010104400F5805080F8107BBDF8A6
:10EDA0001800F32806D006DC05287CD0F12807D00F
:10EDB000F22890D14CE2F42876D0F6288BD149E2A3
:10EDC0009DF8080000EB001202EB002001EBC002EE
:10EDD0009DF8100000EB001002EBC00000F50050A1
:10EDE000007E00289DF8080025D000EB400202EBD1
:10EDF00000109DF8102001EB001000EB021000F550
:10EE0000805090F8890BC00714D09DF808008C46FC
:10EE100000EB001202EB002001EBC0029DF8100095
:10EE200000EB001002EBC00000F5005090F89E00CF
:10EE3000C00722D0BEE000EB001202EB002001EB85
:10EE4000C0029DF8100000EB001002EBC00000F5BE
:10EE5000005006769DF80800F42200EB001303EB47
:10EE6000002001EBC0039DF8100000EB001003EB45
:10EE7000C00000F5005042779CE09DF8080000EBD0
:10EE8000001202EB00200CEBC0029DF8100000EB1A
:10EE9000001002EBC00000F5005090F89000B8B3ED
:10EEA0008DF828702CE04DE2E7E19DF8080000EBBA
:10EEB000001202EB00209DF810200CEBC00002EBCA
:10EEC000021200EBC2009DF82820104400F500500B
:10EED00090F891209DF8080000EB400303EB001030
:10EEE0009DF828300CEB0010184400F5805090F885
:10EEF0005E0B824208D19DF82800401C8DF8280046
:10EF00009DF828000428D0D39DF82800042832D08A
:10EF100050E09DF8080000EB001202EB00200CEB23
:10EF2000C0029DF8100000EB001002EBC0009DF83D
:10EF3000282007E0AC620020D4120020000000006E
:10EF400000002440104400F5005090F891009DF816
:10EF5000082002EB420303EB02129DF828300CEB71
:10EF600002121A4402F5805292F85E2B904208D1A8
:10EF70009DF82800401C8DF828009DF828000A28DC
:10EF8000C7D39DF828000A2814D09DF8080000EB8C
:10EF9000001202EB002001EBC0029DF8100000EB14
:10EFA000001002EBC00042F29E021044027842F0D0
:10EFB000010202709DF80C00112844D09DF80C004D
:10EFC00014289DF8080000EB400202EB001001EB52
:10EFD00000129DF8100002EB001076D02844027851
:10EFE00022F0040202709DF8080000EB001202EB10
:10EFF000002001EBC0029DF8100000EB001002EBB6
:10F00000C00000F5005090F89E00C0077ED09DF82B
:10F01000080000EB001202EB002001EBC0029DF89B
:10F02000100000EB001002EBC00000F50050A0F84B
:10F030009C7005229DF8080000EB001303EB0020F4
:10F0400001EBC0016FE29DF8080000EB400202EB0B
:10F05000001001EB00129DF8100002EB00104219A5
:10F06000107840F0040313708DF82870424625E0B4
:10F070009DF8080000EB4003C3EBC01002EBC00397
:10F080009DF82800184443799DF8080000EB001C07
:10F090000CEB002001EBC00C9DF8100000EB001001
:10F0A0000CEBC00C9DF82800604400F5005080F87F
:10F0B00057309DF828305B1C8DF828309DF82800CB
:10F0C0000A28D5D38DF8287028E02CE09DF8080098
:10F0D00000EB4003C3EBC0109DF8283002EBC000EA
:10F0E0001844C37B9DF8080000EB001C0CEB0020CB
:10F0F00001EBC00C9DF8100000EB00100CEBC00001
:10F100009DF828C0604400F5005000E088E280F8D7
:10F1100070309DF82800401C8DF828009DF82800CC
:10F120000228D3D38DE54219107840F00403137000
:10F130008DF82870424625E09DF8080000EB40035A
:10F14000C3EBC01002EBC0039DF8280018444379BC
:10F150009DF8080000EB001C0CEB002001EBC00C3C
:10F160009DF8100000EB00100CEBC00C9DF828007F
:10F17000604400F5005080F857309DF828305B1C43
:10F180008DF828309DF828000A28D5D38DF82870EE
:10F190001FE09DF8283002EBC0001844C37B9DF8A7
:10F1A000080000EB001C0CEB002001EBC00C9DF8EC
:10F1B000100000EB00100CEBC0009DF828C060446C
:10F1C00000F5005080F870309DF82800401C8DF844
:10F1D00028009DF8280002289DF8080000EB400355
:10F1E000C3EBC010D5D302EBC0039DF82800184430
:10F1F000407C03049DF8080000EB400CCCEBC010F1
:10F2000002EBC00C9DF828006044807C43EA002398
:10F210009DF8080000EB400CCCEBC01008EBC002DE
:10F220009DF828001044C07C03439DF8080000EBC3
:10F23000001202EB002001EBC0019DF8100000EB72
:10F24000001001EBC00000F50050C0F88430E7E189
:10F25000F122EFE69DF80800032200EB001303EB18
:10F26000002001EBC0039DF8100000EB001003EB41
:10F27000C00000F500500276EAE79DF8080002227F
:10F2800000EB001303EB002001EBC0039DF810001E
:10F2900000EB001003EBC00000F5005002769DF873
:10F2A0000800F62200EB001303EB002001EBC00383
:10F2B0009DF8100000EB001003EBC00000F50050BB
:10F2C00042779DF8080000EB001202EB002001EBF2
:10F2D000C0029DF8100000EB001002EBC00000F52A
:10F2E000005080F890608DF82870424625E09DF827
:10F2F000080000EB4003C3EBC0109DF8283002EB80
:10F30000C000184443799DF8080000EB001C0CEB8A
:10F31000002001EBC00C9DF8100000EB00100CEB7E
:10F32000C0009DF828C0604400F5005080F891307E
:10F330009DF82800401C8DF828009DF828000A2818
:10F34000D5D36DE19DF8080000EB4002C2EBC01080
:10F3500008EBC00083799DF8080000EB400CCCEB73
:10F36000C01008EBC000407943EA00229DF8080075
:10F3700000EB001303EB002001EBC0039DF810002D
:10F3800000EB001003EBC00000F50050A0F89C203B
:10F390009DF8080000EB001202EB002001EBC00218
:10F3A0009DF8100000EB001002EBC00000F50050CB
:10F3B000B0F89C209DF8080000EB400303EB001020
:10F3C00001EB001000F58050B0F86A0B8242B8D310
:10F3D0009DF80800F12200EB001303EB002001EB85
:10F3E000C00C9DF8100000EB00100CEBC00000F505
:10F3F000005042779DF8080000EB001202EB00205D
:10F4000001EBC0019DF8100000EB001001EBC00003
:10F4100042F29E010844017821F00101FDF7E4B9B0
:10F420009DF8080000EB4001C1EBC010FE4A02EB62
:10F43000C00000798DF810008DF82070DFF8EC83A3
:10F440001BE09DF808009DF8201000EB400303EB43
:10F45000001008EB001000EB011000F5805090F850
:10F46000810B9DF8101088429DF8200002D18DF884
:10F47000100012E0401C8DF820009DF8080000EB01
:10F48000400101EB001008EB001000F5805090F8EF
:10F49000570B9DF820309842D3D89DF8080000EB18
:10F4A0004001C1EBC01002EBC000C078ADF81800FD
:10F4B000BDF81800182812D2DFE800F0110C0E1168
:10F4C00085857D857F111111818585858583111144
:10F4D000851185851A2000E00D208DF80C009DF81F
:10F4E0000C00001FC1B29DF80800914600EB4003DC
:10F4F000C3EBC01302EBC300C01CF9F70BFF8DF880
:10F5000000009DF8080000EB4001C1EBC01109EBC1
:10F51000C1009DF80C10084410F8010C9DF8001073
:10F5200088427DD100E0FCE39DF808004A4600EBEC
:10F530004001C1EBC01009EBC000407800286FD03B
:10F540009DF8080000EB4001C1EBC0109DF80C10C5
:10F5500002EBC0000844C3789DF8080000EB0011DE
:10F5600001EB002108EBC10C9DF81010404601EBA7
:10F5700001110CEBC10101F5005181F854309DF8E7
:10F58000081008EB01139DF81010194401F5805183
:10F5900081F8107BBDF81810CE291CD01CDCB929CD
:10F5A0007DD012DC5A29CAD0B22979D0B529F7D03A
:10F5B000B629B6D1FDE307208FE708208DE70C20A0
:10F5C0008BE70A2089E7062087E7C32969D0C52988
:10F5D00068D0CA29A5D1EDE3E129FCD006DCD52904
:10F5E00009D0D729ABD0D9299BD1C6E2E5297DD056
:10F5F000E72996D1FEE39DF8081001EB4103C3EB28
:10F60000C11109EBC101C97884F8A2119DF8081055
:10F6100001EB410202EB0112014600EB021000E097
:10F620003CE39DF8102000EB021094F8A22128443E
:10F63000A6EBD213027863F3000202709DF8080073
:10F6400000EB400202EB00109DF8102001EB0010CF
:10F6500000EB021094F8A22128445309027863F3C6
:10F66000410202709DF8080000EB400202EB00101E
:10F6700001EB00129DF8100002EB001000F5805025
:10F6800090F8820BC0F340029DF8080000EB0013D5
:10F6900003EB002008EBC0019DF8100003E0F1E34C
:10F6A000F1E3F1E3F1E300EB001001EBC00000F542
:10F6B000005090F83000C0F34000824251D09DF8D5
:10F6C0000800424600EB001101EB002008EBC001EE
:10F6D0009DF8100000EB001001EBC00042F2300179
:10F6E00001449DF8080000EB400300E0FEE303EB5B
:10F6F00000109DF8103008EB001000EB031000F52F
:10F70000805090F8820B4308087863F3410008703A
:10F710009DF8080000EB400101EB00109DF810106F
:10F7200002EB001000EB011000F5805090F8820B06
:10F73000800717D59DF80800D92100EB001303EBD3
:10F74000002008EBC0029DF8100000EB001002EB57
:10F75000C00000F5005041779DF808100220FAF72C
:10F7600041FA46E09DF8080000EB001101EB002093
:10F7700002EBC0019DF8100000EB001001EBC0008F
:10F7800000F5005080F825609DF80800D92100EBB5
:10F79000001303EB002002EBC0039DF8100000EB08
:10F7A000001003EBC00000F5005041779DF8080001
:10F7B00000EB400101EB001002EB00119DF810007E
:10F7C00001EB00104119087820F020030B709DF820
:10F7D000080000EB001101EB002008EBC0019DF8D0
:10F7E000100000EB001001EBC00000F5005080F8A5
:10F7F00056609DF80800434600EB400101EB001005
:10F8000008EB00119DF8100001EB001000F580508E
:10F8100090F8820B00F001019DF8080000EB001247
:10F8200002EB002004E00000AC620020D4120020B3
:10F8300008EBC0029DF8100000EB001002EBC000C6
:10F8400000F5005090F8300000F00100814271D0C6
:10F850009DF808009DF8102000EB001101EB00203E
:10F86000194603EBC00002EB021200EBC20042F2A9
:10F87000300210449DF8082002EB420303EB021211
:10F880009DF8103001EB021202EB031202F58052D8
:10F8900092F8822B037862F3000303709DF808004E
:10F8A00000EB400202EB00109DF8102001EB00106D
:10F8B00000EB021000F5805090F8820BC0079DF815
:10F8C000080038D000EB001202EB002001EBC00270
:10F8D0009DF8100000EB001002EBC00000F5005096
:10F8E00090F8560000289DF8080000EB001202EB8B
:10F8F000002001EBC0029DF8100000EB001002EBAD
:10F90000C00000F5005038D080F855709DF8080010
:10F9100000EB400202EB001001EB00129DF810001A
:10F9200002EB00104219107820F00103137094F8D4
:10F93000620728B3D9E000EB400202EB00109DF80B
:10F94000102001EB001000EB02102844027822F096
:10F95000200202709DF8080000EB001202EB00206C
:10F9600001EBC0019DF8100000EB001001EBC0009E
:10F9700000F5005080F85570B7E080F85560D6E784
:10F98000087D012868D1486DCA8A904264D29DF8EA
:10F99000080000EB001202EB002001EBC0029DF812
:10F9A000100000EB001002EBC00000F5005090F8D2
:10F9B0005500012850D19DF8080000EB001202EB21
:10F9C000002001EBC0029DF8100000EB001002EBDC
:10F9D000C00000F5005090F88F00E8BB9DF80800CB
:10F9E00000EB400202EB001001EB00129DF810004A
:10F9F00002EB001000F5805090F8802B9DF8080075
:10FA000000EB001303EB002001EBC00000F50050F9
:10FA100042749DF80800C32200EB001303EB0020A2
:10FA200001EBC0039DF8100000EB001003EBC000D9
:10FA300000F5005042779DF8080000EB400202EB11
:10FA4000001008EB00119DF8100001EB001000F50C
:10FA50008050C0F8847B00E047E09DF80810022049
:10FA6000FAF7C0F88DF82870414619E09DF80800B3
:10FA700000EB001202EB002001EBC0029DF8100029
:10FA800000EB001002EBC0009DF82820104400F5A8
:10FA9000005080F857709DF82800401C8DF8280011
:10FAA0009DF828001428E1D38DF8287019E09DF8FE
:10FAB000080000EB001202EB002001EBC0029DF8F1
:10FAC000100000EB001002EBC0009DF8282010444D
:10FAD00000F5005080F873709DF82800401C8DF8E8
:10FAE00028009DF828000A28E1D39DF808009DF819
:10FAF000102000EB400101EB0010414608EB001024
:10FB000000EB021000F5805090F8820B80077BF527
:10FB1000DBAC9DF80800D92200EB001303EB0020BA
:10FB200001EBC0039DF8100000EB001003EBC000D8
:10FB300000F500504277FBF7C7BC9DF8080000EBCA
:10FB4000001202EB002001EBC00000F50050C7746A
:10FB50009DF80800022200EB001303EB002001EBEC
:10FB6000C0039DF8100000EB001003EBC00000F58F
:10FB700000500276B622FBF736BE9DF8081001EB66
:10FB8000410303EB011108EB011000F5805090F8E0
:10FB90005C0B00289DF80C0002D00A287ED197E06B
:10FBA0000828FBD18DF8287024E09DF8080000EBB0
:10FBB0004001C1EBC0109DF8281002EBC0000844C2
:10FBC000C07800F00F00092818D89DF8080000EB55
:10FBD0004001C1EBC0109DF8281002EBC0000844A2
:10FBE000C07800F0F000902808D89DF82800401C4C
:10FBF0008DF828009DF828000628D6D39DF8280007
:10FC000006284BD39DF8080000EB4001C1EBC01063
:10FC100002EBC000C07801049DF8080000EB40032F
:10FC2000C3EBC01002EBC000007941EA00239DF84D
:10FC3000080000EB4001C1EBC01002EBC0004079AE
:10FC400003439DF8080000EB001101EB002008EBD6
:10FC5000C00C9DF81000414600EB00100CEBC000FA
:10FC600000F50050C0F831309DF8080000EB40036B
:10FC7000C3EBC01002EBC000807903049DF80800BC
:10FC800000EB400CCCEBC01002EBC000C07943EAA3
:10FC900000239DF8080000EB400C00E0C8E0CCEB2E
:10FCA000C01002EBC000007A03439DF8080000EB8F
:10FCB000001202EB002001EBC0019DF8100000EBE8
:10FCC000001001EBC00000F50050C0F83530AEE088
:10FCD0008DF8287024E09DF8080000EB4001C1EB8E
:10FCE000C0109DF8281002EBC0000844C07800F056
:10FCF0000F0009281AD89DF8080000EB4001C1EB5D
:10FD0000C0109DF8281002EBC0000844C07800F035
:10FD1000F00090280AD89DF82800401C8DF8280093
:10FD200000E047E19DF828000828D4D39DF828007A
:10FD300008287DD39DF8080000EB4001C1EBC010FE
:10FD400002EBC00081799DF8080000EB4003C3EB93
:10FD5000C01002EBC000C07841EA00619DF80800C5
:10FD600000EB4003C3EBC01002EBC00000790304BA
:10FD70009DF8080000EB400CCCEBC01002EBC0007B
:10FD8000407943EA002001439DF8080000EB00138E
:10FD900003EB002008EBC0039DF8100000EB0010FF
:10FDA00003EBC00000F50050C0F831109DF80800CA
:10FDB00001E007E1E8E000EB4001C1EBC01002EB1D
:10FDC000C000817A9DF8080000EB4003C3EBC0102F
:10FDD00002EBC000C07941EA00619DF8080000EB29
:10FDE0004003C3EBC01002EBC000007A03049DF88F
:10FDF000080000E0F7E300EB400CCCEBC01002EB96
:10FE0000C000407A43EA002001439DF8080000EB5F
:10FE1000001202EB002008EBC0029DF8100000EB7E
:10FE2000001002EBC00000F50050C0F8351000E0F3
:10FE30002EE29DF8080000EB001101EB002008EB1A
:10FE4000C0029DF81000414600EB001002EBC0001C
:10FE500000F50050007E032818D09DF8080000EB44
:10FE6000400202EB00109DF8102001EB001000EBA7
:10FE7000021000F5805090F8820B80077BF5BDAC36
:10FE80005A4678E682E046E14FE072E19DF80800CC
:10FE900000EB001202EB002001EBC00000F5005067
:10FEA000C7749DF80800042200EB001303EB002048
:10FEB00001EBC0039DF8100000EB001003EBC00045
:10FEC00000F500500276C52255E69DF8080000EBCB
:10FED000001202EB002001EBC0029DF8100000EBC5
:10FEE000001002EBC00000F5005000E052E380F883
:10FEF00026709DF80800B62200EB001303EB0020EB
:10FF000001EBC0039DF8100000EB001003EBC000F4
:10FF100000F5005042779DF8080000EB001202EB5C
:10FF2000002008EBC000FBF730BD9DF8081001EB86
:10FF3000011303EB012100EBC1039DF8101001EB4D
:10FF4000011103EBC10101F5005181F81DB09DF8CD
:10FF5000081001EB011202EB012100EBC10101F5D8
:10FF60000051CE749DF8081001EB410202EB011123
:10FF700008EB01109DF8101000EB011028440178E7
:10FF800041F02002027083E35A460BE09DF808100E
:10FF900001EB011202EB012100EBC10101F500515F
:10FFA000CF74C3229DF8081001EB011303EB01216C
:10FFB00008EBC1019DF8100000EB001001EBC00040
:10FFC000FCF722B89DF8081001EB410303EB011187
:10FFD00000EB011101F5805191F85C1B00299DF89F
:10FFE000081001EB4103C3EBC11102EBC10155D075
:10FFF000C9780B049DF8081001EB410CCCEBC11142
:020000040801F1
:1000000002EBC101097943EA01239DF8081001EBD5
:10001000410CCCEBC11109EBC10149790B439DF8AF
:10002000081001EB011202EB012100EBC1029DF867
:10003000101001EB011102EBC10101F50051CB647D
:100040009DF8081001EB011202EB012100EBC10247
:100050009DF8101001EB011102EBC10101F50051F7
:10006000097E022938D09DF80810C52201EB011342
:1000700003EB012100EBC1039DF8101001EB01110E
:1000800003EBC10101F500514A779DF8081001EB1F
:10009000011202EB012108EBC10044E70B799DF846
:1000A000081001EB410CCCEBC11109EBC101C9787F
:1000B00043EA01229DF8081001EB011303EB012133
:1000C00000EBC1039DF8101001EB011103EBC1011E
:1000D00001F50051CA64B3E79DF8081001EB011265
:1000E00002EB012100EBC10101F50051CF749DF835
:1000F0000810032201EB011303EB012100EBC10304
:100100009DF8101001EB011103EBC10101F5005145
:100110000A76D9227FE29DF8081001EB011202EB6A
:10012000012100EBC10101F50051CE749DF80810CA
:1001300001EB011303EB012100EBC1039DF810104B
:1001400001EB011103EBC10101F5005181F81DB074
:100150009DF8081001EB410202EB011108EB0110C0
:100160009DF8101000EB01102844017841F00402C2
:1001700008E79DF80810C64601EB410303EB0111A7
:1001800008EB011000F5805090F85C0B00289DF8FA
:100190000C0002D00E287BD1A0E00C2878D18DF87D
:1001A000287024E09DF8081001EB4100C0EBC1105D
:1001B0009DF8281002EBC0000844C07800F00F0042
:1001C000092818D89DF8081001EB4100C0EBC110B8
:1001D0009DF8281002EBC0000844C07800F0F00041
:1001E000902808D89DF82810491C8DF828109DF8F3
:1001F00028000A28D6D39DF828000A2848D30020D2
:10020000CDE90000034638468DF828701EE00099BD
:100210001B0243EA11630902CDE900139DF808109F
:1002200001EB4103C3EBC1119DF8283002EBC10182
:100230001944C978DDE9003C194340EA0C03CDE9D3
:1002400000139DF82810491C8DF828109DF82810DF
:100250000529DCD3DDE9003C9DF8081001EB01180D
:1002600008EB01210EEBC1099DF81010F04601EBDF
:10027000011109EBC10101F50059C9F839304946AE
:10028000C1F83DC00023CDE900338DF8280020E0FF
:10029000D2E0DDE900131B0243EA11630902CDE954
:1002A00000139DF8081001EB4103C3EBC1119DF849
:1002B000283002EBC1011944097ADDE9003C1943F9
:1002C00040EA0C03CDE900139DF82810491C8DF875
:1002D00028109DF828100529DBD39CE08DF82870A4
:1002E00024E09DF8081001EB4100C0EBC1109DF81F
:1002F000281002EBC0000844C07800F00F00092865
:1003000018D89DF8081001EB4100C0EBC1109DF812
:10031000281002EBC0000844C07800F0F0009028DC
:1003200008D89DF82800401C8DF828009DF828006A
:100330000C28D6D39DF828000C287DD30020CDE9C9
:10034000000038468DF828701FE0DDE900131B021D
:1003500043EA11630902CDE900139DF8081001EB8F
:100360004103C3EBC1119DF8283002EBC1011944D0
:10037000C978DDE9003C194340EA0C03CDE90013DC
:100380009DF82810491C8DF828109DF82810062982
:10039000DBD3DDE9003C9DF8081001EB011808EB08
:1003A00001210EEBC1099DF81010F04601EB01117F
:1003B00009EBC10101F50059C9F839304946C1F8C6
:1003C0003DC00023CDE900338DF828001FE0DDE9B2
:1003D00000131B0243EA11630902CDE900139DF8E3
:1003E000081001EB4103C3EBC1119DF8283002EB6B
:1003F000C1011944497ADDE9003C194340EA0C0384
:10040000CDE900139DF82810491C8DF828109DF89F
:1004100028100629DBD3DDE900129DF8080000EB67
:10042000001303EB002008EBC0039DF8100000EB65
:10043000001003EBC00000E02AE100F50053C3F810
:1004400041101846C0F845209DF80800F04600EB22
:10045000001101EB00200EEBC0029DF8100000EB34
:10046000001002EBC00000F50050027E9DF808006D
:1004700000EB001303EB00200EEBC00000F5005072
:10048000007D824274D194F8620700287BF4F1ACBD
:10049000C8F835709DF8080000EB001101EB002151
:1004A0009DF8100008EBC10100EB001001EBC0004B
:1004B00042F23901014410220C98F7F7C6FE9DF86C
:1004C000080000EB001101EB00219DF8100008EB83
:1004D000C10100EB001001EBC000313000F500500D
:1004E0004146026841F8192F406848609DF80800AD
:1004F00000EB400101EB001108EB01109DF810101A
:1005000000EB011000F5805090F8801B88F818105F
:100510009DF8080000EB001101EB00219DF8100090
:1005200008EBC10100EB001001EBC00000F500502A
:10053000C16CC8F821100B9940468A6A40F8392FDF
:10054000898D8180D8F8540081B20220F8F740FDEF
:1005500000210620F9F746FBD8F85400401CC8F8E3
:10056000540000210520F9F73DFBFBF798BCFFE79D
:100570009DF8080000EB400101EB001108EB0110B1
:100580009DF8101000EB01102844017841F004019F
:100590000170EAE784F8A0669DF8081001EB0112EB
:1005A00002EB012100EBC1029DF8101001EB0111DB
:1005B00002EBC10101F50051097E00299DF80810E8
:1005C00001EB011202EB01210ED000EBC1029DF8FC
:1005D000101001EB011102EBC10101F50051897E00
:1005E000B22927D054E071E000EBC10101F50051C0
:1005F000CF749DF8081001EB011202EB012100EB12
:10060000C1029DF8101001EB011102EBC10101F5CF
:1006100000510E765A469DF8081001EB011303EBCA
:10062000012108EBC1039DF8100000EB001003EB63
:10063000C000C5E49DF8081001EB011202EB012196
:1006400000EBC10101F50051CF749DF80810B222F2
:1006500001EB011303EB012100EBC1039DF8101026
:1006600001EB011103EBC10101F500514A779DF83F
:10067000081001EB011202EB012108EBC1029DF809
:10068000100000EB001002EBC00000F50050877670
:1006900094F8A703B0B120489DF8081000EB410082
:1006A00000F58040B0F830129DF80800012300EBFF
:1006B0004002C2EBC012194800EBC2009DF80820AE
:1006C000FAF772F98DF82870144912E084F8A076D0
:1006D0005AE49DF8080000EB4002C2EBC0109DF800
:1006E000282001EBC00087549DF82800401C8DF89D
:1006F00028009DF828001428EBD309480178427897
:10070000114482781144C278D1427AF40FAB21B0FF
:10071000BDEC028BBDE8F08FD4120020AC6200204B
:10072000100800202DE9F74F90B00020ADF8000030
:10073000ADF80400ADF80400ADF804008DF8100029
:100740008DF814008DF81800CDE90800CDE90800F7
:10075000ADF83C00FEA2D2E90032CDE90232FEA2A1
:10076000D2E90032CDE90A32FD4A1071109800EB4F
:10077000400202EB0010FB4A02EB001E0EF5805017
:10078000834690F8560B8DF81000109802EB00107D
:100790000790084400F58050824690F8102B10987E
:1007A000042A00EB001303EB0020EE4B03EBC00028
:1007B00001EB011300EBC3070D900EEB011007F5E1
:1007C000005500F580591DD105208AF8100B002036
:1007D000287699F8820B20F0800289F8822B9BF80A
:1007E000562BA120072A0DD2DFE802F00C040B0BD8
:1007F00006080A00E52004E0B12002E0312000E014
:10080000F12068779DF810801098DDF848C000EB63
:10081000001404EB0020D34C022304EBC00000F5CD
:100820000050019010984122CF4EC0EB001000EB19
:100830008004ACF1A10CB8F1070F7AD2DFE818F010
:10084000790007008E02D00356052306970699F813
:10085000810B4FF00008414601F056FD8DF8140061
:10086000297E0198007D814202D101980121C17445
:100870009AF8100B401C8AF8100B129BA221A6209C
:10088000CE2B7DD012DC4FF0A502B92B79D006DC3F
:10089000B22B77D0B52B35D0B62B4AD10BE1C32B79
:1008A00071D0C52B70D0CA2BF7D1F9E0E12B6CD0F9
:1008B00006DCD52B09D0D72B68D0D92BEDD10FE092
:1008C000E52B6ED0E72BE8D132E2F52006F83400B4
:1008D0009DF8140006EBC4056870A970D52009E0E6
:1008E000F52006F834009DF8140006EBC405687086
:1008F000A970D920E8702846032101F036FC287140
:10090000052009E2F52106F834109DF8141006EBD5
:10091000C40779709BF85C1B4FF0B50951B1296A87
:10092000B1F1104F37D34FF010410022CDE908123A
:1009300034E08AE2286AB0F5100F05D34FF41000B6
:100940000021CDE9080102E0286ACDE90808BA7063
:1009500040460FE0BDF80000C0F10200C200DDE932
:100960000801F7F760FCBDF800103944C870BDF805
:100970000000401CADF80000BDF80000032806E0B0
:1009800030E126E0A2E080E021E1F8E0DBE1E1D324
:1009900087F80690ECE0296ACDE90818B87040465F
:1009A00010E0BAE1BDF80000C0F10300C200DDE9CB
:1009B0000801F7F738FCBDF800103944C870BDF8DD
:1009C0000000401CADF80000BDF800000428E9D389
:1009D00059E0F52106F834109DF8141006EBC40711
:1009E00079709BF85C1B4FF0B90949B1296AB1F1E4
:1009F000104F2CD02A6ACDE90828B87040463CE058
:100A0000286AB0F5100F05D0296ACDE90818BA7028
:100A1000404615E04FF410000021CDE90801F6E74B
:100A2000BDF80000C0F10200C200DDE90801F7F7DF
:100A3000FAFBBDF800103944C870BDF80000401C36
:100A4000ADF80000BDF800000328E9D3A0E74FF09F
:100A500010410022CDE90812CFE7BDF80000C0F137
:100A60000300C200DDE90801F7F7DDFBBDF8001067
:100A70003944C870BDF80000401CADF80000BDF856
:100A800000000428E9D3484699E0F52006F8340030
:100A90009DF8140006EBC4056870A970C32029E70F
:100AA000F52006F834009DF8140006EBC4056870C4
:100AB000A970CA201EE7F52006F834009DF814003E
:100AC00006EBC4056870A970B62013E7F52006F898
:100AD00034009DF8140006EBC40778709BF85C0B9B
:100AE000B22110B1BA7040462CE0A420B870404644
:100AF0000DE0E86CBDF80020C2F10102D200D04048
:100B0000BDF800203A44D070BDF80000401CADF89C
:100B10000000BDF800000228EBD3797138460521AA
:100B200001F023FBB87173E1E86CBDF80020C2F15D
:100B30000202D200D040BDF800203A44D070BDF887
:100B40000000401CADF80000BDF8000003280DE0D7
:100B500001693230313030000169323045303000C7
:100B600010080020D41200204C590020DCD3B971A9
:100B70003846062101F0F9FAF8710820CCE0F52199
:100B800006F834109DF8141006EBC4077970B8709D
:100B900040460DE0286DBDF80010C1F10301C90009
:100BA000C840BDF800103944C870BDF80000401CB2
:100BB000ADF80000BDF800000428EBD3E120F87187
:100BC0003846072101F0D1FA38720920A4E0F52057
:100BD00006F834009DF8140006EBC4056870A9708F
:100BE000C52087E6F52006F834009DF8140006EBD2
:100BF000C40568709BF85C0B4FF0CE0918B1AE20AD
:100C0000A87040465CE0AC20A870404615E007F5AF
:100C10000050D0F8390007F50051D1F83D10BDF86B
:100C20000020C2F10402D200F7F7FDFABDF800106F
:100C30002944C870BDF80000401CADF80000BDF8A4
:100C400000000528E3D3404615E007F50050D0F832
:100C5000410007F50051D1F84510BDF80020C2F160
:100C60000402D200F7F7DFFABDF800102944087239
:100C7000BDF80000401CADF80000BDF800000528DC
:100C8000E3D385F80D9028460D2101F06EFAA87384
:100C90000F2041E007F50050D0F8390007F500516A
:100CA000D1F83D10BDF80020C2F10502D200F7F7DF
:100CB000BAFABDF800102944C870BDF80000401C05
:100CC000ADF80000BDF800000628E3D3404615E06B
:100CD00007F50050D0F8410007F50051D1F8451054
:100CE000BDF80020C2F10502D200F7F79CFABDF86A
:100CF000001029444872BDF80000401CADF8000007
:100D0000BDF800000628E3D385F80F9028460F2190
:100D100001F02BFA2874112096E2F52006F8340031
:100D20009DF8140006EBC4056870A970E520E1E5A4
:100D3000F52006F834009DF8140006EBC405687031
:100D4000A970E720D6E5F52006F834009DF81400D8
:100D500006EBC4056870A970D720CBE599F8810B24
:100D60008DF81400297E0198007D814202D10198FE
:100D70000121C1749AF8101B491C8AF8101B9DF8B8
:100D8000140020B19DF81400401E8DF81400BCF131
:100D90000A0F5AD2DFE80CF0FDFC4678D4FBFA05C6
:100DA000F95A06F834309DF8140006EBC4074030B9
:100DB0007870BA703020F8703871287F0009787127
:100DC00078790A28787901D2303000E037307871AC
:100DD000287F00F00F00B871B8790A28B87901D2DD
:100DE000303000E03730B8710320F871781C0721EB
:100DF000F8F790FA38720920ADF83C00287E0428F4
:100E000001D10520287601990020C87406201BE036
:100E1000072019E2287103206871681C0521F8F782
:100E200079FAFDE3042306F834309DF8141006EB3C
:100E3000C4004031417082700521C170ADF83C3072
:100E4000287E022801D103202876F3E306F8343007
:100E50009DF8140006EBC40540306870AA7031207C
:100E6000E8703220287103206871681C0521F8F7AA
:100E700051FAA8710720ADF83C0099F8820B20F0D8
:100E8000200189F8821BD5E306F834309DF8140060
:100E900006EBC40740307870BA703120F87030210A
:100EA00039712A6AB2F5100F00D232217971A97F07
:100EB000012902D0A87F28B100E0B8710021ADF867
:100EC000001014E03220F8E7286ABDF80020C2F1D3
:100ED00005029200D040BDF8002000F00F003A4417
:100EE0003030D071BDF80000401CADF80000BDF8F6
:100EF00000000628E8D332207873ADF8001012E025
:100F0000E86CBDF80010C1F103018900C840BDF8CC
:100F1000001000F00F00394430308873BDF8000035
:100F2000401CADF80000BDF800000428E8D3032001
:100F3000B874781C1221F8F7EDF9F874142077E3EF
:100F400006F834309DF8140006EBC4074030787082
:100F5000BA703220F870312139717871B87100217E
:100F6000ADF8001018E0E86CBDF80020C2F10302F3
:100F70009200D040BDF8002000F00F003A4430301D
:100F8000D071BDF80000401C04E069E041E141E19E
:100F900059E048E0ADF80000BDF800000428E2D3B5
:100FA000ADF80010302108E0BDF800003844C172EF
:100FB000BDF80000401CADF80000BDF80000192885
:100FC000F2D3032087F82400781C2421F8F7A2F933
:100FD00087F8250026202BE306EBC401487058E073
:100FE00099F8810B8DF81400297E0198007D8142CB
:100FF00002D101980121C1749AF8100B401C8AF8A3
:10100000100B9DF8140020B19DF81400401E8DF8BF
:101010001400BCF10A0F15D2DFE80CF005152F59AA
:10102000FDFCFB14223E042206F834209DF8141027
:1010300006EBC40040314170512181700521C1701F
:10104000ADF83C20F6E206F834309DF8140006EBCB
:10105000C40540306870AA703120E8703520D9E6A8
:1010600006F834309DF8140006EBC4054030687073
:10107000AA703220E8703020CCE6042306F8343021
:101080009DF8141006EBC4004031417082700521B8
:10109000C170ADF83C30CDE206F834309DF8140054
:1010A00006EBC40540306870AA703120E870322029
:1010B000287103206871681C0521F8F72BF9A871C5
:1010C00099F8820B20F0200189F8821BA0E606F82F
:1010D00034309DF8140006EBC40740307870BA70C5
:1010E0003120F8703A71296AB1F1104F07D03221DE
:1010F0007971A97F012904D0A87F38B102E030219D
:10110000F6E7B8710022ADF8002014E03220F8E7CD
:10111000286ABDF80010C1F107018900C840BDF878
:10112000001000F00F0039443030C871BDF80000E5
:10113000401CADF80000BDF800000828E8D33220BC
:10114000F873ADF8002012E0E86CBDF80010C1F1B2
:1011500005018900C840BDF8001000F00F003944B7
:1011600030300874BDF80000401CADF80000BDF838
:1011700000000628E8D33021B975ADF8002008E05A
:10118000BDF800003844C175BDF80000401CADF842
:101190000000BDF800000628F2D37977ADF80020F2
:1011A00008E0BDF8000038448177BDF80000401C1D
:1011B000ADF80000BDF800000628F2D387F824102F
:1011C000ADF8002009E0BDF80000384480F8251093
:1011D000BDF80000401CADF80000BDF80000062876
:1011E000F1D387F82B10ADF8002009E0BDF800001E
:1011F000384480F82C10BDF80000401CADF8000009
:10120000BDF800000628F1D387F83210ADF80020B1
:101210000CE066E060E018E0BDF80000384480F8BB
:101220003310BDF80000401CADF80000BDF8000010
:101230000628F1D3032087F83900781C3921F8F704
:1012400069F887F83A003B20F2E106F834309DF85F
:10125000140006EBC40740307870BA703220F87082
:101260003121397133217971B8710021ADF8001045
:1012700012E0E86CBDF80020C2F105029200D040F7
:10128000BDF8002000F00F003A443030D071BDF8B6
:101290000000401CADF80000BDF800000628E8D3AF
:1012A000ADF80010302008E0BDF800103944487354
:1012B000BDF80010491CADF80010BDF80010192948
:1012C000F2D3032087F82600781C2621F8F722F8AD
:1012D00087F827002820ABE1102006F834003020E2
:1012E0007AE6102006F83400312075E699F8810B73
:1012F0008DF81400BDF800000D9A00EB001002EB11
:10130000C00000F50050027E0198007D824202D1AB
:1013100001980122C2749AF8100B401C8AF8100B35
:101320000027ADF8007010E0BDF800200EEB0210B1
:1013300000F5805090F8810B9DF8142090420AD05F
:10134000BDF80000401CADF800009BF8570BBDF83D
:1013500000209042E8D8BDF800200EEB021000F506
:10136000805090F8800B081A401C8DF818009DF8EA
:10137000140020B19DF81400401E8DF81400687E02
:101380000F2803D2687E401C687600E06F761298C2
:101390006521B1384FF0FA08092873D2DFE800F070
:1013A000050C40727260721C2D009DF814005030C4
:1013B00006F8340020215EE09DF81400503006F855
:1013C0003400687E06EBC40540F0300068700120F0
:1013D000A870E8702F7133E09DF81400503006F8C3
:1013E0003400687E06EBC40540F030006870A970D8
:1013F0000120E8709DF8180021E09DF8140050309D
:1014000006F83400687E06EBC40540F030006870D2
:10141000A9700120E8709DF8180040F010000EE05F
:101420009DF81400503006F83400687E06EBC405C1
:1014300040F0300068700120A870E8700520287125
:1014400028460521F8F724FBCDE9080768710898BC
:10145000000AA8710320E87185F80880FFF7B5BB82
:10146000A87E6877AF769DF81400503006F83400F7
:10147000687E40F0C00106EBC400417080F8028035
:101480000320D5E088E0BDF800200798104441F61D
:10149000103210440278521C02709BF85C0B30B181
:1014A000491CC9B2012836D0022875D144E01298EF
:1014B000312802D045286FD116E00020ADF8000099
:1014C00002A90CE0BDF80000BDF8003006EBC40234
:1014D000085CD054BDF80000401CADF80000BDF819
:1014E00000000728EED393E40020ADF800000AA91D
:1014F0000CE0BDF80000BDF8003006EBC402085C4B
:10150000D054BDF80000401CADF80000BDF800004C
:101510000728EED37CE48DF814109DF8140006F82B
:10152000340006EBC405032068700027AF70EB7031
:101530002F71092068710EE08DF814109DF81400C9
:1015400006F8340006EBC405032068700027AF706E
:10155000EF702F716B7128460621F8F7ADF8CDE9D1
:101560000807000AE8710898A871FFF706BBF74959
:101570009AF8100B401C8AF8100B99F8810B8DF823
:1015800014001298F3287DD007DC05287BD0F128C1
:1015900008D0F2284ED113E04CE0F42874D0F6289D
:1015A00048D1FAE0F52006F834009DF8140006EB67
:1015B000C40568700027AF700520E870F1201EE1B7
:1015C000F52006F834009DF8141006EBC4008046A0
:1015D00041704FF0000980F80290F221017195F8F6
:1015E0008E10417195F88E0001282ED095F88E004E
:1015F00020287DD00620ADF83C00BDF83C0088F8DE
:1016000003004046BDF83C10F8F756F8CDE908094C
:10161000BDF83C20000A08F80200BDF83C2000E0BC
:10162000F7E0089808EB02014870BDF83C00801C08
:10163000ADF83C00C648C74D109931B3012978D0A8
:10164000022977D0032976D188E12520ADF83C0026
:101650004946ADF8009010E0BDF80000384400F5B0
:10166000005090F86120BDF8003008EB0300827153
:10167000BDF80000401CADF80000BDF800000F28C8
:10168000EAD303E058E0C6E0ACE033E1ADF8001087
:1016900010E0BDF80000384400F5005090F87320C9
:1016A000BDF8003008EB03004275BDF80000401C97
:1016B000ADF80000BDF800000A28EAD395F88820AC
:1016C00088F81F20ADF8001011E0BDF80000384484
:1016D00000F5005090F88910BDF8002008EB0200DA
:1016E00080F82010BDF80000401CADF8000000E0BC
:1016F00004E0BDF800000528E7D37EE70A20ADF836
:101700003C0048460EE0BDF80000384400F50050AB
:1017100090F88910BDF8002008EB02008171BDF837
:101720000000401CADF80000BDF800000428EAD31A
:1017300063E7EDE0F9E008E1F52006F834009DF8F4
:10174000141006EBC400804641704FF0000980F889
:101750000290F322027195F88E2042710C22ADF8AE
:101760003C2095F888208271ADF8009010E0BDF81B
:101770000000384400F5005090F88910BDF80020B2
:1017800008EB0200C171BDF80000401CADF800007C
:10179000BDF800000528EAD32FE70620ADF83C008D
:1017A000F52006F834009DF8140006EBC4056870B7
:1017B0000027AF70BDF83C00E870F620287199F85A
:1017C000880B68712846BDF83C10F7F775FFCDE926
:1017D0000807BDF83C10000A6854BDF83C10089892
:1017E000294421E7F52006F834009DF8140006EBA3
:1017F000C40568700027AF700520E870F4202871D8
:1018000028460521F7F758FFCDE90807000A687157
:101810000898A8715AE440F21320ADF83C00F52076
:1018200006F834009DF8140006EBC4077870BDF884
:101830003C00000AB870BDF83C00F8700520387113
:101840004FF0000840460EE0BDF800200EEB02000D
:1018500000F5805090F85E0BBDF800203A445071BE
:10186000BDF80000401CADF80000BDF800000A28DB
:10187000EAD3BBF86A0B8946000AF873BBF86A0B17
:10188000387435F89C0F000A78742888B874298851
:10189000109801EB802081B20320F7F72DFB45461D
:1018A000ADF8008049464FF400720FE0BDF800002B
:1018B000084400F5805090F8A601BDF800303B4484
:1018C000D874BDF80000401CADF80000BDF8000061
:1018D0009042EBD33846BDF83C10F7F7EDFECDE96A
:1018E0000805BDF83C10000A7854BDF83C10089873
:1018F000394499E6BDF83C1039B38021F8F78FFDE3
:10190000BDF83C00C5F8A40012480121A03031E028
:10191000BDF83C10C9B10821F8F781FDBDF83C00C5
:1019200068670C480121703024E0BDF83C0060B1CC
:101930004FF480710848F8F772FDBDF83C00C5F817
:10194000BC0004480121B83014E015E0D412002096
:10195000000C02400060024000000240BDF83C1054
:1019600051B14FF48061F8F75AFDBDF83C00E865CD
:1019700001210948F7F7F6FE084890F8A703002868
:1019800007D006EBC4000023BDF83C10109AF9F70D
:101990000BF813B0BDE8F08F58600240D42200204D
:1019A0002DE9F04700242DED048B804689469FEDFC
:1019B0001E9B25462646E20040464946F6F733FC84
:1019C000C7B22046F6F7FDFD41EC110BB0EE490A17
:1019D000F0EE690A07F0F0F9380907F00F0100EBA3
:1019E0008000B0EE408AF0EE608A01EB4000F6F72E
:1019F000E8FD53EC182BF6F703FD41EC180B2846D5
:101A00003146F6F7EBFD53EC182BF6F752FCF6F7E0
:101A100018FE641CE4B205460E46082CCBD3BDEC80
:101A2000048BBDE8F0870000000000000000594072
:101A300070B50E4D40F224442146284606F057FE6C
:101A4000012812D1298828462A1D1188214606F02E
:101A5000EBFD0748012180F8B11A0648D0F88C0048
:101A60000549C0F57A70A1F8380270BD0044004005
:101A7000D422002000600240D452002010B50B4C4C
:101A800040F22441204606F032FE01280DD1208884
:101A9000201D00880648012180F8BD1A0548406CC9
:101AA0000549C0F57A70A1F83A0210BD004C00401B
:101AB000D422002000600240D452002010B50B4C0C
:101AC00040F22441204606F012FE01280CD1208865
:101AD000A0880748012180F8C91A064840690649CC
:101AE000C0F57A70A1F83C0210BD00000050004023
:101AF000D422002000600240D452002010B50B4CCC
:101B000040F22441204606F0F2FD01280DD1208844
:101B1000201D00880648012180F8D51A0548C06AB2
:101B20000549C0F57A70A1F83E0210BD004800409A
:101B3000D422002000600240D452002010B5124C84
:101B400010492046F7F7F8FD00212046F7F70AFE76
:101B50000E4C4021204606F0C3FD0028F9D080211C
:101B60000B48F8F75EFC084C0A49183C2046F7F78A
:101B7000E3FD01212046F7F7F5FD07490120087133
:101B800010BD000000802020A06002400044004002
:101B9000000C0240008800201008002010B5124CF4
:101BA00010492046F7F7C8FD00212046F7F7DAFD77
:101BB0000E4C4021204606F093FD0028F9D0082164
:101BC0000B48F8F72EFC084C0A49303C2046F7F742
:101BD000B3FD01212046F7F7C5FD07490120087133
:101BE00010BD00002080002070600240004C0040CA
:101BF000000C0240008020101008002010B5124C8C
:101C000010492046F7F798FD00212046F7F7AAFD76
:101C10000E4C4021204606F063FD0028F9D04FF419
:101C200080710B48F8F7FDFB074C0A49A83C204699
:101C3000F7F782FD01212046F7F794FD06490120C0
:101C4000087110BD00800028B860024000500040BC
:101C500000000240208000101008002010B5124C37
:101C600010492046F7F768FD00212046F7F77AFD76
:101C70000E4C4021204606F033FD0028F9D04FF4E9
:101C800080610B48F8F7CDFB074C0A49303C2046F1
:101C9000F7F752FD01212046F7F764FD06490120C0
:101CA000087110BD008000185860024000480040D4
:101CB000000C024000880010100800202DE9F047B9
:101CC000012190B0480504F087FA8648F7F754FDE3
:101CD000402738010024CDE90540C5010794089448
:101CE000CDE9094546040C940D94DFF8FC917F483A
:101CF0000B94CDE90207CDE9006969460E94794855
:101D0000F7F7E2FD012210217648F7F7C7FDDFF86B
:101D1000D4A1AAF1180A5046F7F72EFD4FF47A78AD
:101D2000CDE90348E811CDE9054007940894CDE9D1
:101D300009456F480B940C940D9400960E94CDE9D0
:101D4000019069465046F7F7BFFD01215046F7F76D
:101D500009FDDFF890A1AAF1300A5046F7F70CFD13
:101D6000E811CDE9054007940894CDE909450C94A4
:101D70000D94DFF8809160480B94CDE90207CDE91E
:101D8000006969460E945046F7F79EFD0122102126
:101D90005046F7F783FDDFF84CA1AAF1600A5046E0
:101DA000F7F7EAFCCDE90348E811CDE905400794CF
:101DB0000894CDE9094551480B940C940D94009674
:101DC0000E94CDE9019069465046F7F77DFD01215B
:101DD0005046F7F7C7FCDFF80CA10AF1180A504685
:101DE000F7F7CAFCE811CDE9054007940894CDE95E
:101DF00009450C940D94DFF8089142480B94CDE905
:101E00000207CDE9006969460E945046F7F75CFD7C
:101E1000012210215046F7F741FDDFF8C8A0AAF1D2
:101E2000900A5046F7F7A8FCCDE90348E811CDE940
:101E3000054007940894CDE9094533480B940C9468
:101E40000D9400960E94CDE9019069465046F7F73F
:101E50003BFD01215046F7F785FCDFF88890A9F19A
:101E600048094846F7F788FC0397E811CDE9054093
:101E700007940894CDE9094525480B940C940D94DA
:101E8000224F00960E94CDE9017069464846F7F757
:101E90001BFD012210214846F7F700FDDFF84490B2
:101EA000A9F178094846F7F767FCCDE90348E8113E
:101EB000CDE9054007940894CDE9094515480B94F0
:101EC0000C940D9400960E94CDE901706946484635
:101ED000F7F7FAFC01214846F7F744FC10B0BDE8DB
:101EE000F0870000A0600240044400404C590020EC
:101EF000AC620020044C0040A45B002094660020EB
:101F000004500040FC5D00207C6A00200448004032
:101F100054600020646E00202DE9FC410121084638
:101F200004F05AF90121042004F056F90121082097
:101F300004F052F90121402004F04EF9DFF8FC8052
:101F4000072205214046F8F753FA072206214046AA
:101F5000F8F74EFA072208214046F8F749FA072217
:101F600009214046F8F744FA354F08220A2138463D
:101F7000F8F73EFA08220B213846F8F739FA08221A
:101F800002214046F8F734FA08220C213846F8F7C7
:101F90002FFA02268DF8056000244FF459708DF851
:101FA0000640012500908DF807508DF804606946C1
:101FB0004046F8F7E1F98DF805604FF4E0508DF8F0
:101FC000064000908DF807508DF804606946384649
:101FD000F8F7D2F94FF4916000908DF806408DF833
:101FE000045069464046F8F7C7F9280200908DF87A
:101FF00006408DF8045069461248F8F7BDF98DF88F
:1020000006404FF4F040104C00908DF804506946A3
:102010002046F8F7B1F9A9032046F8F700FA69035A
:102020002046F8F7FCF9A1142046F8F7F8F9E11476
:102030002046F8F7F4F9BDE8FC810000000C0240EE
:1020400000080240000002400018024070B5002461
:10205000FFF762FFFFF732FE00F022F80E4D00217D
:1020600085F8AC1A012285F8AC2A0C480170817001
:102070004170C2704FF47A718160042085F8AC0A17
:1020800004E0204600F062F9641CE4B295F8AC0A62
:10209000A042F6D870BD0000D42200205055002088
:1020A000F8B511208DF8000002258DF801500124AB
:1020B0008DF802408DF80340684600F01BFB262097
:1020C0008DF800008DF8014000268DF802608DF833
:1020D0000340684600F00EFB0E208DF800008DF8DE
:1020E00001508DF802408DF80340684600F002FB75
:1020F00027208DF800008DF801408DF802608DF8E2
:102100000340684600F0F6FA0F208DF800008DF8C5
:1021100001508DF802408DF80340684600F0EAFA5D
:1021200034208DF800008DF801408DF802608DF8A4
:102130000340684600F0DEFA2F208DF800008DF88D
:1021400001508DF802408DF80340684600F0D2FA45
:1021500035208DF800008DF801408DF802608DF873
:102160000340684600F0C6FAF8BD01B9102110F826
:10217000012B10F8013B491E5A400904090CF8D103
:1021800002F07F00704700002DE9FF5F14460F4604
:102190004FF480564FF480684FF4C0694FF00C0A3A
:1021A00040F2244B002580B1012830D0022851D0C4
:1021B000032871D10121880404F032F80097012C22
:1021C0006DD0022C70D094B377E00121480404F064
:1021D00027F80097012C03D0022C06D054B10DE053
:1021E000ADF80460ADF8088008E0ADF80460ADF823
:1021F000089003E0ADF80450ADF80850ADF8065073
:10220000ADF80C50ADF80AA069463B4C5DE00121E9
:10221000C80404F005F80097012C03D0022C07D065
:102220005CB10EE0ADF80460ADF8088009E040E074
:10223000ADF80460ADF8089003E0ADF80450ADF8D7
:102240000850ADF80650ADF80C50ADF80AA069463C
:102250002A4C3AE00121080503F0E2FF0097012C27
:1022600003D0022C06D054B10DE0ADF80460ADF8F7
:10227000088008E0ADF80460ADF8089003E0ADF820
:102280000450ADF80850ADF80650ADF80C50ADF85C
:102290000AA069461A4C18E02CE000E004E0ADF812
:1022A0000460ADF8088008E0ADF80460ADF808906F
:1022B00003E0ADF80450ADF80850124CADF80650EC
:1022C000ADF80C50ADF80AA06946204606F046FA73
:1022D0000121204606F0ABF901225946204606F0BE
:1022E00025FA1021204606F09FF90122C021204640
:1022F00006F0A7F9BDE8FF9F00440040004C0040F5
:1023000000500040004800402DE9FC410024CDE988
:1023100000446F4664220023F5F754FF0E4605463D
:10232000104619460A220023F5F74CFF010102F07E
:102330000F000818385504F10104E4B2284631466C
:10234000082CE7D3DDE90001BDE8FC812DE9F84F59
:10235000784E80460024042086F8AC0A08EB480139
:1023600001EB0810A6F5805707EB0015009505F561
:10237000805595F85D0B012803D10021404600F0FF
:10238000DDF808EB4802B94607EB8207A7F5AA6714
:1023900007F5005700203870B8707870F8704FF06B
:1023A000050AC7F808A087F8300087F83200012036
:1023B00087F8310087F83300D5F8580B00EB800020
:1023C0004000B86395F8552BD5F8501B4046A7F54B
:1023D0002B67FFF7D9FE95F8561B08EB081202EBA6
:1023E0000820554A072902EBC00B0BF5005014D208
:1023F000DFE801F0130406090B0D1700514600E059
:102400000F21017509E00721FBE70421F9E7D5F861
:10241000580B64214843C7F8E80A4FF0A10ECA469A
:1024200063E00321EDE704EB041300210BEBC30091
:10243000183000F500500173012383734173C17399
:102440004FF47A734361009B03EB041303F580534D
:1024500083F8821B00F8181995F8561B072942D2F9
:10246000DFE801F041040707090B0D00E521417782
:1024700039E07146FBE7B121F9E73121F7E7F121B6
:10248000417700212BE001EB011202EB01220AEB64
:10249000C20701EB410202EB01120AEB021200201B
:1024A00002F5805915E002EB001C0CF5805C9CF8ED
:1024B00080CB93F8888BC44509D193F880CB00EB8F
:1024C000001807EBC80808F5005888F88FC0401CB2
:1024D000C0B299F857CB8445E5D8491CC9B296F8E3
:1024E000AC0A8842CFD8641CE4B295F8570B524628
:1024F000A04298D8002086F8AD0A00EB400101EB1D
:10250000001102EB011101F5805191F8563B052BAA
:1025100009D291F8563B33B196F8AD3A91F8571B72
:10252000194486F8AD1A401CC0B20428E5D3BDE8B2
:10253000F88F0000D4220020D41200202DE9F041B1
:10254000054663484FF4804253100668614884147E
:10255000C71439B1C5B1012D18D0022D18D0032DE3
:102560001BD117E035B1012D06D0022D06D0032D69
:1025700013D105E0114604E0194602E0214600E0CF
:102580003946F7F74EFF08E0114604E0194602E02D
:10259000214600E03946F7F742FF642007F060FD6E
:1025A00000224FF416512846FFF7EEFD4A4905EB8D
:1025B000450001EB800000F58050002280F8E22AFF
:1025C000C0F8E42A05EB450000EB051001EB001014
:1025D00000F58050D0F8583B01F58041C1F88432B5
:1025E000012381F87D3290F8561B3C4C962305EB75
:1025F0008500204406290AD2DFE801F00903050519
:102600000733762102E0837001E06E218170C5EB13
:102610000511334B01EB8101C02403F8314003EB7A
:10262000C10462700821A170E27006F00F0105EB91
:10263000051211442171807860712020A071E17130
:10264000802020724C2060725420A0722548264FB2
:102650000B2645B1012D0FD0022D25D0032D14D10D
:102660002DE06621D2E78021F7F7D9FEC7F8A460F4
:102670001D480121A03006E00821F7F7D0FE7E6753
:10268000194801217030F7F76DF8184890F8A70342
:1026900028B1204600232A460B21F8F785F9BDE82A
:1026A000F041642007F0DCBC4FF480711048F7F76C
:1026B000B6FEC7F8BC600C480121B830E3E74FF420
:1026C0008061F7F7ACFEFE65074801215830DAE774
:1026D000187AFF1F00180240D41200204C7200200C
:1026E0004C590020000C024000600240D42200201F
:1026F0000000024030B50F23C27801780125FAB1FD
:10270000144A126801F1E02102F4E062C2F5E062CD
:10271000C2F30722C2F10404D3404278A240847875
:102720001C401443220181F80024007800F01F01AE
:102730008D404009800000F1E020C0F8005130BD1C
:1027400001F01F0085404809800000F1E020C0F83A
:10275000805130BD0CED00E0024A114001430248B7
:102760000160704780FFFF1F08ED00E0BFF34F8F4F
:1027700004480168044A01F4E06111430160BFF3B9
:102780004F8FFEE70CED00E00400FA05BFF34F8F1A
:1027900004480168044A01F4E06111430160BFF399
:1027A0004F8FFEE70CED00E00400FA0510B50021A4
:1027B000074B0A46002003EBC004401CC0B2625421
:1027C0008028F8D3491CC9B20829F3D310BD0000F2
:1027D0004F7C00202DE9FE4F0026171A8146701EFF
:1027E0003546A3EB010A8846002F02DD4FF00101B8
:1027F00002E003D14FF00001019102E0C7F10007B0
:102800000190BAF1000F02DD4FF0010002E003D1A8
:102810004FF00000009002E0C7F1000A009050461F
:10282000574501DD3C4600E00446601C4FF0000BBC
:10283000029016E008F0FF0109F0FF000C9A00F08A
:1028400015F83E445544A64202DD0199361B8944E1
:10285000A54202DD00992D1B88440BF101001FFAEF
:1028600080FB02998B45E5DBBDE8FE8F30B5CC08D7
:1028700001F0070301259D40EBB2064D05EBC005B5
:10288000C808285C0AB1184302E063EA0000C043AC
:10289000285530BD4F7C00202DE9FC4101210A2044
:1028A00003F09AFC01248DF8044000264FF4C05038
:1028B0008DF80660032700908DF805708DF80740AD
:1028C00069464648F7F758FD8DF804408DF80660D4
:1028D0008DF80570A5028DF80740414C00956946BA
:1028E0002046F7F749FDC82007F0BAFB29462046E5
:1028F000F7F795FDC82007F0B3FB29462046F7F708
:1029000090FDC82007F0ACFB0021FD2000F024FA68
:102910000021122000F020FA0021AE2000F01CFA65
:102920000021D52000F018FA0021A02000F014FAB0
:102930000021A82000F010FA00213F2000F00CFA3E
:102940000021D32000F008FA0021084600F004FA24
:102950000021402000F000FA0021A02000F0FCF946
:102960000021C02000F0F8F90021DA2000F0F4F98D
:102970000021122000F0F0F90021812000F0ECF994
:1029800000217F2000F0E8F90021D92000F0E4F9CF
:102990000021822000F0E0F90021DB2000F0DCF9CA
:1029A0000021342000F0D8F90021A42000F0D4F94F
:1029B0000021A62000F0D0F90021202000F0CCF961
:1029C0000021084600F0C8F9FFF7F0FE0021AF2013
:1029D00000F0C2F900F054F8BDE8FC81000C0240A0
:1029E000000402400346012000E05843491EC9B2DA
:1029F000FBD270472DE9F84F82460A980D465043A6
:102A00006421B0FBF1F0984600F0FF0B4FF0010994
:102A10000AEB02072B4600245046FAB21946CDF8BD
:102A20000090FFF7D7FE05EB0806F3B2FAB2F1B259
:102A30005046CDF80090FFF7CDFE5246F3B229463E
:102A40001046CDF80090FFF7C5FEF3B2FAB2F8B227
:102A50002946CDF80090FFF7BDFE4F460AEB0B0666
:102A600009E02819C3B2C1B2F2B250460097FFF78D
:102A7000B1FE641CE4B24445F3D3BDE8F88F000016
:102A800070B50025B020294600F066F900210846FF
:102A900000F062F90021102000F05EF9084E0024D9
:102AA00006EBC4000121405D00F056F9641CE4B25D
:102AB000802CF5D36D1CEDB2082DF0D370BD000055
:102AC0004F7C002070B50B4C05460221204603F0D8
:102AD0004DFD0028F9D02946204603F050FD012184
:102AE000204603F043FD0028F9D0204603F045FDC1
:102AF000C0B270BD003800402DE9FC4F1D4688462D
:102B000081468B460090082B0ED0680700D001202C
:102B100000EBD500690810FB01F0C0B2203A02F0CA
:102B2000FF0A0026019046E00620F7E7082D10D0A6
:102B30000C2D14D0102D16D0182D3FD121490AEBA1
:102B4000CA0001EB80000027845DE0070FD00B9ADC
:102B500010E01D490AEB4A0001EB4000F3E70AEBE5
:102B60004A001A49EDE71A4901EB0A10EBE70B9806
:102B700030B3002241464846FFF778FE7F1C6408C8
:102B800008F10100FFB200F0FF08082FDDD309F1C2
:102B9000010000F0FF09082D0AD00099A9EB0100FF
:102BA000B0EB550F04D10BF10800894600F0FF0B84
:102BB000761CD846F6B201988642B7D3BDE8FC8FA2
:102BC0000122D7E748BC0108BCAF0108E4B1010805
:102BD00058B601082DE9F84F1D00DDE90A79924643
:102BE0008B4680464FF0000611D11046F5F7E9FC00
:102BF00041EC100B06F048F89FED1C1B51EC100B3C
:102C000053EC112BF5F755FBF5F7FCFCC5B2082F7B
:102C100000D1022600241CE0281B401EC1B20A205D
:102C2000FFF7E0FEBAFBF0F00A21B0FBF1F201FB86
:102C30001200CDF8009088B13030C2B206EB5701D7
:102C400001FB0480C0B23B465946FFF755FF641CA8
:102C5000E4B2AC42E0D32846BDE8F88F06EB57015A
:102C600001FB0480C0B23B463022EDE700000000CB
:102C70000000F03F2DE9FF4F81B0064600900F465F
:102C80004FF0000A8946580700D0012000EBD3001E
:102C90000490002032E0002029E00E98002410F873
:102CA0000A500AF101001FFA80FAE80701D00F9AD2
:102CB00002E00F9848B3002239463046FFF7D6FDB0
:102CC0007F1C641C6D08E4B2FFB2082CEDD3761CA7
:102CD0000098F6B2311A0398814204D109F1080034
:102CE000009E00F0FF0908F101004F46C0B20399B1
:102CF00080468842D1D30BF10100C0B204998346CB
:102D00008842C8D305B0BDE8F08F0122D4E72DE991
:102D1000F8431D46DDE908781646894604460EE06C
:102D20003B4649462046CDF80080FFF7E5FE082FD8
:102D30000ED004EB5700C4B26D1EEDB2761C002D10
:102D400004D03278202A01D37E2AE9D9BDE8F8835D
:102D5000A41DE4B2F0E700002DE9F041114C064655
:102D60004FF4006500292946204602D0F7F759FBA9
:102D700001E0F7F754FB4FF4805739462046F7F748
:102D80004EFB39460848F7F74CFB3046FFF79AFEF2
:102D900039462046F7F745FB29462046BDE8F04175
:102DA000F7F73FBB000C0240000402402DE9F04F52
:102DB00087B04FF00008ADF80C80ADF80480ADF896
:102DC0000880ADF81480ADF81080ADF8008041F6B1
:102DD00082394FF0A30BFD4CFDE394F86407022801
:102DE00002D10720ADF80000F94FBDF800003844CB
:102DF0008079BDF800103944C97840EA0160BDF817
:102E0000001039440979BDF8002009043A44527988
:102E100041EA02210843EF494A68904276D048606F
:102E2000BDF8000038448078BDF800103944497876
:102E300040EA0126B4F82A16BDF800003044801C90
:102E4000814263D3B4F82A06BDF80010801B401AF3
:102E5000801EA4F82A06BDF8000031463844F6F773
:102E60002BFCBDF80010314439444978BDF80020EE
:102E70003244BA5C41EA0221814279D194F8A70335
:102E800040B1B01C81B2BDF80000012338440422D7
:102E9000F7F78AFDBDF800003844007900F0010022
:102EA0000490BDF80000384480790025C0F3420A40
:102EB000F31F0DE028443844C07952460499F6F7D0
:102EC000FDFDBDF8001029443944C8716D1CADB238
:102ED000BDF800009D42EDDB3844C079012184F843
:102EE00062174FF0000AC4F868A684F866A6BA4ACA
:102EF00082F872A2C2F874A2ADF814A011287DD095
:102F00000DDCA0F10B00062815D200E0FEE3DFE89F
:102F100010F0A00802093D093709590B1D00A2282D
:102F20006ED004DC12286CD0A12804D124E3A3289D
:102F300068D0A42867D000205146BDF80020024484
:102F4000B954401C80B20528F7D3FDE35046F0E1A8
:102F5000BDF80C00A14D00EB400101EB001005EBAA
:102F6000001000F5805090F8560B07287ED200E044
:102F7000EBE3DFE800F07B040404047BA30050468D
:102F800088E0BDF80000BDF8141008443844007A09
:102F9000A8B3012802D0022874D112E0BDF80C00B9
:102FA00000EB400101EB0010BDF8041005EB001030
:102FB00000EB011101EB0900017821F0040101701F
:102FC00060E0BDF80C0000EB400101EB0010BDF823
:102FD000041005EB001000EB011101EB0900017872
:102FE00021F008010170BDF80C0000EB400202EB7B
:102FF000001005EB0010BDF8042005E0F0E341E00F
:10300000EFE3EFE3EFE3EFE300EB021000F58050B6
:10301000C0F884ABBDF80C100220F6F7E3FD0020E9
:103020005246BDF80C1001EB011303EB012105EB37
:10303000C103BDF8041001EB011103EBC101014410
:1030400001F5005181F85720401C80B21428E8D3C4
:103050000020BDF80C1001EB011303EB012105EB7F
:10306000C103BDF8041001EB011100E05EE103EBC8
:10307000C101014401F5005181F87320401C80B268
:103080000A28E6D3BDF81400401CADF81400BDF8C2
:103090000400401CADF80400BDF80C0000EB40013A
:1030A00001EB001005EB001000F5805090F8570B75
:1030B000BDF8041088423FF664AF37E1D446ADF85E
:1030C00004A022E1BDF80000BDF814100844384403
:1030D000007A042805D005DC58B1012845D0022823
:1030E00073D130E108287BD010287AD020286CD109
:1030F000E1E1BDF80C0000EB001101EB002005EB55
:10310000C001BDF8040000EB001001EBC00000F5A9
:10311000005090F88E00102823D1BDF80C0000EB71
:10312000001101EB002005EBC001BDF8040000EB2D
:10313000001001EBC00000F5005080F88EC0BDF813
:103140000C00F32100EB001202EB002005EBC002A3
:10315000BDF8040000EB001002EBC00000F50050C9
:103160004177BDF81400401CC8E0BDF80C00F22106
:1031700000EB001202EB002005EBC002BDF80400DA
:1031800000EB001002EBC00000F500504177BDF8E5
:103190000C0000EB400101EB0010BDF8041005EB42
:1031A000001000EB011101EB0900017821F004018E
:1031B0000170BDF80000BDF8141008443844017ACD
:1031C000BDF80C0000EB00120CE099E0D4220020C6
:1031D00060720020180A0020D4520020D41200206F
:1031E000B1E0EEE002EB002005EBC002BDF8040008
:1031F00000EB001002EBC00000F5005080F88E10CC
:103200000020BDF80010BDF81420114401443944D9
:103210004A7ABDF80C1001EB011303EB012105EB19
:10322000C103BDF8041001EB011103EBC10101441E
:1032300001F5005181F86120401C80B20F28E0D3D5
:103240000020BDF80010BDF8142011440144394499
:103250000A7EBDF80C1001EB011303EB012105EB15
:10326000C103BDF8041001EB011103EBC1010144DE
:1032700001F5005181F87320401C80B20A28E0D388
:10328000BDF80000BDF814100844384490F822003E
:10329000BDF80C1001EB011202EB012105EBC1029C
:1032A000BDF8041001EB011102EBC10101F5005161
:1032B00081F888000020BDF80010BDF814201144EA
:1032C0000144394491F82320BDF80C1001EB01139F
:1032D00003EB012105EBC103BDF8041001EB011163
:1032E00003EBC101014401F5005181F88920401C24
:1032F00080B20528DFD3BDF814002030ADF81400EB
:10330000BDF80400401CADF80400BDF80C0000EB53
:10331000400101EB001005EB001000F5805090F823
:10332000570BBDF8041088423FF6CCAEBDF80C0038
:10333000401CADF80C0094F8AC0ABDF80C108842A3
:103340003FF606AE01E6BDF80C00F22100EB0012DC
:1033500002EB002005EBC002BDF8040000EB0010FA
:1033600002EBC00000F500504177BDF80C0000EB07
:10337000400101EB0010BDF8041005EB001000EB5C
:10338000011101EB0900017821F004010170BDF881
:103390000000BDF8141008443844017ABDF80C0050
:1033A00000EB001202EB002005EBC002BDF80400A8
:1033B00000EB001002EBC00000F5005080F88E100A
:1033C000CFE6BDF80C00F32100EB001202EB002069
:1033D00005EBC002BDF8040000EB001002EBC000DA
:1033E00000F500504177BDF80C0000EB400101EB07
:1033F0000010BDF8041005EB001000EB011101EB0B
:103400000900017821F004010170BDF80000BDF849
:10341000141008443844017ABDF80C0000EB001287
:1034200002EB002005EBC002BDF8040000EB001029
:1034300002EBC00000F5005080F88E10BDF80000CF
:10344000BDF8141008443844417ABDF80C0000EB74
:10345000001202EB002005EBC002BDF8040000EBF7
:10346000001002EBC00000F5005080F8881000202A
:10347000BDF80010BDF814201144014439448A7A83
:10348000BDF80C1001EB011303EB012105EBC103A7
:10349000BDF8041001EB011103EBC101014401F57A
:1034A000005181F88920401C80B20528E0D3BDF886
:1034B0001400C01D22E7BDF80C00F22100EB001241
:1034C00002EB002005EBC002BDF8040000EB001089
:1034D00002EBC00000F500504177BDF80C0000EB96
:1034E000400101EB0010BDF8041005EB001000EBEB
:1034F000011101EB0900017821F004010170BDF810
:103500000000BDF8141008443844017ABDF80C00DE
:1035100000EB001202EB002005EBC002BDF8040036
:1035200000EB001002EBC00000F5005080F88E1098
:103530000020BDF80010BDF81420114401443944A6
:103540004A7ABDF80C1001EB011303EB012105EBE6
:10355000C103BDF8041001EB011103EBC1010144EB
:1035600001F5005181F88920401C80B20428E0D385
:10357000BDF81400401DC1E6B01E0D2190FBF1F016
:10358000C0B204905046C8E1ADF804A0FE4DA0E1E1
:10359000BDF80C0000EB400101EB0010BDF8041079
:1035A00005EB001000EB011000F5805090F8820B45
:1035B00080077CD408EB880101EBC800BDF800103F
:1035C00008443844007A0021FEF7EAF9BDF80C20DF
:1035D00002EB420300E0FCE303EB0212BDF804300F
:1035E00005EB021202EB031202F5805292F8802BD7
:1035F0008AEA010342401A4359D1BDF80C0000EB9E
:10360000001101EB002005EBC001BDF8040000EB48
:10361000001001EBC00000F5005090F855000128A3
:1036200075D1BDF800003844407BBDF80010394426
:10363000897A40EA0161BDF800003844C07ABDF8DB
:10364000002000043A44127B40EA02200143BDF806
:103650000C0000EB001202EB002005EBC002BDF8ED
:10366000040000EB001002EBC00000F50050016206
:10367000BDF800003844007DBDF800103944497C95
:1036800040EA0160BDF800103944897CBDF8002093
:1036900009043A44D27C41EA02210843BDF80C10E7
:1036A00001EB410202EB011105EB011100E00BE11E
:1036B000BDF8042001EB021101F58051C1F8840B23
:1036C000BDF80C0000EB400101EB0010BDF8041048
:1036D00005EB001000EB011101EB0900017841F04E
:1036E00020010170BDF80C100220F6F77BFABDF83E
:1036F0000C0000EB400101EB0010BDF8041005EBDD
:10370000001000EB011000F5805001E0FDE364E0E3
:1037100090F8801BBDF80C0000EB001202EB0020BB
:1037200005EBC00000F500504174BDF80C0000EB43
:10373000400101EB001005EB001000F5805090F8FF
:10374000560B012807D001E0F0E0FCE302284CD042
:10375000032842D149E0BDF800003844407A10B156
:1037600001283AD13AE0BDF80C0000EB400101EB32
:10377000001005EB001000F5805090F85C0B00285D
:10378000BDF80C0000EB001101EB002005EBC001BF
:10379000BDF8040000EB001001EBC00000F5005084
:1037A000006A03D0B0F1104F03D104E0B0F5100F60
:1037B00001D0B52100E0C321BDF80C0000EB0012E0
:1037C00002EB002005EBC002BDF8040000EB001086
:1037D00002EBC00000F5005041776EE0B921EBE745
:1037E000FEE36DE1FDE3AAE2A1E0BDF80C0000EB11
:1037F000001101EB002005EBC001BDF8040000EB57
:10380000001001EBC00000F50050017EBDF80C0077
:1038100000EB001202EB002005EBC00000F50050A9
:10382000007D814249D1BDF800003844807BBDF85D
:10383000001000043944C97B40EA0121BDF80000B2
:103840003844007C0143BDF80C0000EB001202EB91
:10385000002005EBC002BDF8040000EB001002EBF5
:10386000C00000F50050C164BDF800003844417A42
:10387000BDF80C0000EB001202EB002005EBC002CB
:10388000BDF8040000EB001002EBC00000F5005092
:103890008177BDF80C00A42100EB001202EB0020A0
:1038A00005EBC002BDF8040000EB001002EBC00005
:1038B00000F50050817659467EE708F10100049931
:1038C00000F0FF08884515D2BDF80400401CADF893
:1038D0000400BDF80C0000EB400101EB001005EB0B
:1038E000001000F5805090F8570BBDF80410884286
:1038F0003FF64EAEBDF80C0000EB400101EB0010AE
:1039000005EB001000F5805090F8570BBDF804103F
:1039100088420BD8BDF80C00401CADF80C0094F8A0
:10392000AC0ABDF80C1088423FF62EAE1AE15046A4
:103930004BE0ADF804A0144D20E0BDF80000384481
:10394000007A0021FEF72CF8BDF80C2002EB4203B0
:1039500003EB0212BDF8043005EB021202EB031276
:1039600002F5805292F8802B8AEA010342401A4302
:1039700034D0BDF80400401CADF80400BDF80C00C4
:1039800000EB400102E00000D412002001EB001027
:1039900005EB001000F5805090F8570BBDF80410AF
:1039A0008842CAD8BDF80C0000EB400101EB0010C2
:1039B00005EB001000F5805090F8570BBDF804108F
:1039C0008842B3D8BDF80C00401CADF80C0094F848
:1039D000AC0ABDF80C108842ABD8C3E0BDF80C00AF
:1039E00000EB400101EB0010BDF8041005EB0010E6
:1039F00000EB011000F5805090F8801BBDF80C0022
:103A000000EB001202EB002005EBC00000F50050B7
:103A10004174BDF80C0000EB400101EB001005EB18
:103A2000001000F5805090F8560B012835D0022880
:103A300001D00328B6D1BDF80C0000EB001101EB5A
:103A4000002005EBC001BDF8040000EB001001EB05
:103A5000C00000F50050017EBDF80C0000EB001224
:103A600002EB002005EBC00000F50050007D814214
:103A700098D1BDF80C00AA2100EB001202EB002047
:103A800005EBC002BDF8040000EB001002EBC00023
:103A900000F500508176594600E0CA21BDF80C00BF
:103AA00000EB001202EB002005EBC002BDF80400A1
:103AB00000EB001002EBC00000F50050417771E709
:103AC000002047E00020ADF80400DFF8B0A61EE0BB
:103AD000BDF800003844007A0021FDF761FFBDF811
:103AE0000C2002EB420303EB02130AEB0312BDF8B6
:103AF000043002EB031202F5805292F8802B424010
:103B00000A4330D0BDF80400401CADF80400BDF8F5
:103B10000C0000EB400101EB00110AEB011000F575
:103B2000805090F8570BBDF804108842D0D8BDF8EB
:103B30000C0000EB400101EB00110AEB011000F555
:103B4000805090F8570BBDF8041088420AD8BDF891
:103B50000C00401CADF80C0094F8AC0ABDF80C1039
:103B60008842AFD870E1BDF80C00BDF8042000EB2E
:103B7000400101EB001051460AEB001000EB02106F
:103B800000F5805090F8802BBDF80C0000EB00137E
:103B900003EB00200AEBC00000F500504274BDF8B2
:103BA00000003844407ABDF8002000043A44927A7C
:103BB00040EA0222BDF800003844C07A0243BDF852
:103BC0000C0000EB001303EB002001EBC003BDF879
:103BD000040000EB001003EBC00000F50050C264CD
:103BE000BDF80C0000EB400202EB001001EB0010EE
:103BF00000F5805090F8560B012846D0022801D0DD
:103C0000032894D1BDF80C0000EB001202EB002059
:103C100001EBC002BDF8040000EB001002EBC00095
:103C200000F50050027EBDF80C0000EB001303EB22
:103C3000002001EBC00000F50050007D8242E0D181
:103C4000BDF80C00A52200EB001303EB002001EBF4
:103C5000C003BDF8040000EB001003EBC00000F54A
:103C600000508276BDF80C0000EB001303EB00203F
:103C70000AEBC001BDF8040000EB001001EBC0002E
:103C800000F5005080F81DB051E7BDF80C0000EBC6
:103C9000001202EB002001EBC002BDF8040000EBB3
:103CA000001002EBC00000F50050027EBDF80C00D1
:103CB00000EB001303EB002001EBC00000F5005007
:103CC000007D8242E0D1BDF80C00B22200EB00136F
:103CD00003EB002001EBC003BDF8040000EB001073
:103CE00003EBC00000F500508276BDF80C00E52221
:103CF00000EB001303EB002001EBC003BDF8040050
:103D000000EB001003EBC00000F500504277002DDF
:103D1000BAD1BDF804000128B6D1BDF80C0000EB03
:103D2000001202EB00200AEBC001BDF8040000EB1A
:103D3000001001EBC00000F50050C06CF7E6BDF8C4
:103D400000003844007A05287ED2BDF800003844CF
:103D5000007A401EADF80C00BDF800003844407AEF
:103D6000BDF8001000043944897A40EA0120BDF80A
:103D700000103944C97A0843C117FDF711FEBDF898
:103D80000C10FE4D01EB410202EB011205EB02119A
:103D900001F58051C1F8500BBDF800003844007B9C
:103DA0000021FDF7FDFDBDF80C1001EB410202EB17
:103DB000011205EB021101F5805181F8540BBDF899
:103DC00000003844407B0021FDF7EAFDBDF80C10EF
:103DD00000E0F6E301EB410202EB011205EB0211F8
:103DE00001F5805181F8550BBDF800003844807B07
:103DF0000021FDF7D5FDBDF80C1001EB410202EBEF
:103E0000011205EB021101F5805181F8560BBDF846
:103E100000003844C07B0021FDF7C2FDBDF80C1046
:103E200001EB410202EB011205EB021101F5805199
:103E300081F8570BBDF800003844007C0021FDF7E5
:103E4000AFFDBDF80C1000E065E201EB410202EBB2
:103E5000011205EB021101F58051C1F8580BBDF8B4
:103E600000003844407C0021FDF79AFDBDF80C109D
:103E700001EB410202EB011205EB021101F5805149
:103E800081F85C0BBDF80C0000EB400101EB001168
:103E900005EB011000F5805090F8560B06285046AF
:103EA0005DD0ADE0BDF80000BDF804100844384412
:103EB000807C0021FDF774FDBDF804204FF0030A5B
:103EC000B2FBFAF2BDF80C1001EB410303EB011158
:103ED00005EB011101EB021101F5805181F8800B16
:103EE000BDF80000BDF8041008443844C07C00212F
:103EF000FDF756FDBDF80420BDF80C10B2FBFAF238
:103F000001EB410303EB011100E08EE305EB01112E
:103F100001EB021101F5805181F8810BBDF8000021
:103F2000BDF8041008443844007D0021FDF738FD39
:103F3000BDF80420BDF80C10B2FBFAF201EB41030E
:103F400003EB011100E061E305EB011101EB02114C
:103F500001F5805181F8880BBDF80400C01CADF854
:103F60000400BDF80C0000EB400101EB001005EB74
:103F7000001000F5805090F8570BBDF8041000EBCE
:103F8000400088428ED84EE0BDF80000BDF8041015
:103F900008443844807C0021FDF702FDBDF80C1078
:103FA00001EB410202EB0111BDF8042005EB011108
:103FB000520801EB021101F5805181F8800BBDF828
:103FC0000000BDF8041008443844C07C0021FDF70F
:103FD000E7FCBDF80C1001EB410202EB011101E01E
:103FE0009AE1A1E1BDF8042005EB0111520801EBB3
:103FF000021101F5805181F8810BBDF80400801C8D
:10400000ADF80400BDF80C0000EB400101EB00101E
:1040100005EB001000F5805090F8570BBDF8041028
:10402000B1EB400FB0D3BDF80C100220F5F7DAFD6C
:10403000BDF80C00C0B2FEF789F9BDF80C000121F3
:1040400000EB400205EB820000F5805080F871160D
:10405000D7E2BDF800003844007A84F8AD03BDF81B
:1040600000003844407A84F8AC03BDF800003844BE
:10407000807A84F8AB03BDF800003844C07A84F835
:10408000AA03BDF800003844007B84F8A903BDF8FA
:1040900000003844407B84F8A80304F56A74F5F7FF
:1040A000C3FCF5F785FC2078A4F56A74FF2829D1B4
:1040B000F5F734FCBDF800003844007A84F8AD030D
:1040C000BDF800003844407A84F8AC03BDF8000025
:1040D0003844807A84F8AB03BDF800003844C07AD5
:1040E00084F8AA03BDF800003844007B84F8A903D3
:1040F000BDF800003844407B84F8A803F5F794FC31
:10410000F5F756FC1D48406D08B10F2000E00E2069
:1041100084F8660775E2102084F86607BDF8000091
:104120003844007A84F8AD03BDF800003844407A82
:1041300084F8AC03BDF800003844807A84F8AB03FF
:10414000BDF800003844C07A84F8AA03BDF8000026
:104150003844007B84F8A903BDF800003844407B54
:1041600084F8A80304F56A74F5F75EFC02F0DEF843
:10417000A060A068A068A4F56A7442E2D41200208E
:104180000E2084F8660784F8A1A13AE25146ADF802
:104190000CA0FE4D3EE0ADF8041016E0BDF80C009A
:1041A00000EB400202EB0010BDF8042005EB00100C
:1041B00000EB021000F5805090F8820BC00714D17C
:1041C000BDF80400401CADF80400BDF80C0000EB85
:1041D000400202EB001005EB001000F5805090F853
:1041E000570BBDF804209042D8D8BDF80C0000EB66
:1041F000400202EB001005EB001000F5805090F833
:10420000570BBDF80420904208D8BDF80C00401CA4
:10421000ADF80C00BDF80C000428BCD3BDF80C00B0
:1042200004286FD3DA4B8A465970DA490120C1F865
:104230008802C1F8880294F8A501E0B30D2084F843
:104240006607BDF800003844407ABDF800103944D4
:10425000097A40EA0120ADF80800BDF800003844B2
:10426000C07ABDF800103944897A40EA01205880AC
:1042700000204FF4007CBDF80010014439440A7B53
:10428000291801F5805181F8A621401C80B26045B3
:10429000F1D3BF48408800F2FF3081B20120F4F72B
:1042A00097FE40B184F8A1A1B948418864225143E6
:1042B000BDF8082000E022E0B1FBF2F184F8A01183
:1042C0000121A9714188491C41804088BDF808102E
:1042D000884214D994F89C0140F0010084F89C01B4
:1042E00094F89C0120F00600801C84F89C01BDF825
:1042F0000800A4F89E0100210120F5F773FC504648
:1043000059E1FFE7102084F8660794F89C0140F01B
:10431000800084F89C0174E1BDF800003844007A04
:1043200084F8A1011120F3E65146ADF80CA0974D99
:104330003EE0ADF8041016E0BDF80C0000EB4002C2
:1043400002EB0010BDF8042005EB001000EB02109A
:1043500000F5805090F8820BC00714D1BDF804001E
:10436000401CADF80400BDF80C0000EB400202EB6D
:10437000001005EB001000F5805090F8570BBDF8C9
:1043800004209042D8D8BDF80C0000EB400202EBAC
:10439000001005EB001000F5805090F8570BBDF8A9
:1043A0000420904208D8BDF80C00401CADF80C0069
:1043B000BDF80C000428BCD3BDF80C0004287CD345
:1043C000734B0020587073490120C1F88802C1F86E
:1043D000880294F8A501E8B3122084F86607BDF8B6
:1043E00000003844007A84F8A10194F8A101401E2D
:1043F000ADF80C000020BDF80010014439444A7AA1
:10440000BDF80C1001EB410C0CEB011105EB011197
:10441000014401F5805181F85E2B401C80B20A28CE
:10442000E9D3BDF800003844007DBDF800103944E0
:10443000C97C40EA0120ADF80800BDF8000038440E
:10444000807DBDF800103944497D40EA0120588044
:10445000002000E059E04FF40072BDF80010014464
:10446000394491F817C0291801F5805181F8A6C187
:10447000401C80B29042F0D358889A46BDF80C1088
:1044800000EB8120401E81B20320F4F7A1FDE0B3D0
:10449000BAF80210504664225143BDF80820B1FB1F
:1044A000F2F184F8A0110121A971BAF80210491C97
:1044B000AAF80210BAF8021000E0A2E0BDF8082045
:1044C000914243D9002041F68932BDF80C1001EB2E
:1044D000410303EB011105EB011101EB0011114444
:1044E0000B7843F001030B70401C80B21028ECD312
:1044F000BDF80C0000EB400101EB001005EB0010D3
:1045000041F668310844027800E053E042F00102CD
:104510000270BDF80C0000EB400202EB001005EB4E
:1045200000100844017821F00601891C0170BDF8D3
:104530000810BDF80C0000EB400202EB001005EB88
:10454000001000F58050A0F86A1B2EE0408801287A
:1045500030D1002041F68932BDF80C1001EB410347
:1045600003EB011105EB011101EB001111440B7874
:1045700023F001030B70401C80B21028ECD3BDF86F
:104580000C0000EB400101EB001005E0D41200200C
:10459000180A00200000424205EB001141F6683085
:1045A0000844017821F001010170BDF80C100220CF
:1045B000F5F718FB00202A49C1F88802C1F88802E3
:1045C0001FE046E0274D686D0A21B0FBF1F0BDF811
:1045D00000103944097A884213D1BDF800003844EC
:1045E000007A18B1686D0A38686504E0C5F854A00F
:1045F000102084F8660700210520F5F7F3FA012062
:10460000A871B4F82A0620B300201EE0002001465D
:10461000BDF800200244B954401C80B20528F7D3ED
:10462000A4F82A1607B0BDE8F08F0020A4F82A06E7
:10463000F8E7BDF800103144014439448978BDF8E9
:1046400000200244B954401C80B2B4F82A168142BA
:10465000EFD8B4F82A0600287EF4BFABE2E70000EA
:1046600000004242D41200202DE9F74F002084B010
:10467000FF4D019006468146009095F86606012898
:104680007ED195F8620701287AD1A5F5805809EB0B
:10469000490101EB091108EB0110002700F5805BCF
:1046A00002905DE0029800EB071404F5805494F842
:1046B000820B000652D594F8820B40F0040084F877
:1046C000820B94F8820B000748D594F8820B20F0F7
:1046D000080084F8820B0020C1F8350009EB0911AD
:1046E00001EB092108EBC10007EB071100EBC10A40
:1046F00042F2390151441022DE4804F53864F3F7E0
:10470000A4FD0AF500504146D0F8312041F8192F98
:10471000D0F835204A60227888F81820C16CC8F893
:104720002110D54940468A6A40F8392F898D818009
:104730006168C8F83F10D8F8540081B20220F4F73D
:1047400047FC00210620F5F74DFAD8F85400401C2C
:10475000C8F8540000210520F5F744FA7F1CBFB2C9
:104760009BF8570B4146B8429CD849460220F5F7C2
:1047700039FA09F101001FFA80F9B9F1040F00E0DC
:1047800006E084D3002085F862070B2085F86607D1
:10479000BA4F0020387000980DE001F0C7FDC5F851
:1047A000B003D5F8B003C0F300400190D5F8B003D2
:1047B000C0F3420000900028EFD095F86407AF499D
:1047C0003A31022816D1AE4890F872222AB100215F
:1047D00080F8721201F074FBFEE307265520087082
:1047E000FD204870AA2088700020C87008716122DE
:1047F0004A718871F52088550020D5F8B013C0F1B2
:104800000302D200D1409D4A33183A321A44D17083
:10481000401C80B20428F0D395F8630720B1994872
:10482000D0F80802A0B907E0944906983A3131441B
:10483000C87106F108042FE08E482538007838B199
:1048400095F86407032803D0012085F86606D4E3B1
:10485000884A8A4B0020253A3A33111801F58051D5
:1048600091F8E91634181C44E171401C80B21428F8
:10487000F3D30020111801F5805191F87417341802
:104880001C44E176401C80B20A28F3D3991906989B
:1048900081F8250006F12604002C9DD0069885F8A5
:1048A000270606981021FF2211287DD008DCA0F1F0
:1048B0000B00062817D2DFE800F01616EA08E91701
:1048C000A22810DA12280ED13DE285F866176B4A4D
:1048D00000206D493A3227180B5CD355401C80B23A
:1048E0000A28F8D30A3440E395F89C01C0077CD02D
:1048F000012080F31388FDF739FF00EB400101EB45
:104900000A105C49253901EB0017029707F580571B
:1049100097F8560B032816D097F8560B012812D09B
:1049200097F8560B02280ED097F8560B04280AD099
:1049300097F8560B894605287ED097F8560B0B46FC
:1049400006287AD07AE14D4A01203A321055E41C0B
:10495000A0B2022303901354401C80B21D231354B1
:10496000401C84B20020C4E00298944600EB091277
:1049700002F5805292F8800B40493A310855641C88
:1049800092F8823BA0B20B54401C84B292F8820B86
:10499000400707D492F8820B000703D492F8820BE9
:1049A000800764D5002000E072E1D2F8843BC0F1BA
:1049B00003084FEAC80823FA08F300EB040801F8DB
:1049C0000830401C80B20428EDD3241DA3B20AEBAA
:1049D0000A1404EB0A220CEBC20409EB091204EBE3
:1049E000C208002008F5005200E02AE1D2F8314068
:1049F000C0F1030C4FEACC0C24FA0CF400EB030CCE
:104A000001F80C40401C80B20428EDD31B1D9BB262
:104A10000020D2F83540C0F1030C4FEACC0C24FA48
:104A20000CF400EB030C01F80C40401C80B204288D
:104A3000EFD31B1D9BB201E06CE0A2E00020D46C20
:104A4000C0F1020C4FEACC0C24FA0CF400EB030C7E
:104A500001F80C40401C80B20328F0D3DB1C1FFA85
:104A600083FB002408F50050D0F8390010E03DE049
:104A7000D4220020F912002054260020180A002019
:104A8000D452002000004042B0A4010894E1DFE0CD
:104A900008F50051D1F83D10C4F10502D200F3F73A
:104AA000C2FBFF4904EB0B028854641CA4B2062C21
:104AB000D8D30BF106001FFA80FB002408F5005044
:104AC000D0F8410008F50051D1F84510C4F10502B5
:104AD000D200F3F7A8FBF24904EB0B028854641CE4
:104AE000A4B2062CEAD30BF1060084B209F101004E
:104AF00080B2EC4A97F8571B814649453FF634AFE0
:104B00000398E749039A201A1144030A01F8023D69
:104B1000487093E0DFF888C302200CF80400E41C1E
:104B2000A4B22746002221E0531C0CF8043009EB04
:104B3000020101F58051641C91F84515A0B20CF8F2
:104B40000010401C81B2002009EB0214221802F56B
:104B5000805292F8512500EB01080CF80820401C07
:104B600080B21028F2D310318CB29AB295F8440575
:104B70009042D9D80CEB0700002100F8021DE11B80
:104B80005BE0C74A03201055E41CA0B20221814615
:104B90001154401C80B20E211154401C84B20021DB
:104BA0009E4693463EE0029800EB011202F5DC526D
:104BB00010780BF80400641CA0B294780BF8004045
:104BC000401C84B2907840072AD50AEB0A1303EB05
:104BD0000A220EEBC20201EB0113002002EBC3021A
:104BE000131803F5005393F8573000EB0408DC4624
:104BF0000BF80830401C80B20A28F1D30A34A3B263
:104C00000020141804F5005494F8704000EB0308D9
:104C10000CF80840401C80B20228F2D39B1C9CB2C6
:104C2000491C89B297F8570B8842BCD80BEB090096
:104C3000002100F8021DA4EB090141700AF10100F6
:104C400080B295F8AC1A824651453FF656AE8CE1DB
:104C50007878401C78707878052803D295F89C0104
:104C6000C00706D085F8661795F89C01C00704D0E8
:104C700005E00D2085F8660701E085F8A021788819
:104C8000010A87480155798820444170A41C6CE1D1
:104C900085F8661795F8A101DFF8048208F804008A
:104CA0000022DFF800C2641C3EE095F8A10102EB8F
:104CB000021700EB001101EB00200CEBC00000EB31
:104CC000C70000F5805090F8080801282AD195F80F
:104CD000A10100EB400101EB00100CEB001000EB18
:104CE000021000F5805090F8500A08F80400641C87
:104CF000A3B2002095F8A11101EB011404EB0121EE
:104D00000CEBC10101EBC701014401F5805191F8A1
:104D100009181C1808F80410401C80B20A28E9D3AE
:104D20000A339CB2521C92B295F8A10100EB4001EB
:104D300001EB00100CEB001000F5805090F8270AF2
:104D40009042B2D811E17878401C787078780528C4
:104D50000ED295F8A10100EB400303EB001351487C
:104D600000EB031000F5805090F8380AC00711D00E
:104D700085F8661795F8A10100EB400101EB0011E1
:104D8000484800EB011000F5805090F8380AC00741
:104D900004D005E0122085F8660701E085F8A0211F
:104DA00095F8A1113E48015579882044090A4170BF
:104DB00079888170E41CD8E0DFF8E890012189F857
:104DC0000610D9F854100A22B1FBF2F234490A5500
:104DD000D9F85400641C0A2804D900204FF00A0AAC
:104DE000029003E0D9F854A00022029201F804A036
:104DF0002220641C085500278B46641CAEE0D9F8BD
:104E00005400C84638B1D8F85400C01B401E81B2C7
:104E10000220F4F771F898F818004346DC460BF8C6
:104E20000400641CA1B20020D3F81920C0F10304CF
:104E3000E400E24044180CF80420401C80B204282E
:104E4000F2D3091D89B20020D3F81D20C0F103045C
:104E5000E400E24044180CF80420401C80B204280E
:104E6000F2D3091D89B20020D3F82120C0F1020439
:104E7000E400E24044180CF80420401C80B20328EF
:104E8000F2D3C91C1FFA81F800249946494651F80B
:104E9000250F4968C4F10502D200F3F7C4F903E015
:104EA000520A0020D412002004EB08020BF8020082
:104EB000641CA4B2062CE9D308F106001FFA80F89E
:104EC0000024494651F82D0F4968C4F10502D2006B
:104ED000F3F7A9F904EB08020BF80200641CA4B272
:104EE000062CEED308F1060099F83E3080B2494610
:104EF0005A460BF80030401C99F83D3080B20BF850
:104F00000030401C99F83C3080B20BF80030401C57
:104F100099F83B3080B20BF80030401C91F83A30E1
:104F200080B21354401C91F8393080B21354401CA5
:104F300083B20020D1F83F40C0F1030C4FEACC0C03
:104F400024FA0CF400EB030C02F80C40401C80B275
:104F50000428EFD31B1D7F1C9CB2BFB2029A002015
:104F6000B7EB0A019041FFF64AAFA71B24493A0A62
:104F7000881981464270877000238A460BE0F11839
:104F800051448846C879DDE90021F4F7A7FD88F887
:104F900007005B1C9BB29F42F1DC95F8A70328B188
:104FA000B9B2484600230422F5F7FEFCB9B25646D2
:104FB0004846F4F781FB010A3155641CA1B27054D4
:104FC000491C95F864078CB202280CD1601F010AB5
:104FD000F170307181B200E00FE0701D01F0EDFA68
:104FE0003055641CA4B2074804600121001FF4F787
:104FF000B9FB204607B0BDE8F08F0020FAE70000BB
:10500000520A0020BC64024070B5164C40F22445A0
:105010002946204603F06BFB002821D02946204674
:1050200003F002FB104D00212846F4F79BFB6110B2
:105030002846F4F781FB0D49012081F86507208897
:10504000A088281D0268C2F5FA62A1F82A264FF44A
:10505000FA6101602846BDE870400121F4F782BB87
:1050600070BD00000010014088640240D42200207E
:1050700010B5074C05492046F4F75EFB0021204699
:10508000F4F770FB03490120087010BD0080002870
:10509000B8640240180A00202DE9F04301218FB0C6
:1050A000880501F099F8DFF894904846F4F764FB1E
:1050B0004020050103900024CDE90545C602079470
:1050C0000894CDE909464FF000681E480B940C94F3
:1050D0000D941B4FCDF800800E94CDE90170694608
:1050E0004846F4F7F1FB012210214846F4F7D6FBBD
:1050F000DFF84890A9F130094846F4F73DFB4FF43A
:10510000FA60CDE90340CDE9054507940894CDE95F
:1051100009460D480B940C940D94CDF800800E9424
:10512000CDE9017069464846F4F7CEFB01214846B7
:10513000F4F718FB0FB0BDE8F0830000B86402403C
:1051400004100140520A0020607200207CB5012149
:10515000032001F041F8134D072206212846F5F7F8
:1051600047F9072211462846F5F742F9C0200221E7
:1051700000908DF8051000248DF8064001208DF870
:1051800007008DF8041069462846F5F7F5F8072062
:1051900000908DF804408DF8074069460248F5F705
:1051A000EBF87CBD00040240000002402DE9F04114
:1051B0000024FFF7CBFFFFF76FFF4FF4E13000F063
:1051C00089F800F069F80121402001F01DF8012064
:1051D00001F09EF82D490B2081F82A0100250D765B
:1051E0008D764D76CD764FF47A70086281F828502E
:1051F000012381F82A3081F8293081F82B30C20050
:105200000A630D708B704B70CB7088600D738B735D
:105210004B73CB7342104A611D4A157095705370E1
:10522000D37042F2107696601A4E42F6F827A1F239
:105230003C6104EB440206EB8202A2F5196202F51E
:105240000052157095705370D5709760641C042CD3
:10525000EFD391F86127120706D091F8612702F089
:105260000F02521E81F8632791F86127120906D0B8
:1052700091F86127FF2303EB121281F8642704F0F1
:10528000EFFEBDE8F04100F023B900001029002036
:1052900044550020D412002038B546208DF8000077
:1052A00002208DF8010001248DF802408DF80340A2
:1052B0006846FDF71FFA25208DF800008DF80140A3
:1052C00000208DF802008DF803406846FDF712FAC1
:1052D00038BD00001FB504460121102000F0B8FFC2
:1052E0000020ADF804000094ADF80600ADF8080009
:1052F000ADF80C000C200D4CADF80A0069462046B4
:1053000003F02CFA0121204603F091F9012240F22A
:105310002441204603F00AFA1021204603F084F9C4
:105320000122C021204603F08CF91FBD001001406E
:105330002DE9F04F8DB034225E496846F2F785FFC3
:105340005D4F002697F8630700287DD0DFF86CB129
:105350000121CBF888124FF0000987F86597584D66
:10536000584C02E0A85DA055761C5548F2F78BFF1B
:10537000B042F7D8DFF85081C8F800600121A8F1E9
:105380000400F4F7EFF94FF4FA7004F069FE87F8BF
:105390006597DFF82CA100260AF17C0A03E01AF8D1
:1053A0000600A055761C46487C30F2F76CFFB042F0
:1053B000F5D8C8F8006044480121001FF4F7D2F97D
:1053C0004FF47A7004F04CFE87F86597DFF8F0A090
:1053D00000260AF1020A03E01AF80600A055761C1E
:1053E0003748801CF2F74FFFB042F5D8C246C8F8E4
:1053F000006035480121001FF4F7B4F94FF47A70CA
:1054000004F02EFEC84687F86597002602E0A85DE6
:10541000A055761C2A48F2F736FFB042F7D8554619
:10542000CAF80060DFF8A0A00121AAF1040A5046E2
:10543000F4F798F94FF47A7004F012FE23496846A5
:10544000F2F715FF1E4900E030E0891D6846F2F7CB
:105450000EFF87F865870026E94603E019F8060085
:10546000A055761C6846F2F70EFFB042F6D82E60C3
:1054700001215046F4F776F94FF47A7004F0F0FD0C
:10548000464687F865870E4900200A310A5C225497
:10549000401C0728FAD3401E286001215046F4F72B
:1054A00061F9642004F0DCFDCBF888620DB0BDE842
:1054B000F08F00006CAD0108D422002000004242B1
:1054C00050AA0108520A0020BC640240D1290020E1
:1054D0002DE9F04FFE4C89B0002594F86307AB46E8
:1054E00000282AD094F8A106032826D294F8A10611
:1054F000401C84F8A10600210920F4F773FBF5484D
:105500000126C0F8886294F8641741F2B760A4F5E8
:1055100080573844009041F2E9603844DFF8B8839E
:10552000089002290AD094F86407DFF8B0A3002895
:105530007ED094F8640703287BD0F1E0584608F841
:1055400005006D1C642DFAD3824684F86507E34993
:1055500000205A310A5C08F80020401C0828F9D3C2
:1055600041F22571B94600250F4409E009EB050019
:1055700000F5805090F8250708EB050108726D1CB6
:105580003846F2F780FEA842F0D808EB05012C203F
:10559000087241F24D71002709EB010009350190B5
:1055A0000AE009EB070000F5805090F84D17EA1962
:1055B00008F802107F1C0198F2F765FEB842F0D897
:1055C000C7A1C548F2F753FEC348F2F75CFEC549D0
:1055D0000860C4480121001FF4F7C4F806E0012068
:1055E00004F03EFD7F1CB7F57A7F7DD894F86507FF
:1055F0000028F4D094F86307B84A7732022819D00B
:105600000020514647463954401C6428FBD384F897
:1056100065170025505D78556D1C0E2DFAD3009846
:10562000F2F731FE0004000C36D0002549462DE08B
:105630007FE0D4E284F865A70025474604E0A74848
:105640007730405D78556D1CA4487730F2F71BFE2B
:10565000A842F4D8A34805600121001FF4F782F89E
:105660004FF47A7705E0012004F0FAFC6D1CBD428E
:10567000BBD894F865070028F5D017E04A1902F561
:10568000805292F8B7267B199A736D1C8542F5D328
:1056900093A19148F2F7EBFD8F48F2F7F4FD9149A1
:1056A000086090480121001FF4F75CF84FF47A7706
:1056B00094F86507A8B38C488C494A46006808608E
:1056C00089485546001D00684860874808300068D2
:1056D00088600020131803F5805383F8E956401CB6
:1056E0001428F7D3CE7A00E01AE1087A04AF8B7A57
:1056F0004A7A87E84D000879CE798B794A798DE826
:105700004D008B780A787AA1089803F08FF8002171
:105710000320F4F767FA002802D06E48C0F88852D8
:10572000B4E3FFE7012004F09BFC6D1CBD42BFD930
:10573000A4E384F865B7DFF8A491A9F17C0904E03B
:1057400019F8051008F805106D1C64487C38F2F74C
:105750009AFDA842F4D8634805600121001FF4F7C0
:1057600001F84FF4FA7004F07BFC84F865B700256B
:1057700004E01AF8051008F805106D1C5748F2F7F8
:1057800082FDA842F5D8574805600121001FF3F7B4
:10579000E9FF4FF47A7004F063FC84F865B7DFF832
:1057A0003CA10025AAF17A0A04E01AF8051008F8CD
:1057B00005106D1C49487A38F2F765FDA842F4D807
:1057C000DFF820A1CAF800500121AAF10400F3F784
:1057D000C9FF4FF47A7004F043FC84F865B70025E4
:1057E00004E019F8051008F805106D1C3B487C38DA
:1057F000F2F749FDA842F4D8CAF80050394801210F
:10580000001FF3F7AFFF4FF47A7004F029FCDA467B
:1058100084F865B7002505E030480B38415D08F88D
:1058200005106D1C2D480B38F2F72DFDA842F3D85A
:105830002C4805600121001FF3F794FF4FF4FA791B
:1058400005E0012004F00CFC6D1C4D4568D894F86F
:1058500065070028F5D0D34684F865A7DFF87CA05B
:105860000025AAF13C0A04E01AF8051008F8051012
:105870006D1C1A483C38F2F706FDA842F4D81948C6
:1058800005600121001FF3F76DFF05E0012004F022
:10589000E7FB6D1C4D45D9D894F865070028F5D075
:1058A00084F865B71D48D0F818020C49643970B106
:1058B000002045460A5C2A54401C0D28FAD3009863
:1058C000F2F7E1FC0104090C47D000203EE028E09B
:1058D000D422002000004242520A0020CCAA010833
:1058E0000D0A0000BC640240107AFF1F307A0020CD
:1058F00025303278253032782530327825303278AC
:10590000253032782530327825303278253032789B
:1059100025303278253032782500000000004342DF
:105920004DE2002504E0F948415D08F805106D1CC2
:10593000F648F2F7A8FCA842F5D812E03A1802F5AA
:10594000805292F8B7262B185A73401C8842F5D320
:10595000AFF27401EE48F2F78AFCED48F2F793FCDF
:105960000546EC4805600121001FF3F7FBFE4FF4EC
:105970007A7A05E00A2004F073FB6D1C55458AD83D
:1059800094F865070028F5D0DA4684F865B7002555
:1059900005E0DE483730415D08F805106D1CDB4836
:1059A0003730F2F770FCA842F3D8DA4805600121DD
:1059B000001FF3F7D7FE05E0012004F051FB6D1C3A
:1059C0004D45DCD894F865070028F5D084F865A724
:1059D000002505E0CD484830415D08F805106D1CF4
:1059E000CA484830F2F74FFCA842F3D8C9480560CE
:1059F0000121001FF3F7B6FE05E0012004F030FBA3
:105A00006D1C4D45BBD894F865070028F5D0D346EA
:105A100084F865A7BD4800256E304146425D4A5571
:105A20006D1C0C2DFAD3BB49681E0860B9480121D2
:105A3000001FF3F797FE05E0012004F011FB6D1C39
:105A40004D459CD894F865070028F5D0B2A1B4481C
:105A500004F0A6FC10B3B24B002145189A4605EBA2
:105A60000A0255797A1802F58052B94682F8A25690
:105A7000491C1429F1D394F8FE06A8B3A448A949F7
:105A80003238F2F7F4FBA149A14812393238F2F763
:105A9000EEFB84F865B7002547460CE0012004F0D2
:105AA000DFFA6D1CB5F5FA7FD0D9E7E198483238B6
:105AB000405D78556D1C96483238F2F7E4FBA842F9
:105AC000F4D8944805600121001FF3F74BFE4FF412
:105AD000FA7705E0012004F0C3FA6D1CBD42E4D85A
:105AE00094F865070028F5D0642004F0B9FA84F82A
:105AF00065B7864800257A304146425D4A556D1C9F
:105B00000B2DFAD38349681E086082480121001FCB
:105B1000F3F728FE06E0012004F0A2FA6D1CB5F5AB
:105B2000FA7FC2D894F865070028F4D07EA17C489B
:105B300004F036FC071E3FD0642004F091FA0020E8
:105B40004A465D46111801F5805181F8E956401C1E
:105B50001428F7D3002053463918194491F801C08E
:105B6000111801F5805181F8EEC6401C0F28F3D3BF
:105B700000210320F4F736F810B16C48C0F88852C1
:105B8000642004F06DFA84F86557604900250E39E9
:105B900040464A5D42556D1C072DFAD35D49681E8B
:105BA00008605C480121001FF3F7DCFD642004F06D
:105BB00057FA4FF4FA770DE0012004F051FA6D1C0A
:105BC000B5F5FA7FB2D959E1012004F049FA6D1C0C
:105BD000BD42F8D894F865070028F5D056E184F85E
:105BE00065B704E01AF8051008F805106D1C474861
:105BF0006430F2F748FBA842F4D84648056001211A
:105C0000001FF3F7AFFD4FF47A7004F029FA84F81F
:105C100065B7DFF8F8A00025AAF1160A04E01AF823
:105C2000051008F805106D1C38481638F2F72BFBE4
:105C3000A842F4D8374805600121001FF3F792FD10
:105C40004FF47A7004F00CFAD94684F865B7DFF89F
:105C5000BCA00025AAF1180A04E01AF8051008F8FB
:105C600005106D1C29481838F2F70DFBA842F4D82E
:105C7000DFF8A0A0CAF800500121AAF10400F3F750
:105C800071FD4FF47A7004F0EBF9CB4684F8659718
:105C9000DFF87890002509F1590904E019F805109A
:105CA00008F805106D1C19485930F2F7ECFAA842B3
:105CB000F4D8CAF8005017480121001FF3F752FD2D
:105CC0004FF4FA7905E0012004F0CAF96D1C4D4546
:105CD00075D894F865070028F5D084F865B70025D5
:105CE00005E00A48AF30415D08F805106D1C074813
:105CF000AF30F2F7C8FAA842F3D8CAF80050054806
:105D00000121001FF3F72EFD18E0000068AA01082A
:105D1000520A0020BC64024049434349443A00000F
:105D200060720020D1290020493A00000000424260
:105D3000012004F095F96D1C4D4540D894F8650795
:105D40000028F5D084F865B794F86307564902280F
:105D50000ED0002045460A5C2A54401C0D28FAD378
:105D60000098F2F790FA0104090C1DD0002014E00D
:105D7000002504E04C48415D08F805106D1C4A48B8
:105D8000F2F781FAA842F5D812E03A1802F58052EB
:105D900092F8B7262B18DA73401C8842F5D3AFF27D
:105DA000C0414248F2F763FA4048F2F76CFA054600
:105DB000CAF8005001213E48F3F7D4FC07E05DE04B
:105DC0000A2004F04DF96D1CB5F57A7F56D894F889
:105DD00065070028F4D0374837495D4600680860F9
:105DE0003448001D00684860324808300068886008
:105DF00000203A1802F5805282F8E956401C142817
:105E0000F7D3087A0DF1100CCF7A8B7A4A7A8CE8A6
:105E10008D000879CF798B794A798DE88D008B7860
:105E20000A78AFF23451089802F000FD00210320F7
:105E3000F3F7D8FE10B12148C0F88852642004F06E
:105E40000FF984F865571849002540468C394A5D9A
:105E500042556D1C072DFAD3681ECAF800000121B7
:105E60001348F3F77FFC642004F0FAF84F4609E08A
:105E7000012004F0F5F86D1CBD4203D986F31388A8
:105E8000FCF774FC94F865070028F1D05D4684F8AF
:105E9000A1B600210920F3F7A5FE0848C0F88852F2
:105EA00009B0BDE8F08F0000EDAA0108520A0020F9
:105EB000B8640240107AFF1F307A0020000042428E
:105EC0002DE9F04700205C4F01463954401C6428FE
:105ED000FBD35A4D894685F86517594900200A5C5D
:105EE0003A54401C0828FAD3DFF8588141F2257053
:105EF000002608EB000408E008EB060000F58050DF
:105F000090F82507B9190872761C2046F2F7BBF9FC
:105F1000B042F1D82C20B9190872002441F24D7119
:105F200008EB010A093608E008EB040000F5805090
:105F300090F84D0731197854641C5046F2F7A3F9D4
:105F4000A042F1D840A13C48F2F791F93A48F2F763
:105F50009AF93E4E3060A6F1040A01215046F3F74B
:105F600001FC05E0012004F07BF8641C642C03D8DC
:105F700095F865070028F5D03548D0F81802304963
:105F80001D31B0B100204A463A54401C6428FBD36E
:105F900085F865270024085D3855641C0E2CFAD35B
:105FA0002C48F2F770F90004000C30D00024414670
:105FB00027E085F865970024884603E018F8040078
:105FC0003855641C1E481D30F2F75DF9A042F5D823
:105FD000346001215046F3F7C5FB05E0012004F0D1
:105FE0003FF8641C642C21D895F865070028F5D08B
:105FF0001CE00A1902F5805292F8B7263B199A73F1
:10600000641C8442F5D310A10B48F2F730F90A481A
:10601000F2F739F9306001215046F3F7A3FB05E0B0
:10602000012004F01DF8641C642C03D895F8650762
:106030000028F5D0BDE8F087520A0020D4220020C5
:1060400026AB0108D41200200D0A0000BC640240F7
:10605000000043428B2900202DE9FC5F01215920DB
:1060600000F0BAF800248DF804400220DFF894B064
:106070004FF47C578DF80700009769465846F4F7AF
:106080007BF9FC20DFF8809000908DF8044001251A
:106090008DF8075069464846F4F76EF9DFF86CA0B2
:1060A0004FF440468DF8044000968DF8075069463D
:1060B0005046F4F761F90720DFF8548000908DF81E
:1060C00004408DF8075069464046F4F755F907211A
:1060D0004046F4F7A6F931465046F4F7A2F939469E
:1060E0005846F4F79EF9FC214846F4F79AF9094816
:1060F000D0F828120848012902D00470BDE8FC9F9E
:106100000570FBE70010024000180240000C02403E
:106110000000024000004242D412002010B5FFF7F8
:106120009BFF642003F09CFF1048D0F83C121048FD
:1061300019B1002180F8631710BD0E49D1F818225B
:1061400092B1012280F86327D1F80822D1F80C120D
:1061500042EA4101C94380F8641790F8641701F0DE
:10616000030180F8641710BD0222EBE70080414272
:10617000D4220020000043427CB50121102000F011
:106180002BF84CF20400012400908DF8044000200C
:106190008DF8060003208DF80500084D8DF80740A6
:1061A00069462846F4F7E8F804212846F4F737F959
:1061B0000348C0F8B842C0F8BC427CBD00100240A1
:1061C00000004242FFF7D8BF4FF400610148F4F7E6
:1061D0001FB9000000040240044A0029116801D0E0
:1061E000014300E0814311607047000030380240F5
:1061F000044A0029116801D0014300E08143116085
:106200007047000010380240044A0029116801D08C
:10621000014300E0814311607047000034380240C0
:10622000044A0029116801D0014300E08143116054
:106230007047000040380240044A0029116801D02C
:10624000014300E0814311607047000020380240A4
:10625000044A0029116801D0014300E08143116024
:106260007047000044380240044A0029116801D0F8
:10627000014300E081431160704700002438024070
:1062800070B5204B1968204C11F00C0104D0661039
:10629000042903D0082903D004601BE0066019E03C
:1062A000184A121F1168C1F38055116801F03F01AF
:1062B00015B1B6FBF1F101E0B4FBF1F1146812681D
:1062C000C4F388146143C2F30142521C5200B1FB73
:1062D000F2F1016019680F2202EA11110B4A545CB5
:1062E0000168E14041601C68072505EA9424145DBB
:1062F00021FA04F484601B6805EA5333D25CD14070
:10630000C16070BD083802400024F4000000002085
:1063100005490028086802D040F0040001E020F0A0
:10632000040008607047000000080650014800683B
:10633000704700000808065070B5012080F31088EF
:106340000C4D10212846F4F76AF808212846F4F786
:1063500068F8D720F2F7F4FEFF20F2F7F1FE0446CA
:1063600010212846F4F75DF8002181F310882046BB
:1063700070BD00000000024070B5012080F310885D
:10638000194C0020A080FFF7D7FF000609D4012098
:1063900003F066FEA088401C80B2A080C828F2D31B
:1063A0001EE0A088C8281BD2104D10212846F4F703
:1063B00036F808212846F4F734F89F20F2F7C0FE9B
:1063C000FF20F2F7BDFEFF20F2F7BAFE6070102149
:1063D0002846F4F726F8002080F31088607870BD16
:1063E000002080F3108870BD2212002000000240BF
:1063F00070B5012188B08803FFF712FF0121022048
:10640000FFF7EAFE00244FF400602F4E8DF80440A1
:1064100000908DF8074069463046F3F7ADFF012143
:106420008DF8041002258DF8055008038DF80640FC
:106430008DF80710009069463046F3F79DFF05225E
:106440000D213046F3F7D4FF05220E213046F3F735
:10645000CFFF05220F213046F3F7CAFF4FF460400B
:1064600000908DF8045003208DF805008DF806404B
:106470008DF8074069463046F3F77EFF134D2846F6
:1064800000F04AF8ADF810406815ADF81200182079
:10649000ADF814000720ADF81800ADF808404FF42F
:1064A0008270ADF80C40ADF80A00ADF80E40ADF8C2
:1064B000164002A9284600F064F80121284600F0A1
:1064C00021F808B070BD0000000402400038004010
:1064D00070B50B4C05460221204600F047F8002815
:1064E000F9D02946204600F04AF80121204600F064
:1064F0003DF80028F9D0204600F03FF8C0B270BD4A
:10650000003800400029018802D041F0400101E03C
:1065100021F0400101807047114910B588420AD12D
:10652000841401212046FFF79FFE2046BDE810405D
:106530000021FFF799BE0B49884202D101210414C2
:1065400004E0094988420AD10121C4132046FFF71B
:1065500073FE2046BDE810400021FFF76DBE10BD60
:106560000030014000380040003C0040024600205E
:1065700012890A4200D001207047808970478181CA
:10658000704730B502884C8802F441530A88CD88A0
:1065900022438C882C4322430C8922434C8922437A
:1065A0008C892243CC8922431A430280828B22F4B5
:1065B00000628283098A018230BD0246002003E026
:1065C00012F8013B1844C0B2491E89B2F8D2704794
:1065D0002DE9F04101218D070024284601F0EEFC51
:1065E000F0B3F4F7D1F9284E002006F580533DE0D2
:1065F00006EB840101F58051D1F880271278012A39
:10660000D1F8802703D05278012A08D02CE01070EE
:10661000D1F880275070D1F88027907030E0D1F801
:106620008027927802BBD1F8802757687F1C57607B
:10663000D1F880275268D1F88077BF68BA4213D367
:10664000D1F880770122BA70D1F88027D278012A58
:1066500016D0D1F880275070D1F88027506000E024
:1066600008E0D1F88017C870641CE4B293F87E1774
:10667000A142BDD82846BDE8F041012101F0E8BBA8
:10668000D1F880174860EFE7D41200200CB5002243
:10669000254900920192086840F4803008604FF468
:1066A000A063086800F4003001900098401C00903E
:1066B000019810B900989842F3D10868800330D54A
:1066C0000120019018484030026842F08052026078
:1066D0001648026842F4804202601348083002689B
:1066E00002600268026002680260031F104A1A60BA
:1066F0000A6842F080720A600A689201FCD50D4A6D
:1067000040F205611160016821F003010160016838
:1067100041F0020101600168C1F381010229FAD14F
:106720000CBD01920CBD000000380240007000401A
:1067300008544007003C02407CB500229FED170A38
:1067400000928DED010A6D4601AC16E0835CA3F169
:106750003006102E05D2009B1B010093865C303E54
:1067600007E0413B062B0CD2009B1B010093865C8B
:10677000373E1E43521CD2B200968A42E6D3002016
:1067800006E0BFEE000A7CBD2A5C2254401CC0B269
:10679000B0EB510FF8D39DED010A7CBD0000000065
:1067A00030B505460022104611E0AB5CA3F1300481
:1067B000102C02D244EA001007E0A3F14104062C99
:1067C00008D20401A3F137002043521CD2B28A42FE
:1067D000EBD330BD4FF0FF3030BD00002DE9FC4160
:1067E0004C4C4FF03808A0780021FBF7D9F8012570
:1067F0000826CDE900650246182000234146FCF733
:10680000E9F9071D07EB47004006000E08232D227B
:1068100041460095FCF770F9607800217F1CFBF77A
:10682000BFF8024607EB4700CDE900654006000EC1
:1068300000234146FCF7CEF9074407EB470040062A
:10684000000E08232D2241460095FCF755F92078CB
:1068500000217F1CFBF7A4F8024607EB4700CDE9B7
:1068600000654006000E00234146FCF7B3F90744DB
:1068700007EB47004006000E082320224146009502
:10688000FCF73AF9607900217F1CFBF789F8024692
:1068900007EB4700CDE900654006000E00234146A6
:1068A000FCF798F9074407EB47004006000E082361
:1068B0002D2241460095FCF71FF9207900217F1C0D
:1068C000FBF76EF8024607EB4700CDE9006540068E
:1068D000000E00234146FCF77DF9074407EB470013
:1068E0004006000E08232D2241460095FCF704F9CE
:1068F000E07800217F1CFBF753F8024607EB4700C6
:10690000CDE900654006000E00234146FCF762F920
:10691000BDE8FC817C2600200249C87001208871F6
:1069200070470000D41200202DE9FC5F00252C46A2
:10693000F3F774FBDFF80C8498F8060000287CD08D
:10694000AB4688F806B0FBF731FF98F80300FE4F1E
:106950004FF0080A4FF0010908F5805610286DD253
:10696000DFE810F010008800F50083017802C4020F
:106970008603420530067D06DD06A5074A08910814
:106980001209ED09F3F7F0FF01280AD0022808D018
:10699000042806D0082804D10220FFF7BDFF86F89E
:1069A000A0B11020CDE9000900214C461523E7A233
:1069B0000846FCF7ACF996F8A10118B3CDE900A49C
:1069C00055460523E6A214210020FCF7A0F9CDE9E5
:1069D000005496F8A121002314211E20FCF7FAF898
:1069E000CDE9005496F8A1010A2300EB400101EB28
:1069F000001008EB001041F62E2142181421282027
:106A0000FCF785F996F8A001FF2826D096F8A0019A
:106A1000CDE900040A2364221E211846FBF7EAFF91
:106A2000CDE900A496F8A02100232D213220FCF707
:106A3000D1F800EB4001322001E0FDE3B8E300EBC8
:106A40004100C0B2082325222D210094FCF754F800
:106A500096F8A001642807D0AAE3CDE900A4152385
:106A60002D21C1A21420E2E286F8A0B10220FFF796
:106A700053FFF1E7F3F778FF01280BD0022809D084
:106A8000042802D0082805D101E0092000E00420F4
:106A9000FFF742FF96F8620738B196F8630738B1FE
:106AA000012808D0022811D108E01523B2A207E07E
:106AB0001523B4A204E01523B6A201E01523B8A261
:106AC000CDE900A900210846FCF721F998F8020059
:106AD000012802D002280CD101E0B54901E0B449F7
:106AE0001231CDE9001909231A460A210020FCF7CA
:106AF000C1F8AF4818234838CDE900094C461A467A
:106B000000216820FCF7B6F8CDE900A4554615230E
:106B1000A8A21A210020FCF7FAF8CDE900541523A9
:106B2000AAA224210020FCF7F2F8CDE90054D8F8FD
:106B30005420002324215420FCF74CF8D8F85400AA
:106B400010B90220FFF7E8FEFFF748FE84E7F3F7ED
:106B50000BFF012817D0022815D0042802D00828DE
:106B600011D107E096F89C0120F0800086F89C0186
:106B7000092006E096F89C0120F0800086F89C0130
:106B80000420FFF7C9FE96F8620738B196F863074C
:106B900068B101280ED0022814D118E0CDE900A96F
:106BA000002115238DA20846FCF7B1F815E0152346
:106BB00074A201E0152377A2CDE900A900210846BF
:106BC000FCF7A5F896F827060F2803D005E0152353
:106BD00073A2F1E70120FFF79FFE98F80200012859
:106BE00002D0022811D106E071480923CDE900093D
:106BF0001A460A2106E06E4909231231CDE900192F
:106C00001A460A210020FCF735F896F8A00110B1C9
:106C10000020FFF781FE664818234838CDE90009B7
:106C20004C461A4600216820FCF724F81025CDE9CF
:106C300000542B466BA214212820FCF768F8CDE9FC
:106C400000A4152369A224211220FCF760F896F80D
:106C50009C0100067FF578AFCDE90054102368A2AF
:106C60002E210020FCF753F86EE7F3F77DFE012894
:106C700006D002280BD0042812D0082810D114E026
:106C800098F8040060B198F80400401E06E098F8F7
:106C90000400402804D298F80400401C88F804003E
:106CA00098F80300032805D0D6E60220FFF734FE4B
:106CB0005846F3E73E4801220021A43001F066F86F
:106CC0001024CDE9004998F8040000EB8001C1EBE5
:106CD0008010404490F85C20002319465020FBF7B8
:106CE00079FF0326CDE9006B10235D464AA21946C1
:106CF0000020FCF70CF8CDE9004998F8040000EBFF
:106D00008001C1EB80104044D0F85D20002319467B
:106D10005020FBF75FFFCDE90065102343A2182147
:106D20000020FBF7F4FFCDE9004998F8040000EBE0
:106D30008001C1EB80104044D0F861200023194647
:106D400050207DE0D4120020000042424669726D5E
:106D500077617265446F776E6C6F6164000000004C
:106D6000506F72743A000000446F776E6C6F61640C
:106D7000204661696C2100004E6F205369676E6187
:106D80006C000000547970653A53746174696F6ED9
:106D900000000000547970653A436C6F7564000020
:106DA000547970653A436C6F75642D546573740043
:106DB000F4C901084F66666C696E65205265636FA1
:106DC00072642055706C6F61640000005265636FDF
:106DD0007264206E756D6265723A00004F66666C73
:106DE000696E6500424C5545534B5900454E45521E
:106DF000475920544543484E4F4C4F4759000000D7
:106E0000557067726164652045525220436865631E
:106E10006B2047756E0000004C3A20202020202077
:106E2000202020202020202000000000503A202098
:106E300020202020202020202020202000000000D2
:106E4000FBF7C8FE1023AFF2EC02CDE9006500218C
:106E5000502008E6F3F788FD012806D002280BD061
:106E6000042813D0082824D128E098F8040000B39F
:106E700098F80400401E06E098F80400032818D291
:106E800098F80400401C88F8040012E098F8040008
:106E900030B1012806D0022806D0032809D105E028
:106EA000052004E0062002E0072000E00820FFF7AC
:106EB00033FD98F80300042805D0CDE50220FFF744
:106EC0002BFD5846DFE704220021FE4800F05EFF5C
:106ED0001021CDE9001B98F80400FA4901EB0012DB
:106EE00098F804000007010E1023F6E3F3F73CFDC9
:106EF000082802D10420FFF70FFD98F803000528A9
:106F0000DBD1F04804220021403000F03FFF96F82A
:106F1000630720B101280AD0022823D12EE01023D4
:106F2000AFF2A012CDE900A91946002018E04C46A6
:106F300057461023AFF2A412CDE900A9194600204C
:106F4000FBF7E5FECDE900741023DFA23821002015
:106F5000FBF7DDFECDE900741123DD4A38211E2048
:106F6000FBF7D5FE96F8640708B396F86407012886
:106F70001DD096F8640702285AD06DE5CDE900A926
:106F800010234C465746D3A219460020FBF7BFFEFC
:106F9000CDE900741023CCA238210020FBF7B7FE06
:106FA000CDE9007411233821CE4A1E20D8E744468B
:106FB000601900F5805090F8A20618B96D1CADB2AA
:106FC000152DF5D3CDE900A94E4657461023C6A28C
:106FD0001A210020FBF79BFE601941F2A2614218C2
:106FE000CDE9007610231A212020FBF790FECDE991
:106FF00000761023BEA224210020FBF788FEB44AAD
:10700000CDE900762421102339320846FBF77FFEB4
:10701000CDE900761023B8A22E210020FBF777FEE1
:10702000AB4ACDE900760F232A322E21242075E3C6
:10703000CDE900A94C4655461023B1A21A210020E3
:10704000FBF765FEA24ACDE90054102361321A21F4
:107050001E20FBF75CFECDE900541023A6A22421DC
:107060000020FBF754FE9A4A142325322E21FDE31B
:10707000F3F77AFC012804D0022809D0082814D19B
:1070800010E098F8040080B198F80400401E06E073
:1070900098F80400032808D298F80400401C88F8E7
:1070A000040002E00420FFF737FC98F8030047468D
:1070B00006287DD1834804220021C03000F066FEFE
:1070C0004E461020CDE900063A79B946B84601236C
:1070D00000213E20521CFBF77DFDCDE900A657465E
:1070E000102389A200214820FBF711FEDFF8D4A16C
:1070F0000823AAF1740ACDE900A61A4600217820D7
:10710000FBF7B8FDCDE90076102382A208214820C4
:10711000FBF7FDFD08231A4619467820CDE900ABA0
:10712000FBF7A8FDCDE9007610237DA219460020CB
:10713000FBF7EDFD98F8040000EB400101EB0011B6
:1071400008EB011000F5805090F85D0B4FF0100334
:10715000012842D074A2CDE9007610211E20FBF751
:10716000D6FDCDE90076B846102371A21821002083
:10717000FBF7CDFD99F8040000EB400101EB001096
:1071800009EB001000F5805090F8560BCDE9008611
:10719000052899F8040000EB400101EB001009EB11
:1071A000001000F580501AD090F8560B634900E0AB
:1071B00007E201EB00120C2318213620FBF7A7FD94
:1071C0000120CDE9008010235DA220210020FBF7E3
:1071D0009EFD09264FF0200BF6E05CA2BBE790F87D
:1071E0005C0B56497031E2E706EB46014FF07A0935
:1071F000B9EB410F02D2641CA4B20026387900EB2F
:10720000400101EB001007EB001000EB051000F54A
:10721000805090F8820BC009CDE90080387900EBEE
:10722000400101EB001007EB001000EB051000F52A
:10723000805090F8802B00E0F1E30BEBC400C1B26A
:1072400006EB46004006000E0023FBF7C3FC30446B
:1072500086B206EB4601CA46B9EB410F02D2641C66
:10726000A4B20026387900EB400101EB001007EBD7
:10727000001000EB051000F5805090F8820BD94605
:10728000C00900900BEBC400C1B206EB46004006FB
:10729000000E08232D22FBF72FFC761CB6B206EB5E
:1072A0004601BAEB410F02D2641CA4B20026387921
:1072B00000EB400101EB001007EB001000EB0510A4
:1072C00048E0000018CA010855524C3A000000007E
:1072D00098290020547970653A436C6F75642D5479
:1072E0006173740075AA01084943434944000000D2
:1072F00041504E203A000000494D45493A000000F7
:10730000535349443A0000004F6E4C696E65203A71
:10731000200000004F66664C696E653A2000000050
:10732000547970653A00000052533438350000003B
:1073300050726F746F636F6C3A00000018CB0108D5
:1073400047756E2D416464723A0000004C4F524103
:107350000000000000F5805090F8820BC009CDE9D4
:107360000080387900EB400101EB001007EB0010C2
:1073700000EB051000F5805090F8812B09EBC4005C
:10738000C1B206EB460040064F46000E0023FBF755
:1073900021FC304486B206EB4601BAEB410F02D223
:1073A000641CA4B200260120009007EBC400C1B207
:1073B00006EB46004006000E08233B22FBF79CFB31
:1073C000761C6D1CB6B2ADB2FB4F387900EB4001B4
:1073D00001EB001007EB001000F5805090F8570B00
:1073E000A8423FF601AFECE0F3F7BEFA012804D063
:1073F000022809D0082814D110E098F8040080B1C0
:1074000098F80400401E06E098F80400032808D20B
:1074100098F80400401C88F8040002E00420FFF7FC
:107420007BFA98F803000728DDD1012688F806606A
:1074300004220021E14800F0A9FC1020CDE900065B
:1074400098F80420012300214020521CFBF7C2FBC6
:10745000CDE900A6D1461023D9A214210020FBF7C4
:1074600056FC09269EE006EB46014FF07A08B8EB81
:10747000410F02D2641CA4B200264FF0010BCDE9EB
:10748000009B387900EB400101EB001007EB001086
:1074900000EB051000F5805090F8802B4FF0140A97
:1074A0000AEBC400C1B206EB46004006000E002302
:1074B000FBF790FB304486B206EB46017A20B0EB36
:1074C000410F02D2641CA4B200260AEBC400C1B270
:1074D00006EB4600D846CDF800B04006D346000E75
:1074E00008232D22FBF708FB761CB6B206EB4601FB
:1074F0004FF07A0ABAEB410F02D2641CA4B2002604
:10750000CDE90098387900EB001101EB002007EB82
:10751000C00005EB051100EBC10000F5005090F82C
:107520005400642110FB01F0020A0BEBC400C1B24D
:1075300006EB460040065F46000E0023FBF74AFBC1
:10754000304486B206EB4601BAEB410F02D2641C0E
:10755000A4B2002607EBC400C1B206EB4600400609
:10756000000E08232522CDF80080FBF7C5FA761C13
:10757000B6B206EB4601BAEB410F02D2641CA4B2CC
:10758000002607EBC400C1B206EB46004006000E21
:1075900008233B22CDF80080FBF7AEFA761C6D1C69
:1075A000B6B2ADB2844F387900EB400101EB001068
:1075B00007EB001000F5805090F8570BA8423FF6FB
:1075C00052AFDAE3F3F7D0F9082802D10420FFF72D
:1075D000A3F998F803000828F3D178480422002181
:1075E000403000F0D3FBCDE900A94E4657461023AA
:1075F000764A14210020FBF78AFBC14605EB4500C3
:1076000000EB051109EB011841F6683010F808008D
:10761000C0071FD005EB8501142000EB4104CDE924
:107620000076E1B205236AA20020FBF770FBCDE9EA
:107630000076E1B201236A1C1E20FBF7CBFA41F66B
:107640005E31CDE9007608EB0102E1B20A232A207F
:10765000FBF75DFB6D1CADB2042DCFD38DE3F3F7CB
:1076600083F9012806D002280DD0042815D0082857
:1076700037D13BE098F8040018B198F80400401E98
:1076800028E0052026E098F80400052803D298F8A1
:107690000400401C1EE058461CE098F80400062830
:1076A0001FD2DFE800F003050709111B0A2016E0CE
:1076B0000B2014E00C2012E00D20FFF72DF996F8B6
:1076C000610700F00F0005E00E20FFF725F996F89E
:1076D0006107000988F8040003E01EE00F20FFF7AF
:1076E0001BF998F80300092804D046E30220FFF7AD
:1076F00013F9D0E798F80400304C0422803404EBEE
:107700000010002100F042FB1021CDE9001B98F889
:1077100004000B4604EB00120021002031E2F3F7D5
:1077200023F9012806D002280BD0042813D00828FA
:107730006AD16EE098F8040040B398F80400401E47
:1077400006E098F8040003285ED298F80400401C74
:1077500088F8040058E098F8040000EB400101EBC1
:10776000001008EB001000F5805090F85D0B012828
:107770000DD098F8040000EB400101EB001008EB7D
:10778000001000F5805090F85D0B28B33CE098F8AD
:1077900004005C4600EB400101EB001008EB001018
:1077A00000F5805080F85DBB98F804100220F2F7D5
:1077B00019FAC7F8884227E0D4120020B8CB010894
:1077C00047756E2D525353493A000000B0A401088A
:1077D000506F72742D00000098F804004C4600EBC6
:1077E000400101EB001008EB001000F5805080F81C
:1077F0005D9B98F80400FAF7A9FDC7F8884298F84D
:1078000004100220F2F7EEF998F803000A2805D0D8
:10781000B3E20920FFF780F8584699E704220021D7
:10782000F74800F0B3FACDE900A94C4655461523B8
:10783000F4A214212820FBF76AFACDE9005498F845
:107840000420012314214620521CFBF7C3F998F8A9
:10785000040000EB400101EB001008EB001000F504
:10786000805090F85D0B01280FD000E01BE098F8E5
:10787000040000EB400101EB001008EB001000F5E4
:10788000805090F85D0B18B10AE01523DFA201E0EB
:107890001523E1A2CDE900541E210020FBF737FAA1
:1078A0001523E0A23221CDE90054002069E1F3F76D
:1078B0005BF8E14C012806D0022812D0042821D020
:1078C000082837D123E098F80400F8B194F8890229
:1078D00018B198F80400FAF739FD98F80400401E32
:1078E0000DE098F80400032824D294F8890218B116
:1078F00098F80400FAF72AFD98F80400401C88F86C
:10790000040017E084F8899284F87D9212E009203F
:10791000FFF702F8584688F804B084F87C9294F88F
:10792000891239B1C7F8880284F8890298F80400EE
:10793000FAF70CFD98F803000B2831D1B048042267
:107940000021403000F022FACDE900A94D4656460C
:107950001523ACA212212820FBF7D9F9CDE9006547
:1079600098F80420012312214620521CFBF732F91B
:10797000CDE900651523B1A21C210020FBF7C7F952
:10798000CDE900651523B3A226210020FBF7BFF93E
:10799000CDE900651523B5A230210020FBF7B7F92A
:1079A00094F88902012826D14D4688F8069094F86B
:1079B0007E0280B1C7F888B284F87EB298F80400DD
:1079C0000121FAF7BBFDCDE900A51523ACA23821B2
:1079D0000020FBF79CF994F8880200280BD084F86B
:1079E00088B2CDE900A51523A9A238210020FBF714
:1079F0008EF9C7F88852C0E1F2F7B6FF012814D01B
:107A0000022812D0042802D008280ED10AE0F1F78B
:107A100013FD142804D0584686F8A70305E0B0E10A
:107A20004846F9E70920FEF777FF98F803000C288D
:107A300074D1734804220021803000F0A7F9CDE909
:107A400000A94C465546152395A21A210020FBF7A4
:107A50005EF9CDE90054152396A224210020FBF7FE
:107A600056F9CDE90054152396A22E210020FBF7EC
:107A70004EF996F8A7034FF0150308B197A200E05E
:107A80009CA238210FE7F2F76FFF012806D00228E9
:107A90000DD0042817D0082845D140E098F80400FC
:107AA00018B198F80400401E0AE0032008E098F896
:107AB0000400032803D298F80400401C00E0584654
:107AC00088F804002FE098F8041096F8610761F335
:107AD000030086F8610700210320F2F783F810B352
:107AE00096F86147022006F5CE76FEF715FFF2F70D
:107AF000CFF886F8C54500210320F2F773F83078F7
:107B000020F001003070307840F006003070A6F8A8
:107B100002B000210120F2F765F81DE133E00920F1
:107B2000FEF7FAFECBE798F803000D282BD1344876
:107B300004220021C03000F029F91024CDE90049C9
:107B400096F861076E4D00F00F0005EB001223461A
:107B500021460020FBF7DBF896F8610798F804103F
:107B600000F00F00884202D0CDE9004B01E0CDE9E2
:107B7000004998F804000C2305EB00122021002096
:107B8000121DFBF7C4F8F8E0F2F7EEFE012806D06C
:107B900002280DD0042817D0082827D12BE098F808
:107BA000040018B198F80400401E0AE0042008E020
:107BB00098F80400042803D298F80400401C00E060
:107BC000584688F8040011E098F8041096F8610708
:107BD00061F3071086F8610700210320F2F702F82D
:107BE00020B10220FEF798FEFDF7E0FA98F80300B6
:107BF0000E2804D0C1E00920FEF78EFEE0E781E008
:107C0000C8CC0108504F52543A0000005459504516
:107C10003A4C4F5241000000545950453A525334A7
:107C2000383500005061737320456E7465722043CF
:107C300068616E6765000000D4520020313A4469E3
:107C400070207377697463682031616E6432204FED
:107C50004E000000323A496E7365727420736C6195
:107C60007665206D6F64756C65000000333A506175
:107C7000737320456E7465722053746172740000D2
:107C800053746174653A53656E64696E67000000F1
:107C900053746174653A436F6D706C657465000070
:107CA000496E7365727420552D4469736B20466963
:107CB000727374005468616E205061737320456E56
:107CC00074657200466F726D61743A464154333286
:107CD0003B4D41583A3332470000000046696E641C
:107CE00020552D4469736B2C4F7574707574696ED3
:107CF0006700000053746174653A49646C65000064
:107D000008CE0108042200211F4800F03FF810248B
:107D1000CDE9004996F861071B4D20F00F00803532
:107D20004219234621460020FAF7F1FF98F8040093
:107D300096F86117B0EB111F3FF419AF14E7F2F793
:107D400013FE01280FD002280DD0042802D00828E5
:107D500009D105E0F1F79CFF89F31388FAF716FDC6
:107D60000920FEF7D9FD98F803000F2805D1064831
:107D700004220021D03000F009F8BDE8FC5FFAF7DA
:107D80007FBEBDE8FC9F0000C8CD01082DE9F84F7B
:107D90000025924688468146012715E000242E01E1
:107DA00009EB040101EB081000EB051000970278C5
:107DB000E006F1B2000E1023FAF79EFE641CE4B256
:107DC000102CEDD36D1CEDB25545E7D3BDE8F88F0F
:107DD000064800210172817201214172C172642240
:107DE000026181710220FEF797BD0000D4120020CD
:107DF000124810B5016841F4700101601048016833
:107E000041F0010101600E4A002108321160026850
:107E10000C4B1A400260031D0B4A1A60026822F4E0
:107E20008022026006480C300160FEF72FFC0349F7
:107E30004FF000608039086010BD000088ED00E060
:107E400000380240FFFFF6FE10300024FEF7C0BBF2
:107E5000C943018270470029018802D041F0010125
:107E600001E021F00101018070470000464910B592
:107E7000884206D101210846FEF7F6F900210120CB
:107E80005BE0B0F1804F09D0404988420DD101211B
:107E90000220FEF7D1F90021022070E001210846FE
:107EA000FEF7CAF90021012069E03949884206D16C
:107EB00001210420FEF7C0F9002104205FE03549CC
:107EC000884206D101210820FEF7B6F900210820DA
:107ED00055E03149884206D101211020FEF7ACF966
:107EE000002110204BE02D49884206D1012120209D
:107EF000FEF7A2F90021202041E02949884206D15D
:107F000001210220FEF7B0F90021022015E02549E9
:107F1000884202D101210C040AE02349884202D19F
:107F200001214C0404E0214988420AD101218C043A
:107F30002046FEF799F900212046BDE81040FEF7E3
:107F400093B91B49884206D101214020FEF774F9FC
:107F50000021402013E01749884206D101218020EA
:107F6000FEF76AF90021802009E0134988420AD10E
:107F7000841501212046FEF75FF900212046BDE867
:107F80001040FEF759B910BD000001400004004048
:107F900000080040000C00400010004000140040A9
:107FA00000040140004001400044014000480140FD
:107FB00000180040001C0040002000400246002045
:107FC000138A92890B4202EA010202D0002A00D0F1
:107FD00001207047002A828901D00A4300E08A43C9
:107FE0008281704730B50288164C174DA0420DD0E3
:107FF000A8420BD0B0F1804F08D0144B984205D066
:10800000134B984202D0134B984203D122F07003D5
:108010004A881A43104B984206D0104B984203D01E
:1080200022F440730A891A4302804A68C2620A88AD
:108030000285A04201D0A84201D1897A018601219E
:10804000818230BD00000140000401400004004076
:1080500000080040000C00400010004000140040E8
:1080600010B5FEF75BF8FEF7ADF800F095F9F1F703
:10807000AFFE1348017821F001010170017841F051
:1080800006010170002141800120F1F7ABFDF2F7FC
:10809000BDFBF0F7DDFFF1F741FCF2F77DFCFAF7ED
:1080A000FBFBFFF795FEF1F7FDFFF9F7CFFFFDF7BB
:1080B0007DF804484FF4FA61C1820121017510BDB9
:1080C00070240020D41200202DE9F0470024F2F79C
:1080D000ABF9B04D95F832060026A5F5805701287A
:1080E00005D185F83266F1F763FC0120B87126E10D
:1080F00004EB440007EB800000F5805090F8721606
:10810000012901D180F8726690F87116002970D1AA
:1081100090F8E21A0129FAD104EB440101EB0411B1
:1081200007EB011909F5805292F8561B002960D01F
:1081300080F8E26A92F8560B072859D2DFE800F07F
:10814000DB04315A81D0D00004EB041000EB042092
:1081500007EBC00101F50050C37C012B09D0837CE3
:1081600003EB031301EBC30303F500531B7E002B4A
:108170003ED1837C5B1C8374037C13B1037C8374CA
:108180000674837C03EB031301EBC30303F5005375
:108190001B7E052B2CD0807C00EB001001EBC00077
:1081A0009AE004EB041000EB042007EBC00101F59A
:1081B0000050C37C012B09D0837C03EB031301EB3C
:1081C000C30303F500531B7E002B11D1837C5B1C82
:1081D0008374037C13B1037C83740674837C03EB88
:1081E000031301EBC30303F500531B7E0F2BD2D106
:1081F00081E0A2E004EB041000EB042007EBC001D7
:1082000001F50050C37C012B08D0837C03EB0313E2
:1082100001EBC30303F500531B7EE3BB837C5B1CB4
:108220008374037C13B1037C83740674837C03EB37
:10823000031301EBC30303F500531B7E072BAAD1E5
:1082400059E004EB041000EB042007EBC00303F536
:108250000050C17C012908D0817C01EB011103EBA6
:10826000C10101F50051097EA9B9817C1CE090F89B
:10827000128009EB081C0CF5805C9CF8818B09EBE3
:10828000011C0CF5805C9CF891CBE04504D0817C0E
:10829000491C81740CE022E090F812C00CF1010C32
:1082A00080F812C0491CC9B292F857CB8C45DED871
:1082B000017C11B1017C81740674817C01EB011198
:1082C00003EBC10101F50051097E052913D0807C23
:1082D00000EB001003EBC00000F5005006760AE04A
:1082E00004EB041000EB042007EBC00000F5005085
:1082F000817C491C817404EB041000EB042007EB23
:10830000C00303F50050817C92F8572B914200D3B3
:108310008674417C29B1817C0174417C491E817441
:108320004674817C01EB011103EBC10101F50051A1
:108330004A7F817C2046F8F7F5F9641CE4B295F891
:10834000AC0AA0423FF6D4AE95F8630720B195F889
:108350003E06012807D010E095F84A0601280CD106
:1083600085F84A6601E085F83E6695F8662795F837
:10837000621795F86307FCF777F9F2F7F3FB95F8C6
:10838000650718B185F86567FAF710FDBDE8F04795
:10839000FEF7CABAD42200202DE9FE4F01210024A5
:1083A0000846FDF73DFFA720ADF80000002540F28C
:1083B000E73001904FF0804AADF80250ADF8085018
:1083C00069465046FFF70EFE854880F87E5741F219
:1083D000706C41F6B02844F24029A0F5805642F274
:1083E000240704EB440106EB810190F87E2701EBA2
:1083F0000C0306EB820202F58052C2F8803790F837
:108400007E27521C80F87E2790F87E3701F5D752E0
:1084100006EB830303F58053C3F8802790F87E278B
:10842000521C80F87E2790F87E2701EB080306EBAC
:10843000820202F58052C2F8803790F87E27521CE3
:1084400080F87E2701EB090290F87E1706EB810188
:1084500001F58051C1F8802790F87E17491C80F8FB
:108460007E1704EB041202EB0422002106EBC20586
:1084700001EB011205EBC20290F87E373A4406EB9D
:10848000830303F58053C3F8802790F87E27521C9E
:1084900080F87E27491CC9B21029E9D3641CE4B2D4
:1084A000042C9ED34F4A90F87E1706EB810101F50C
:1084B0008051C1F8802790F87E17491C80F87E17FC
:1084C00090F87E17283A06EB810101F58051C1F83A
:1084D000802790F87E17491C80F87E1790F87E1749
:1084E0000C3206EB810101F58051C1F8802790F82C
:1084F0007E17491C80F87E1790F87E170C3206EB29
:10850000810101F58051C1F8802790F87E17491C40
:1085100080F87E1790F87E1702F58A7206EB8101CB
:1085200001F58051C1F8802790F87E17491C80F82A
:108530007E1702F54E7190F87E2706EB820202F557
:108540008052C2F8801790F87E17491C80F87E1779
:10855000244A90F87E17343A06EB810101F58051E8
:10856000C1F8802790F87E17491C80F87E171E4AB4
:1085700090F87E1706EB810101F58051C1F8802744
:1085800090F87E17491C80F87E17184990F87E27CE
:1085900006EB820202F58052C2F8801790F87E172F
:1085A000491C80F87E17104A90F87E170C3A06EBAB
:1085B000810101F58051C1F8802790F87E17491C90
:1085C00080F87E17012154465046FFF744FC0122F3
:1085D00011462046FFF7FEFC00F00AF8BDE8FE8FCA
:1085E000D42200203829002050550020DC12002021
:1085F00008B51C208DF8000001208DF80100022133
:108600008DF802108DF803006846FAF773F808BD7C
:10861000F9F734BAF9F752BAFCF7F6BCF9F708BA29
:10862000F9F76CBAF2F70EB8C94301807047002918
:10863000818902D041F4005101E021F4005181818F
:108640007047002A828A01D00A4300E08A4382826E
:10865000704700001C4910B5884206D10121102046
:10866000FDF702FE0021102028E01849884202D1BF
:1086700001214C0410E01649884202D101218C04EA
:108680000AE01449884202D10121CC0404E01249D5
:1086900088420AD101210C052046FDF7CDFD204678
:1086A000BDE810400021FDF7C7BD0C49884209D143
:1086B00001212020FDF7D8FD00212020BDE8104039
:1086C000FDF7D2BD10BD0000001001400044004085
:1086D00000480040004C00400050004000140140A1
:1086E0000246002012880A4200D00120704770B56F
:1086F00001F01F0501260024C1F3421306FA05F21A
:10870000012B0FD0022B0FD0838A4FEA1121008852
:10871000134206FA01F600EA060001D000B1012476
:10872000204670BD8389F0E7038AEEE710B5C1F3F8
:10873000421301F01F040121A140012B07D0022B9D
:1087400007D01430002A026805D00A4304E00C3038
:10875000F8E71030F6E78A43026010BD7FB50446A3
:10876000008A0D46C98820F4405001432182A08927
:1087700041F20C618843A9882A8911436A8902431E
:108780001143A181A08A20F44071A8890843A082E6
:108790006846FDF775FD1A48844202D019488442A4
:1087A00001D1039800E00298A189090400EBC001FF
:1087B00001EB0010296801D5490000E08900B0FBF9
:1087C000F1F06422B0FBF2F109010B096FF018051A
:1087D0006B4300EB8300A3891D044FF0320306D5E1
:1087E00003EBC000B0FBF2F000F0070005E003EB84
:1087F0000010B0FBF2F000F00F00084320817FBDB5
:10880000001001400014014070B50024064DFDF732
:10881000DBFC20B1641CAC42F9D3FA2070BDBDE88A
:108820007040F0F737BE0000404B4C000FB4084BCF
:1088300010B504A902AA039801F0E2F9044602A9BE
:10884000002001F008FC204610BC5DF814FB00007D
:1088500057A0010803B401984100009850EAC120D4
:1088600018BF04204A0D18BF40F0010040F2FF720B
:10887000B2EB515F08BF40F00200012808BF05209D
:1088800002B070470000000030B583B0044601F02C
:1088900093F99FED090B05468DED000B0022214653
:1088A0006846EFF77AFF284601F09CF99DED000B32
:1088B00003B030BD00000000000000000000000018
:1088C00070B5D94B00242DED020B2DED108BDDE999
:1088D0001010984205DA20F000429A4201D809D1DE
:1088E00041B19DED100BBDEC108B02B0BDE87040A6
:1088F00001F01EB9B0F5801F26DA11430BD0002815
:1089000013DA012001F06EF9BDEC108B02B0BDE866
:10891000704001F021B9022001F064F901F0F0F893
:1089200051EC100B81F000419EE06FF035049FED9B
:10893000C00B53EC102B9DED100B51EC100BEFF70F
:108940005FFDCDE91001084604EB2051C0F313048C
:10895000B948A1F2FF31204400F4801080F07F621A
:1089600082F04052224301EB20559FEDB50B11924E
:1089700053EC102B9DED100B51EC100BEFF73AFD63
:1089800041EC180BA01CC0F313009FEDAFDB9FED73
:10899000B0EBB14E7E4403286CD296ED000B51EC47
:1089A000180B53EC102BF0F739FA1DD1002D01BF35
:1089B00096ED000BBDEC108B02B070BD2846EFF7B2
:1089C000CAFF41EC180B53EC1D2BEFF719FD41ECDE
:1089D000190B53EC1E2B51EC180BEFF711FD53EC58
:1089E000192BEFF766FC3FE09FED9D0B51EC180B48
:1089F00053EC102BEFF704FD9FED9B1B53EC112B59
:108A0000EFF7FBFC41EC190B53EC182B51EC180B56
:108A1000EFF7F6FC53EC192BEFF7F2FC41EC190BD6
:108A2000002D04BF53EC192B51EC180B1AD028461B
:108A3000EFF791FF41EC1A0B53EC1D2BEFF7E0FC25
:108A400053EC192BEFF7D9FC53EC182BEFF7D2FCB2
:108A500041EC180B53EC1E2B51EC1A0BEFF7D0FC2A
:108A600053EC182BEFF7C6FCBDEC108B02B041ECB9
:108A7000100B70BD9FED7E0B51EC180B53EC102BBF
:108A8000EFF717FC41EC100B51EC180B53EC102BCB
:108A9000EFF728FD41EC190B2846EFF75CFF41EC9E
:108AA0001B0B53EC192B51EC190BEFF7A9FC41EC04
:108AB0001A0B714853EC1A2B261851EC1A0BEFF7CE
:108AC0009FFC41EC1F0B6D48C4F1510404F5D72401
:108AD000B0EE4F0AF0EE6F0A0321784400F094FFE5
:108AE00053EC1F2B51EC100BEFF78AFC41EC1C0BE5
:108AF0006348B0EE4F0AF0EE6F0A0421784400F0AC
:108B000083FF53EC1A2B51EC100BEFF779FC344335
:108B100053EC1C2BEFF7CDFB41EC1C0B002C4CDD78
:108B20009FED510B51EC180B53EC102BEFF768FC39
:108B300053EC182BEFF764FC41EC1A0B55B353ECD4
:108B40001D2B51EC1B0BEFF75BFC41EC1D0B53ECA9
:108B50001C2B51EC1A0BEFF7ACFB53EC192BEFF776
:108B60004FFC53EC1D2BEFF7A4FB53EC1A2BEFF744
:108B700044FC53EC182BEFF73DFC41EC180B53EC85
:108B80001E2B51EC1B0BEFF73BFC53EC182BEFF7B4
:108B900031FC69E753EC1C2B51EC1A0BEFF789FB06
:108BA00053EC192BEFF72CFC53EC1A2BEFF725FCA9
:108BB00053EC182BEFF721FC56E735B353EC1D2B84
:108BC00051EC1B0BEFF71CFC41EC1A0B53EC1C2B6C
:108BD00051EC180BEFF70EFC53EC192BEFF710FCD0
:108BE00053EC1A2BEFF706FC53EC182BEFF702FCB3
:108BF00041EC180B53EC1E2B51EC1B0BEFF700FC58
:108C000053EC182BEFF7F6FB2EE753EC1C2B51EC33
:108C1000180BEFF7EFFB53EC192BEFF7F1FB53ECCD
:108C2000182BEFF7EAFB1FE70000F07F00000000C1
:108C30000000000000005043645F090000000000D5
:108C4000000000000000F03F763C7935EF39EA3D46
:108C50000000E0FE422EE63F00460000000000005B
:108C6000555555555555D53F000000000000E03FD3
:108C7000000000000000004086EBF9FF8244000085
:108C8000784400000000000070B5414A00252DED39
:108C9000020B2DED048BDDE90404944205DA24F087
:108CA0000041914201D809D140B19DED040BBDECCA
:108CB000048B02B0BDE8704000F03ABFB4F5801FED
:108CC00026DA08430BD0002C13DA012000F08AFFCB
:108CD000BDEC048B02B0BDE8704000F03DBF022047
:108CE00000F080FF00F00CFF51EC100B81F0004110
:108CF00046E09FED290B6FF0350553EC102B9DEDF1
:108D0000040B51EC100BEFF77BFBCDE904010C4693
:108D100005EB2450A0F2FF30C10F40F2FF32521A8F
:108D200062F31F540844EFF716FE05949DED040B03
:108D300041EC180B51EC100B01F0C6FA9FED181B1B
:108D400053EC112BEFF75CFB9FED170B41EC190B6C
:108D500053EC102B51EC180BEFF752FB53EC192B83
:108D6000EFF7A7FA9FED120B41EC190B53EC102B08
:108D700051EC180BEFF744FB53EC192BEFF799FA72
:108D8000BDEC048B02B041EC100B70BD0000000084
:108D90000000F07F000000000000000000005043D1
:108DA0000EE526157BCBDB3F362BF111F3FE593D4B
:108DB00000609F501344D33F2DE9F04D2DED040B7F
:108DC0002DED0E8B96B0DDE92550279CDDF890A0A7
:108DD00025F0004624F00048BAF1000F14BF01212D
:108DE000002101EB4502FC4953184A1093422AD353
:108DF000002814BF0123002303EB44030B44F7496D
:108E00008B4220D358EA00019FEDF59B76D0DFF826
:108E1000D8B35D4503D1BAF1000F05D188E0BAF1AE
:108E2000000F08BF002100D0012101EB450111F521
:108E3000001F08D8002814BF0121002101EB4401C4
:108E400011F5001F0BD99DED261B9DED240B16B0CF
:108E5000BDEC0E8B04B0BDE8F04D00F073BE0027F2
:108E6000002DBCBFE149884521DAE1498845A8BF0A
:108E700002271CDAC3451ADCDE4901EB285114290C
:108E800008DDC1F1340220FA02F101FA02F2824255
:108E90000DD108E058B9C1F1140228FA02F101FA23
:108EA00002F2424503D101F00101C1F1020756EA85
:108EB0000A0124D1002C22DA002D18BF022F01D084
:108EC000012F0AD0022000F08DFE16B0BDEC0E8BF3
:108ED00004B0BDE8F04D00F013BE022000F082FEA9
:108EE00000F00EFE51EC100B81F0004141EC100B34
:108EF00016B0BDEC0E8B04B0BDE8F08D18E09FED10
:108F0000BEAB9FEDBF8B002871D1B848804522D100
:108F100005F1804010F5801008BFBAF1000F07D0AE
:108F2000B3450ADC002CA8BF9DED260BE0DA0DE06E
:108F3000B0EE490AF0EE690ADAE7002C06DA9DED98
:108F4000260B51EC100B81F000416FE0AE487844E5
:108F500090ED000BCCE7D8454DD1002C48DA2EB16E
:108F600086423AD1BAF1000F42D126E0BAF1000FA1
:108F700013D0022000F036FE00F0FEFD8DED020B56
:108F80009DED240B8DED000B10EE900A039961F31B
:108F90001E0003909DED020BAAE78DED02AB9DED47
:108FA000240B1AEE901A10EE900A8DED000B61F36F
:108FB0001E0003909DED020B9AE78DED028B9DED57
:108FC000240B18EE901A10EE900A8DED000B61F351
:108FD0001E0003909DED020B8AE709DA9DED240B3C
:108FE00051EC190B53EC102BEFF77CFA1EE020E04C
:108FF0009DED240B7CE786421BDAB4F1804F0DD047
:10900000A4F10050B0F1FF5013D1002D11DB9DED04
:10901000240B51EC100B01F0E2F907E09DED240B5D
:1090200053EC102B51EC100B00F0C2BC41EC100BB8
:109030005EE79DED240B51EC100B01F039F8BAF10D
:10904000000FCDE90E0142D19FED710B46B3A6F1A1
:10905000E040B0F17F600CD05E4538D1002D00DAE1
:10906000A7B3022F0CBF01204FF0FF30EFF773FCC6
:10907000DCE7002D01DD002C0DDA002D01DD002CD8
:109080001FDB002D16DA002C14DB012F08BF9FED2B
:10909000620B3FF42DAFB0EE4A0AF0EE6A0A27E702
:1090A000022F18BF002D0CD0012F0AD1002DFFF682
:1090B0001FAF06E0002DB8BF002C08DA012F3FF4E7
:1090C00017AFB0EE480AF0EE680A11E71BE0012086
:1090D00000EBE57050EA070115D0791EB0EE498A21
:1090E000F0EE698A084308BF9FED4D8B4E4800257E
:1090F000804570DD4D494E48884514DDB0420DDB9A
:10910000002C19DB2FE0012000F06CFD16B0BDEC47
:109110000E8B04B0BDE8F04D00F01EBDB34502DC7F
:10912000002C09DC1FE0864202DA002C1BDA03E087
:109130005E452BDD002C16DD022000F053FD00F013
:109140001BFD8DED020B53EC1A2B51EC180BEFF7B6
:1091500057F9CDE900010399019861F31E000390CE
:109160009DED020BC4E6022000F03CFD00F014FD72
:1091700010EE901A18EE900A8DED020B8DED008B1B
:1091800061F31E0003909DED020BB1E69DED0E0B09
:1091900053EC192B51EC100BEFF72CF99FED260B2C
:1091A000CDE9080153EC102B9DED080B51EC100B91
:1091B000EFF726F99FED221B53EC112BEFF71DF96A
:1091C0009DED081B53EC112BEFF71AF99FED1E1BB9
:1091D00053EC112B3CE08CE0FFFF1F00FFFF0F0062
:1091E000000000000000F03F0000F03F0000F07FB2
:1091F0000000404301FCFFFF000000000000F07F82
:1092000000000000000000004640000000000000D8
:109210000000000000000080000000000000F0FFDF
:10922000000000000000F0BF0000E0410000F0433B
:10923000FFFFEF3F00000000000000000000D03FF3
:10924000555555555555D53F000000000000E03FED
:10925000EFF7D3F89DED080B41EC1A0B53EC102BF4
:1092600051EC100BEFF7CCF853EC1A2BEFF7C8F8D2
:1092700041EC1A0B9FEDFE0B53EC102B9DED080BF0
:1092800051EC100BEFF7BCF841EC1B0B9FEDFA0B08
:1092900051EC1A0B53EC102BEFF7B2F841EC1A0B10
:1092A0009FEDF70B53EC102B9DED080B51EC100BC1
:1092B000EFF7A6F853EC1A2BEFF79CF841EC1A0BDA
:1092C00051EC1B0B53EC1A2BEEF7F3FF0690CDE994
:1092D00006519DED060B53EC1B2B51EC100BEFF7D9
:1092E00089F853EC1A2BEFF788F841EC100B00F0DB
:1092F000A1B90020B6F5801F0EDA9FEDE30B53EC09
:10930000102B9DED0E0B51EC100BEFF779F8CDE91A
:109310000E016FF034000E4600EB2650A0F2FF372E
:10932000C6F31300DA4940F07F6646F040568842A3
:10933000D8BF002408DDD7498142C8BF012403DC1F
:109340000024A6F580167F1CD348784400EBC400A7
:109350000F9690ED00CB9DED0E0B53EC1C2B51ECBA
:10936000100BEFF747F89DED0E0B41EC1B0B53EC88
:109370001C2B51EC100BEEF79CFF41EC100B51EC49
:10938000190B53EC102BEFF7ADF841EC1D0B51EC22
:109390001B0B53EC1D2BEFF733F841EC1A0BBF48B6
:1093A0008DED10AB7844109590ED000B4FF0005010
:1093B00040EA660000EB84408DED080B00F50020CC
:1093C00009909DED080B53EC1C2B51EC100BEFF7A3
:1093D00011F89DED0E1B53EC112BEFF70EF841EC3D
:1093E000100B53EC102B9DED100B51EC100BEFF705
:1093F00007F89DED080B41EC1C0B53EC102B9DED79
:10940000100B51EC100BEEF7FBFF53EC1B2BEEF7A0
:10941000F4FF53EC1C2BEEF7EDFF53EC1D2BEEF796
:10942000EFFF41EC1C0B53EC1A2B51EC1A0BEEF72F
:10943000E7FF41EC1B0B9A480621B0EE4B0AF0EE19
:109440006B0A784400F0E0FAB0EE401AF0EE601AD1
:10945000B0EE41DAF0EE61DA53EC1B2B51EC1B0B52
:10946000EEF7CEFF53EC1D2BEEF7CAFF9DED100B70
:1094700041EC1B0B53EC1A2B51EC100BEEF719FFC0
:1094800053EC1C2BEEF7BCFF53EC1B2BEEF711FF3C
:109490009DED100B41EC1B0B53EC102B51EC100B02
:1094A000EEF7AEFF41EC1D0B9FED7FEB53EC1E2B57
:1094B000EEF7FFFE53EC1B2BEEF7FBFE0890CDE919
:1094C00008519DED080B53EC1E2B51EC100BEEF7E1
:1094D00091FF53EC1D2BEEF78DFF53EC1B2BEEF79A
:1094E0008CFF9DED080B41EC1D0B53EC102B9DEDFB
:1094F000100B51EC100BEEF783FF41EC1B0B53EC00
:109500001A2B51EC1D0BEEF77BFF9DED080B41EC88
:109510001A0B53EC102B51EC1C0BEEF771FF53ECB4
:109520001A2BEEF7C6FE41EC1A0B51EC1B0B53EC59
:109530001A2BEEF7BEFE0C90CDE90C519DED0C0BF5
:1095400053EC1B2B51EC100BEEF754FF53EC1A2B82
:10955000EEF753FF41EC1B0B9FED550B53EC102B1B
:109560009DED0C0B51EC100BEEF74AFF41EC1A0B82
:109570009FED510B51EC1B0B53EC102BEEF740FF02
:1095800041EC1B0B9FED4E0B53EC102B9DED0C0B88
:1095900051EC100BEEF734FF53EC1B2BEEF789FE6A
:1095A00041EC100B4848784400EBC40090ED001BE0
:1095B00051EC100B53EC112BEEF77BFE41EC1B0B27
:1095C0003846EFF7C8F9CDE9080153EC1B2B51ECF5
:1095D0001A0BEEF76EFE41EC100B3C48784400EBA2
:1095E000C40090ED00CB51EC100B53EC1C2BEEF7AC
:1095F00060FE9DED081B53EC112BEEF75AFE069012
:10960000CDE906519DED080B53EC102B9DED060B9B
:1096100051EC100BEEF7EEFE53EC1C2BEEF7EAFECE
:1096200053EC1A2BEEF7E6FE53EC1B2BEEF7E5FEA0
:1096300041EC100B9DED261B53EC102B8DED001B08
:1096400000959DED260B51EC100BEEF7D9FE9DED2C
:10965000000B41EC1A0B53EC102B9DED260B51EC3B
:10966000100BEEF7C7FE9DED061B53EC112B2FE000
:10967000000000604715F73FFE822B654715F73F56
:1096800044DF5DF80BAE543E000000000000404394
:109690008E9803007AB60B008A3B0000F03B000076
:1096A000C23A000000000000000000000000084076
:1096B000000000E009C7EE3FFD033ADC09C7EE3FBA
:1096C000F5015B14E02F3EBE4E3900000839000062
:1096D000EEF796FE53EC1A2BEEF7EBFD9DED060B25
:1096E00041EC1A0B53EC102B9DED000B51EC100BC1
:1096F000EEF786FECDE90C019DED0C0B51EC1A0B3B
:1097000053EC102BEEF7D5FDCDE902010C46AA492A
:109710008C422FDB611A084318D19DED0C0B53ECE2
:10972000102B9DED020B51EC100BEEF763FE41EC9C
:109730001B0B9FEDA30B51EC1A0B53EC102BEEF708
:10974000B8FD53EC1B2BEFF717F92DD2022000F0D8
:1097500049FA00F011FA10EE901A18EE900A8DED09
:10976000020B8DED008B61F31E0003909DED020B4B
:10977000FFF7BEBB944A24F00041914214D39349B1
:10978000214408437FF4EFAC9DED0C0B53EC102B00
:109790009DED020B51EC100BEEF72CFE53EC1A2B47
:1097A000EFF7EAF87FF6DFAC24F000408849894AF9
:1097B000002601EB205182422BDA481C4FF4801125
:1097C00021FA00F02044844AC0F30A517A44A1F2FD
:1097D000FF3192ED000B814A8DED080BCA4020EA63
:1097E0000202C0F3130040F48010C1F1140120FA0A
:1097F00001F60992002CB8BF76429DED080B53ECA0
:10980000102B9DED0C0B51EC100BEEF7F3FDCDE999
:109810000C019DED0C0B51EC1A0B53EC102BEEF7D9
:1098200048FD9FED6F0B0890CDE9085153EC102BCC
:109830009DED080B51EC100BEEF7E2FD41EC1B0B1C
:109840009FED690B53EC102B9DED080B51EC100BA9
:10985000EEF7D6FD9DED0C0B41EC1C0B53EC102BE1
:109860009DED080B51EC100BEEF7C4FD53EC1A2BD9
:10987000EEF7C3FD9FED5E1B53EC112BEEF7C0FD21
:1098800053EC1C2BEEF715FD41EC1A0B51EC1B0BA6
:1098900053EC1A2BEEF70DFDCDE902019DED020B05
:1098A00053EC1B2B51EC100BEEF7A4FD53EC1A2BD1
:1098B000EEF7A3FD9DED020B41EC1A0B53EC102BC0
:1098C00051EC100BEEF79CFDCDE908014A489DEDE7
:1098D000080B0521784400F097F89DED081B51EC2A
:1098E000100B53EC112BEEF78BFD9DED021B53EC8F
:1098F000112BEEF782FDCDE906019DED020B53EC35
:109900001A2B51EC100BEEF77BFD53EC1A2BEEF7F4
:10991000D0FC9FED3B0B41EC1A0B53EC102B9DED53
:10992000060B51EC100BEEF765FD9DED060B41ECBF
:109930001B0B53EC102B9DED020B51EC100BEEF7B3
:109940005FFD53EC1B2BEEF7CDFD53EC1A2BEEF71E
:1099500051FD9DED021B53EC112BEEF74BFD53EC2B
:10996000192BEEF74AFDCDE9020101EB0650011576
:109970000029C8BF039015DC9DED020B324651EC67
:10998000100BEEF7D1FFFEF765FF042808BF00F0CB
:1099900003F932469DED020B51EC100BEEF7C4FFBC
:1099A000CDE902019DED020B51EC180B53EC102B8D
:1099B000EEF726FDFFF73ABB0000904000000000E4
:1099C000FE822B654715973C00CC904000346F3FDA
:1099D00001FCFFFF0000E03FC8370000FFFF0F0061
:1099E00000000000432EE63F396CA80C615C20BEED
:1099F000EF39FAFE422EE63F60360000000000001C
:109A0000000000000000004070B504462DED028B00
:109A10004D1E00EBC500B0EE408AF0EE608A90ED7E
:109A2000000B35F0060017D053EC182B51EC100B3F
:109A3000EEF7E6FC41EC100B6D1E04EBC50090ED5B
:109A4000001B51EC100B53EC112BEEF732FC41ECE8
:109A5000100B35F00600E7D1022D36D0042D1CD0B6
:109A6000062D1CBFBDEC028B70BD53EC182B51ECC6
:109A7000100BEEF7C5FC94ED0A1B53EC112BEEF71F
:109A800018FC53EC182BEEF7BBFC94ED081B53ECC1
:109A9000112BEEF70EFC41EC100B53EC182B51EC94
:109AA000100BEEF7ADFC94ED061B53EC112BEEF70B
:109AB00000FC53EC182BEEF7A3FC94ED040B53ECD5
:109AC000102BEEF7F6FB41EC100B53EC182B51EC7E
:109AD000100BEEF795FC94ED021B53EC112BEEF7F7
:109AE000E8FB53EC182BEEF78BFC94ED001B53ECCA
:109AF000112BEEF7DEFBBDEC028B41EC100B70BDC1
:109B00009FED070B10B553EC102B9FED070B51EC9D
:109B1000100BEEF7E7FC41EC100B10BD000000004D
:109B20000000000000000000000000000000F03F06
:109B300010B553EC102B51EC100BEEF7BAFB41ECC7
:109B4000100B10BD10B553EC112B51EC100BEEF7B0
:109B5000B0FB41EC100B10BD9FED050B10B553ECA5
:109B6000102B51EC100BEEF7BDFC41EC100B10BDAF
:109B700000000000000000009FED050B10B553EC45
:109B8000102B51EC100BEEF73BFC41EC100B10BD11
:109B900000000000000000709FED050B10B553ECB5
:109BA000102B51EC100BEEF72BFC41EC100B10BD01
:109BB000000000000000001001480068704700002D
:109BC000D012002002E008C8121F08C1002AFAD1F2
:109BD00070477047002001E001C1121F002AFBD12D
:109BE000704700000149086070470000D012002053
:109BF00030380A2801D20120704700207047000049
